
StellarisFilter.elf:     file format elf32-littlearm

Sections:
Idx Name          Size      VMA       LMA       File off  Algn
  0 .text         00002340  00000000  00000000  00008000  2**2
                  CONTENTS, ALLOC, LOAD, READONLY, CODE
  1 .data         00000800  20000000  00002400  00010000  2**10
                  CONTENTS, ALLOC, LOAD, DATA
  2 .bss          00000528  20000800  00002c00  00010800  2**2
                  ALLOC
  3 .debug_info   00003045  00000000  00000000  00010800  2**0
                  CONTENTS, READONLY, DEBUGGING
  4 .debug_abbrev 00000a24  00000000  00000000  00013845  2**0
                  CONTENTS, READONLY, DEBUGGING
  5 .debug_loc    0000275a  00000000  00000000  00014269  2**0
                  CONTENTS, READONLY, DEBUGGING
  6 .debug_aranges 000006f8  00000000  00000000  000169c3  2**0
                  CONTENTS, READONLY, DEBUGGING
  7 .debug_ranges 00000668  00000000  00000000  000170bb  2**0
                  CONTENTS, READONLY, DEBUGGING
  8 .debug_macro  0000b18f  00000000  00000000  00017723  2**0
                  CONTENTS, READONLY, DEBUGGING
  9 .debug_line   00001ea8  00000000  00000000  000228b2  2**0
                  CONTENTS, READONLY, DEBUGGING
 10 .debug_str    0003941f  00000000  00000000  0002475a  2**0
                  CONTENTS, READONLY, DEBUGGING
 11 .comment      0000003a  00000000  00000000  0005db79  2**0
                  CONTENTS, READONLY
 12 .ARM.attributes 00000035  00000000  00000000  0005dbb3  2**0
                  CONTENTS, READONLY
 13 .debug_frame  000016a0  00000000  00000000  0005dbe8  2**2
                  CONTENTS, READONLY, DEBUGGING

Disassembly of section .text:

00000000 <_start_text>:
       0:	20008000 	.word	0x20008000
       4:	0000026d 	.word	0x0000026d
       8:	000002dd 	.word	0x000002dd
       c:	00000321 	.word	0x00000321
      10:	00000339 	.word	0x00000339
      14:	00000339 	.word	0x00000339
      18:	00000339 	.word	0x00000339
	...
      2c:	00000339 	.word	0x00000339
      30:	00000339 	.word	0x00000339
      34:	00000000 	.word	0x00000000
      38:	00000339 	.word	0x00000339
      3c:	000012b9 	.word	0x000012b9
      40:	00000339 	.word	0x00000339
      44:	00000339 	.word	0x00000339
      48:	00000339 	.word	0x00000339
      4c:	00000339 	.word	0x00000339
      50:	00000339 	.word	0x00000339
      54:	00000d65 	.word	0x00000d65
      58:	00000339 	.word	0x00000339
      5c:	00000339 	.word	0x00000339
      60:	00000339 	.word	0x00000339
	...
      78:	00000339 	.word	0x00000339
      7c:	00000339 	.word	0x00000339
      80:	00000339 	.word	0x00000339
      84:	00000339 	.word	0x00000339
      88:	00000339 	.word	0x00000339
      8c:	00000339 	.word	0x00000339
      90:	00000339 	.word	0x00000339
      94:	00000339 	.word	0x00000339
      98:	00000339 	.word	0x00000339
      9c:	00000339 	.word	0x00000339
      a0:	00000339 	.word	0x00000339
      a4:	00000339 	.word	0x00000339
      a8:	00000339 	.word	0x00000339
      ac:	00000000 	.word	0x00000000
      b0:	00000339 	.word	0x00000339
      b4:	00000339 	.word	0x00000339
      b8:	00000339 	.word	0x00000339
	...
      c4:	00000339 	.word	0x00000339
      c8:	00000339 	.word	0x00000339
      cc:	00000339 	.word	0x00000339
      d0:	00000339 	.word	0x00000339
      d4:	00000339 	.word	0x00000339
      d8:	00000000 	.word	0x00000000
      dc:	00000339 	.word	0x00000339
	...
      ec:	00000339 	.word	0x00000339
      f0:	00000339 	.word	0x00000339
      f4:	00000000 	.word	0x00000000
      f8:	00000339 	.word	0x00000339
      fc:	00000339 	.word	0x00000339
     100:	00000339 	.word	0x00000339
     104:	00000339 	.word	0x00000339
     108:	00000339 	.word	0x00000339
     10c:	00000339 	.word	0x00000339
	...
     124:	00000339 	.word	0x00000339
     128:	00000339 	.word	0x00000339
     12c:	00000339 	.word	0x00000339
     130:	00000339 	.word	0x00000339
     134:	00000339 	.word	0x00000339
     138:	00000339 	.word	0x00000339
     13c:	00000339 	.word	0x00000339
	...
     150:	00000339 	.word	0x00000339
     154:	00000339 	.word	0x00000339
     158:	00000339 	.word	0x00000339
     15c:	00000339 	.word	0x00000339
	...
     1b0:	00000339 	.word	0x00000339
     1b4:	00000339 	.word	0x00000339
     1b8:	00000339 	.word	0x00000339
     1bc:	00000339 	.word	0x00000339
     1c0:	00000339 	.word	0x00000339
     1c4:	00000339 	.word	0x00000339
     1c8:	00000339 	.word	0x00000339
     1cc:	00000339 	.word	0x00000339
     1d0:	00000339 	.word	0x00000339
     1d4:	00000339 	.word	0x00000339
     1d8:	00000339 	.word	0x00000339
     1dc:	00000339 	.word	0x00000339
     1e0:	00000339 	.word	0x00000339
     1e4:	00000339 	.word	0x00000339
     1e8:	00000339 	.word	0x00000339
	...

0000026c <rst_handler>:
* The stack pointer should be set at the beginning with the NVIC table already.
* Copy the .data segment from flash into ram.
* 0 to the .bss segment 
*/
	
void rst_handler(void){	
     26c:	b580      	push	{r7, lr}
     26e:	b082      	sub	sp, #8
     270:	af00      	add	r7, sp, #0
	// source and destination pointers
	unsigned long *src;
	unsigned long *dest;
	
	//this should be good!
	src = &_end_text;
     272:	f242 3340 	movw	r3, #9024	; 0x2340
     276:	f2c0 0300 	movt	r3, #0
     27a:	607b      	str	r3, [r7, #4]
	dest = &_start_data;
     27c:	f240 0300 	movw	r3, #0
     280:	f2c2 0300 	movt	r3, #8192	; 0x2000
     284:	603b      	str	r3, [r7, #0]
	
	//this too
    while(dest < &_end_data)
     286:	e009      	b.n	29c <rst_handler+0x30>
    {
        *dest++ = *src++;
     288:	687b      	ldr	r3, [r7, #4]
     28a:	681a      	ldr	r2, [r3, #0]
     28c:	683b      	ldr	r3, [r7, #0]
     28e:	601a      	str	r2, [r3, #0]
     290:	683b      	ldr	r3, [r7, #0]
     292:	3304      	adds	r3, #4
     294:	603b      	str	r3, [r7, #0]
     296:	687b      	ldr	r3, [r7, #4]
     298:	3304      	adds	r3, #4
     29a:	607b      	str	r3, [r7, #4]
	//this should be good!
	src = &_end_text;
	dest = &_start_data;
	
	//this too
    while(dest < &_end_data)
     29c:	683a      	ldr	r2, [r7, #0]
     29e:	f640 0300 	movw	r3, #2048	; 0x800
     2a2:	f2c2 0300 	movt	r3, #8192	; 0x2000
     2a6:	429a      	cmp	r2, r3
     2a8:	d3ee      	bcc.n	288 <rst_handler+0x1c>
    {
        *dest++ = *src++;
    }
	
    // now set the .bss segment to 0!
    dest = &_start_bss;
     2aa:	f640 0300 	movw	r3, #2048	; 0x800
     2ae:	f2c2 0300 	movt	r3, #8192	; 0x2000
     2b2:	603b      	str	r3, [r7, #0]
	while(dest < &_end_bss){
     2b4:	e005      	b.n	2c2 <rst_handler+0x56>
		*dest++ = 0;
     2b6:	683b      	ldr	r3, [r7, #0]
     2b8:	2200      	movs	r2, #0
     2ba:	601a      	str	r2, [r3, #0]
     2bc:	683b      	ldr	r3, [r7, #0]
     2be:	3304      	adds	r3, #4
     2c0:	603b      	str	r3, [r7, #0]
        *dest++ = *src++;
    }
	
    // now set the .bss segment to 0!
    dest = &_start_bss;
	while(dest < &_end_bss){
     2c2:	683a      	ldr	r2, [r7, #0]
     2c4:	f640 5328 	movw	r3, #3368	; 0xd28
     2c8:	f2c2 0300 	movt	r3, #8192	; 0x2000
     2cc:	429a      	cmp	r2, r3
     2ce:	d3f2      	bcc.n	2b6 <rst_handler+0x4a>
	}
	
	// after setting copying .data to ram and "zero-ing" .bss we are good
	// to start the main() method!
	// There you go!
	main();
     2d0:	f000 ff64 	bl	119c <main>
}
     2d4:	f107 0708 	add.w	r7, r7, #8
     2d8:	46bd      	mov	sp, r7
     2da:	bd80      	pop	{r7, pc}

000002dc <nmi_handler>:

// NMI Exception handler code NVIC 2
void nmi_handler(void){
     2dc:	b480      	push	{r7}
     2de:	af00      	add	r7, sp, #0
	// Just loop forever, so if you want to debug the processor it's running.
    while(1){
    }
     2e0:	e7fe      	b.n	2e0 <nmi_handler+0x4>
     2e2:	bf00      	nop

000002e4 <prvGetRegistersFromStack>:
}

typedef int uint32_t;

void prvGetRegistersFromStack( uint32_t *pulFaultStackAddress ) {
     2e4:	b480      	push	{r7}
     2e6:	b08b      	sub	sp, #44	; 0x2c
     2e8:	af00      	add	r7, sp, #0
     2ea:	6078      	str	r0, [r7, #4]
volatile uint32_t r12;
volatile uint32_t lr; /* Link register. */
volatile uint32_t pc; /* Program counter. */
volatile uint32_t psr;/* Program status register. */

    r0 = pulFaultStackAddress[ 0 ];
     2ec:	687b      	ldr	r3, [r7, #4]
     2ee:	681b      	ldr	r3, [r3, #0]
     2f0:	627b      	str	r3, [r7, #36]	; 0x24
    r1 = pulFaultStackAddress[ 1 ];
     2f2:	687b      	ldr	r3, [r7, #4]
     2f4:	685b      	ldr	r3, [r3, #4]
     2f6:	623b      	str	r3, [r7, #32]
    r2 = pulFaultStackAddress[ 2 ];
     2f8:	687b      	ldr	r3, [r7, #4]
     2fa:	689b      	ldr	r3, [r3, #8]
     2fc:	61fb      	str	r3, [r7, #28]
    r3 = pulFaultStackAddress[ 3 ];
     2fe:	687b      	ldr	r3, [r7, #4]
     300:	68db      	ldr	r3, [r3, #12]
     302:	61bb      	str	r3, [r7, #24]

    r12 = pulFaultStackAddress[ 4 ];
     304:	687b      	ldr	r3, [r7, #4]
     306:	691b      	ldr	r3, [r3, #16]
     308:	617b      	str	r3, [r7, #20]
    lr = pulFaultStackAddress[ 5 ];
     30a:	687b      	ldr	r3, [r7, #4]
     30c:	695b      	ldr	r3, [r3, #20]
     30e:	613b      	str	r3, [r7, #16]
    pc = pulFaultStackAddress[ 6 ];
     310:	687b      	ldr	r3, [r7, #4]
     312:	699b      	ldr	r3, [r3, #24]
     314:	60fb      	str	r3, [r7, #12]
    psr = pulFaultStackAddress[ 7 ];
     316:	687b      	ldr	r3, [r7, #4]
     318:	69db      	ldr	r3, [r3, #28]
     31a:	60bb      	str	r3, [r7, #8]

    /* When the following line is hit, the variables contain the register values. */
    for( ;; );
     31c:	e7fe      	b.n	31c <prvGetRegistersFromStack+0x38>
     31e:	bf00      	nop

00000320 <HardFault_Handler>:

/* The fault handler implementation calls a function called
prvGetRegistersFromStack(). */
static void HardFault_Handler(void)
{
    __asm volatile
     320:	f01e 0f04 	tst.w	lr, #4
     324:	bf0c      	ite	eq
     326:	f3ef 8008 	mrseq	r0, MSP
     32a:	f3ef 8009 	mrsne	r0, PSP
     32e:	6981      	ldr	r1, [r0, #24]
     330:	4a00      	ldr	r2, [pc, #0]	; (334 <handler2_address_const>)
     332:	4710      	bx	r2

00000334 <handler2_address_const>:
     334:	000002e5 	.word	0x000002e5

00000338 <empty_def_handler>:
    while(1){
    }
}

// Empty handler used as default.
void empty_def_handler(void){
     338:	b480      	push	{r7}
     33a:	af00      	add	r7, sp, #0
	// Just loop forever, so if you want to debug the processor it's running.
    while(1){
    }
     33c:	e7fe      	b.n	33c <empty_def_handler+0x4>
     33e:	bf00      	nop

00000340 <IsBufferFull>:
//*****************************************************************************
#ifdef UART_BUFFERED
static tBoolean
IsBufferFull(volatile unsigned long *pulRead,
             volatile unsigned long *pulWrite, unsigned long ulSize)
{
     340:	b480      	push	{r7}
     342:	b087      	sub	sp, #28
     344:	af00      	add	r7, sp, #0
     346:	60f8      	str	r0, [r7, #12]
     348:	60b9      	str	r1, [r7, #8]
     34a:	607a      	str	r2, [r7, #4]
    unsigned long ulWrite;
    unsigned long ulRead;

    ulWrite = *pulWrite;
     34c:	68bb      	ldr	r3, [r7, #8]
     34e:	681b      	ldr	r3, [r3, #0]
     350:	617b      	str	r3, [r7, #20]
    ulRead = *pulRead;
     352:	68fb      	ldr	r3, [r7, #12]
     354:	681b      	ldr	r3, [r3, #0]
     356:	613b      	str	r3, [r7, #16]

    return((((ulWrite + 1) % ulSize) == ulRead) ? true : false);
     358:	697b      	ldr	r3, [r7, #20]
     35a:	3301      	adds	r3, #1
     35c:	687a      	ldr	r2, [r7, #4]
     35e:	fbb3 f2f2 	udiv	r2, r3, r2
     362:	6879      	ldr	r1, [r7, #4]
     364:	fb01 f202 	mul.w	r2, r1, r2
     368:	1a9a      	subs	r2, r3, r2
     36a:	693b      	ldr	r3, [r7, #16]
     36c:	429a      	cmp	r2, r3
     36e:	bf14      	ite	ne
     370:	2300      	movne	r3, #0
     372:	2301      	moveq	r3, #1
     374:	b2db      	uxtb	r3, r3
}
     376:	4618      	mov	r0, r3
     378:	f107 071c 	add.w	r7, r7, #28
     37c:	46bd      	mov	sp, r7
     37e:	bc80      	pop	{r7}
     380:	4770      	bx	lr
     382:	bf00      	nop

00000384 <IsBufferEmpty>:
//*****************************************************************************
#ifdef UART_BUFFERED
static tBoolean
IsBufferEmpty(volatile unsigned long *pulRead,
              volatile unsigned long *pulWrite)
{
     384:	b480      	push	{r7}
     386:	b085      	sub	sp, #20
     388:	af00      	add	r7, sp, #0
     38a:	6078      	str	r0, [r7, #4]
     38c:	6039      	str	r1, [r7, #0]
    unsigned long ulWrite;
    unsigned long ulRead;

    ulWrite = *pulWrite;
     38e:	683b      	ldr	r3, [r7, #0]
     390:	681b      	ldr	r3, [r3, #0]
     392:	60fb      	str	r3, [r7, #12]
    ulRead = *pulRead;
     394:	687b      	ldr	r3, [r7, #4]
     396:	681b      	ldr	r3, [r3, #0]
     398:	60bb      	str	r3, [r7, #8]

    return((ulWrite  == ulRead) ? true : false);
     39a:	68fa      	ldr	r2, [r7, #12]
     39c:	68bb      	ldr	r3, [r7, #8]
     39e:	429a      	cmp	r2, r3
     3a0:	bf14      	ite	ne
     3a2:	2300      	movne	r3, #0
     3a4:	2301      	moveq	r3, #1
     3a6:	b2db      	uxtb	r3, r3
}
     3a8:	4618      	mov	r0, r3
     3aa:	f107 0714 	add.w	r7, r7, #20
     3ae:	46bd      	mov	sp, r7
     3b0:	bc80      	pop	{r7}
     3b2:	4770      	bx	lr

000003b4 <GetBufferCount>:
//*****************************************************************************
#ifdef UART_BUFFERED
static unsigned long
GetBufferCount(volatile unsigned long *pulRead,
               volatile unsigned long *pulWrite, unsigned long ulSize)
{
     3b4:	b480      	push	{r7}
     3b6:	b087      	sub	sp, #28
     3b8:	af00      	add	r7, sp, #0
     3ba:	60f8      	str	r0, [r7, #12]
     3bc:	60b9      	str	r1, [r7, #8]
     3be:	607a      	str	r2, [r7, #4]
    unsigned long ulWrite;
    unsigned long ulRead;

    ulWrite = *pulWrite;
     3c0:	68bb      	ldr	r3, [r7, #8]
     3c2:	681b      	ldr	r3, [r3, #0]
     3c4:	617b      	str	r3, [r7, #20]
    ulRead = *pulRead;
     3c6:	68fb      	ldr	r3, [r7, #12]
     3c8:	681b      	ldr	r3, [r3, #0]
     3ca:	613b      	str	r3, [r7, #16]

    return((ulWrite >= ulRead) ? (ulWrite - ulRead) :
     3cc:	697a      	ldr	r2, [r7, #20]
     3ce:	693b      	ldr	r3, [r7, #16]
     3d0:	429a      	cmp	r2, r3
     3d2:	d303      	bcc.n	3dc <GetBufferCount+0x28>
     3d4:	697a      	ldr	r2, [r7, #20]
     3d6:	693b      	ldr	r3, [r7, #16]
     3d8:	1ad3      	subs	r3, r2, r3
     3da:	e004      	b.n	3e6 <GetBufferCount+0x32>
                                 (ulSize - (ulRead - ulWrite)));
     3dc:	697a      	ldr	r2, [r7, #20]
     3de:	693b      	ldr	r3, [r7, #16]
     3e0:	1ad2      	subs	r2, r2, r3
    unsigned long ulRead;

    ulWrite = *pulWrite;
    ulRead = *pulRead;

    return((ulWrite >= ulRead) ? (ulWrite - ulRead) :
     3e2:	687b      	ldr	r3, [r7, #4]
     3e4:	18d3      	adds	r3, r2, r3
                                 (ulSize - (ulRead - ulWrite)));
}
     3e6:	4618      	mov	r0, r3
     3e8:	f107 071c 	add.w	r7, r7, #28
     3ec:	46bd      	mov	sp, r7
     3ee:	bc80      	pop	{r7}
     3f0:	4770      	bx	lr
     3f2:	bf00      	nop

000003f4 <UARTPrimeTransmit>:
//
//*****************************************************************************
#ifdef UART_BUFFERED
static void
UARTPrimeTransmit(unsigned long ulBase)
{
     3f4:	b580      	push	{r7, lr}
     3f6:	b082      	sub	sp, #8
     3f8:	af00      	add	r7, sp, #0
     3fa:	6078      	str	r0, [r7, #4]
    //
    // Do we have any data to transmit?
    //
    if(!TX_BUFFER_EMPTY)
     3fc:	f640 4008 	movw	r0, #3080	; 0xc08
     400:	f2c2 0000 	movt	r0, #8192	; 0x2000
     404:	f640 4104 	movw	r1, #3076	; 0xc04
     408:	f2c2 0100 	movt	r1, #8192	; 0x2000
     40c:	f7ff ffba 	bl	384 <IsBufferEmpty>
     410:	4603      	mov	r3, r0
     412:	2b00      	cmp	r3, #0
     414:	d160      	bne.n	4d8 <UARTPrimeTransmit+0xe4>
    {
        //
        // Disable the UART interrupt. If we don't do this there is a race
        // condition which can cause the read index to be corrupted.
        //
        MAP_IntDisable(g_ulUARTInt[g_ulPortNum]);
     416:	2348      	movs	r3, #72	; 0x48
     418:	f2c0 1300 	movt	r3, #256	; 0x100
     41c:	681b      	ldr	r3, [r3, #0]
     41e:	330c      	adds	r3, #12
     420:	681b      	ldr	r3, [r3, #0]
     422:	461a      	mov	r2, r3
     424:	f640 4398 	movw	r3, #3224	; 0xc98
     428:	f2c2 0300 	movt	r3, #8192	; 0x2000
     42c:	6819      	ldr	r1, [r3, #0]
     42e:	f242 1394 	movw	r3, #8596	; 0x2194
     432:	f2c0 0300 	movt	r3, #0
     436:	f853 3021 	ldr.w	r3, [r3, r1, lsl #2]
     43a:	4618      	mov	r0, r3
     43c:	4790      	blx	r2

        //
        // Yes - take some characters out of the transmit buffer and feed
        // them to the UART transmit FIFO.
        //
        while(MAP_UARTSpaceAvail(ulBase) && !TX_BUFFER_EMPTY)
     43e:	e020      	b.n	482 <UARTPrimeTransmit+0x8e>
        {
            MAP_UARTCharPutNonBlocking(ulBase,
     440:	2314      	movs	r3, #20
     442:	f2c0 1300 	movt	r3, #256	; 0x100
     446:	681b      	ldr	r3, [r3, #0]
     448:	333c      	adds	r3, #60	; 0x3c
     44a:	681b      	ldr	r3, [r3, #0]
     44c:	461a      	mov	r2, r3
     44e:	f640 4308 	movw	r3, #3080	; 0xc08
     452:	f2c2 0300 	movt	r3, #8192	; 0x2000
     456:	6819      	ldr	r1, [r3, #0]
     458:	f640 0304 	movw	r3, #2052	; 0x804
     45c:	f2c2 0300 	movt	r3, #8192	; 0x2000
     460:	5c5b      	ldrb	r3, [r3, r1]
     462:	6878      	ldr	r0, [r7, #4]
     464:	4619      	mov	r1, r3
     466:	4790      	blx	r2
                                       g_pcUARTTxBuffer[g_ulUARTTxReadIndex]);
            ADVANCE_TX_BUFFER_INDEX(g_ulUARTTxReadIndex);
     468:	f640 4308 	movw	r3, #3080	; 0xc08
     46c:	f2c2 0300 	movt	r3, #8192	; 0x2000
     470:	681b      	ldr	r3, [r3, #0]
     472:	3301      	adds	r3, #1
     474:	f3c3 0209 	ubfx	r2, r3, #0, #10
     478:	f640 4308 	movw	r3, #3080	; 0xc08
     47c:	f2c2 0300 	movt	r3, #8192	; 0x2000
     480:	601a      	str	r2, [r3, #0]

        //
        // Yes - take some characters out of the transmit buffer and feed
        // them to the UART transmit FIFO.
        //
        while(MAP_UARTSpaceAvail(ulBase) && !TX_BUFFER_EMPTY)
     482:	2314      	movs	r3, #20
     484:	f2c0 1300 	movt	r3, #256	; 0x100
     488:	681b      	ldr	r3, [r3, #0]
     48a:	3330      	adds	r3, #48	; 0x30
     48c:	681b      	ldr	r3, [r3, #0]
     48e:	6878      	ldr	r0, [r7, #4]
     490:	4798      	blx	r3
     492:	4603      	mov	r3, r0
     494:	2b00      	cmp	r3, #0
     496:	d00c      	beq.n	4b2 <UARTPrimeTransmit+0xbe>
     498:	f640 4008 	movw	r0, #3080	; 0xc08
     49c:	f2c2 0000 	movt	r0, #8192	; 0x2000
     4a0:	f640 4104 	movw	r1, #3076	; 0xc04
     4a4:	f2c2 0100 	movt	r1, #8192	; 0x2000
     4a8:	f7ff ff6c 	bl	384 <IsBufferEmpty>
     4ac:	4603      	mov	r3, r0
     4ae:	2b00      	cmp	r3, #0
     4b0:	d0c6      	beq.n	440 <UARTPrimeTransmit+0x4c>
        }

        //
        // Reenable the UART interrupt.
        //
        MAP_IntEnable(g_ulUARTInt[g_ulPortNum]);
     4b2:	2348      	movs	r3, #72	; 0x48
     4b4:	f2c0 1300 	movt	r3, #256	; 0x100
     4b8:	681b      	ldr	r3, [r3, #0]
     4ba:	681b      	ldr	r3, [r3, #0]
     4bc:	461a      	mov	r2, r3
     4be:	f640 4398 	movw	r3, #3224	; 0xc98
     4c2:	f2c2 0300 	movt	r3, #8192	; 0x2000
     4c6:	6819      	ldr	r1, [r3, #0]
     4c8:	f242 1394 	movw	r3, #8596	; 0x2194
     4cc:	f2c0 0300 	movt	r3, #0
     4d0:	f853 3021 	ldr.w	r3, [r3, r1, lsl #2]
     4d4:	4618      	mov	r0, r3
     4d6:	4790      	blx	r2
    }
}
     4d8:	f107 0708 	add.w	r7, r7, #8
     4dc:	46bd      	mov	sp, r7
     4de:	bd80      	pop	{r7, pc}

000004e0 <UARTStdioConfig>:
//
//*****************************************************************************
void
UARTStdioConfig(unsigned long ulPortNum, unsigned long ulBaud,
                unsigned long ulSrcClock)
{
     4e0:	b590      	push	{r4, r7, lr}
     4e2:	b085      	sub	sp, #20
     4e4:	af00      	add	r7, sp, #0
     4e6:	60f8      	str	r0, [r7, #12]
     4e8:	60b9      	str	r1, [r7, #8]
     4ea:	607a      	str	r2, [r7, #4]
#endif

    //
    // Check to make sure the UART peripheral is present.
    //
    if(!MAP_SysCtlPeripheralPresent(g_ulUARTPeriph[ulPortNum]))
     4ec:	2344      	movs	r3, #68	; 0x44
     4ee:	f2c0 1300 	movt	r3, #256	; 0x100
     4f2:	681b      	ldr	r3, [r3, #0]
     4f4:	3310      	adds	r3, #16
     4f6:	681b      	ldr	r3, [r3, #0]
     4f8:	461a      	mov	r2, r3
     4fa:	f242 13a0 	movw	r3, #8608	; 0x21a0
     4fe:	f2c0 0300 	movt	r3, #0
     502:	68f9      	ldr	r1, [r7, #12]
     504:	f853 3021 	ldr.w	r3, [r3, r1, lsl #2]
     508:	4618      	mov	r0, r3
     50a:	4790      	blx	r2
     50c:	4603      	mov	r3, r0
     50e:	2b00      	cmp	r3, #0
     510:	f000 8085 	beq.w	61e <UARTStdioConfig+0x13e>
    }

    //
    // Select the base address of the UART.
    //
    g_ulBase = g_ulUARTBase[ulPortNum];
     514:	f242 1388 	movw	r3, #8584	; 0x2188
     518:	f2c0 0300 	movt	r3, #0
     51c:	68fa      	ldr	r2, [r7, #12]
     51e:	f853 2022 	ldr.w	r2, [r3, r2, lsl #2]
     522:	f640 4394 	movw	r3, #3220	; 0xc94
     526:	f2c2 0300 	movt	r3, #8192	; 0x2000
     52a:	601a      	str	r2, [r3, #0]

    //
    // Enable the UART peripheral for use.
    //
    MAP_SysCtlPeripheralEnable(g_ulUARTPeriph[ulPortNum]);
     52c:	2344      	movs	r3, #68	; 0x44
     52e:	f2c0 1300 	movt	r3, #256	; 0x100
     532:	681b      	ldr	r3, [r3, #0]
     534:	3318      	adds	r3, #24
     536:	681b      	ldr	r3, [r3, #0]
     538:	461a      	mov	r2, r3
     53a:	f242 13a0 	movw	r3, #8608	; 0x21a0
     53e:	f2c0 0300 	movt	r3, #0
     542:	68f9      	ldr	r1, [r7, #12]
     544:	f853 3021 	ldr.w	r3, [r3, r1, lsl #2]
     548:	4618      	mov	r0, r3
     54a:	4790      	blx	r2

    //
    // Configure the UART for 115200, n, 8, 1
    //
    MAP_UARTConfigSetExpClk(g_ulBase, ulSrcClock, ulBaud,
     54c:	2314      	movs	r3, #20
     54e:	f2c0 1300 	movt	r3, #256	; 0x100
     552:	681b      	ldr	r3, [r3, #0]
     554:	3314      	adds	r3, #20
     556:	681b      	ldr	r3, [r3, #0]
     558:	461c      	mov	r4, r3
     55a:	f640 4394 	movw	r3, #3220	; 0xc94
     55e:	f2c2 0300 	movt	r3, #8192	; 0x2000
     562:	681b      	ldr	r3, [r3, #0]
     564:	4618      	mov	r0, r3
     566:	6879      	ldr	r1, [r7, #4]
     568:	68ba      	ldr	r2, [r7, #8]
     56a:	2360      	movs	r3, #96	; 0x60
     56c:	47a0      	blx	r4
#ifdef UART_BUFFERED
    //
    // Set the UART to interrupt whenever the TX FIFO is almost empty or
    // when any character is received.
    //
    MAP_UARTFIFOLevelSet(g_ulBase, UART_FIFO_TX1_8, UART_FIFO_RX1_8);
     56e:	2314      	movs	r3, #20
     570:	f2c0 1300 	movt	r3, #256	; 0x100
     574:	681b      	ldr	r3, [r3, #0]
     576:	330c      	adds	r3, #12
     578:	681b      	ldr	r3, [r3, #0]
     57a:	461c      	mov	r4, r3
     57c:	f640 4394 	movw	r3, #3220	; 0xc94
     580:	f2c2 0300 	movt	r3, #8192	; 0x2000
     584:	681b      	ldr	r3, [r3, #0]
     586:	4618      	mov	r0, r3
     588:	2100      	movs	r1, #0
     58a:	2200      	movs	r2, #0
     58c:	47a0      	blx	r4

    //
    // Flush both the buffers.
    //
    UARTFlushRx();
     58e:	f000 fb89 	bl	ca4 <UARTFlushRx>
    UARTFlushTx(true);
     592:	2001      	movs	r0, #1
     594:	f000 fbac 	bl	cf0 <UARTFlushTx>

    //
    // Remember which interrupt we are dealing with.
    //
    g_ulPortNum = ulPortNum;
     598:	f640 4398 	movw	r3, #3224	; 0xc98
     59c:	f2c2 0300 	movt	r3, #8192	; 0x2000
     5a0:	68fa      	ldr	r2, [r7, #12]
     5a2:	601a      	str	r2, [r3, #0]
    // We are configured for buffered output so enable the master interrupt
    // for this UART and the receive interrupts.  We don't actually enable the
    // transmit interrupt in the UART itself until some data has been placed
    // in the transmit buffer.
    //
    MAP_UARTIntDisable(g_ulBase, 0xFFFFFFFF);
     5a4:	2314      	movs	r3, #20
     5a6:	f2c0 1300 	movt	r3, #256	; 0x100
     5aa:	681b      	ldr	r3, [r3, #0]
     5ac:	3348      	adds	r3, #72	; 0x48
     5ae:	681b      	ldr	r3, [r3, #0]
     5b0:	461a      	mov	r2, r3
     5b2:	f640 4394 	movw	r3, #3220	; 0xc94
     5b6:	f2c2 0300 	movt	r3, #8192	; 0x2000
     5ba:	681b      	ldr	r3, [r3, #0]
     5bc:	4618      	mov	r0, r3
     5be:	f04f 31ff 	mov.w	r1, #4294967295	; 0xffffffff
     5c2:	4790      	blx	r2
    MAP_UARTIntEnable(g_ulBase, UART_INT_RX | UART_INT_RT);
     5c4:	2314      	movs	r3, #20
     5c6:	f2c0 1300 	movt	r3, #256	; 0x100
     5ca:	681b      	ldr	r3, [r3, #0]
     5cc:	3344      	adds	r3, #68	; 0x44
     5ce:	681b      	ldr	r3, [r3, #0]
     5d0:	461a      	mov	r2, r3
     5d2:	f640 4394 	movw	r3, #3220	; 0xc94
     5d6:	f2c2 0300 	movt	r3, #8192	; 0x2000
     5da:	681b      	ldr	r3, [r3, #0]
     5dc:	4618      	mov	r0, r3
     5de:	2150      	movs	r1, #80	; 0x50
     5e0:	4790      	blx	r2
    MAP_IntEnable(g_ulUARTInt[ulPortNum]);
     5e2:	2348      	movs	r3, #72	; 0x48
     5e4:	f2c0 1300 	movt	r3, #256	; 0x100
     5e8:	681b      	ldr	r3, [r3, #0]
     5ea:	681b      	ldr	r3, [r3, #0]
     5ec:	461a      	mov	r2, r3
     5ee:	f242 1394 	movw	r3, #8596	; 0x2194
     5f2:	f2c0 0300 	movt	r3, #0
     5f6:	68f9      	ldr	r1, [r7, #12]
     5f8:	f853 3021 	ldr.w	r3, [r3, r1, lsl #2]
     5fc:	4618      	mov	r0, r3
     5fe:	4790      	blx	r2
#endif

    //
    // Enable the UART operation.
    //
    MAP_UARTEnable(g_ulBase);
     600:	2314      	movs	r3, #20
     602:	f2c0 1300 	movt	r3, #256	; 0x100
     606:	681b      	ldr	r3, [r3, #0]
     608:	331c      	adds	r3, #28
     60a:	681b      	ldr	r3, [r3, #0]
     60c:	461a      	mov	r2, r3
     60e:	f640 4394 	movw	r3, #3220	; 0xc94
     612:	f2c2 0300 	movt	r3, #8192	; 0x2000
     616:	681b      	ldr	r3, [r3, #0]
     618:	4618      	mov	r0, r3
     61a:	4790      	blx	r2
     61c:	e000      	b.n	620 <UARTStdioConfig+0x140>
    //
    // Check to make sure the UART peripheral is present.
    //
    if(!MAP_SysCtlPeripheralPresent(g_ulUARTPeriph[ulPortNum]))
    {
        return;
     61e:	bf00      	nop

    //
    // Enable the UART operation.
    //
    MAP_UARTEnable(g_ulBase);
}
     620:	f107 0714 	add.w	r7, r7, #20
     624:	46bd      	mov	sp, r7
     626:	bd90      	pop	{r4, r7, pc}

00000628 <UARTStdioInit>:
//! \return None.
//
//*****************************************************************************
void
UARTStdioInit(unsigned long ulPortNum)
{
     628:	b580      	push	{r7, lr}
     62a:	b082      	sub	sp, #8
     62c:	af00      	add	r7, sp, #0
     62e:	6078      	str	r0, [r7, #4]
    //
    // Pass this call on to the version of the function allowing the baud rate
    // to be specified.
    //
    UARTStdioConfig(ulPortNum, 115200, MAP_SysCtlClockGet());
     630:	2344      	movs	r3, #68	; 0x44
     632:	f2c0 1300 	movt	r3, #256	; 0x100
     636:	681b      	ldr	r3, [r3, #0]
     638:	3360      	adds	r3, #96	; 0x60
     63a:	681b      	ldr	r3, [r3, #0]
     63c:	4798      	blx	r3
     63e:	4603      	mov	r3, r0
     640:	6878      	ldr	r0, [r7, #4]
     642:	f44f 31e1 	mov.w	r1, #115200	; 0x1c200
     646:	461a      	mov	r2, r3
     648:	f7ff ff4a 	bl	4e0 <UARTStdioConfig>
}
     64c:	f107 0708 	add.w	r7, r7, #8
     650:	46bd      	mov	sp, r7
     652:	bd80      	pop	{r7, pc}

00000654 <UARTwrite>:
//! \return Returns the count of characters written.
//
//*****************************************************************************
int
UARTwrite(const char *pcBuf, unsigned long ulLen)
{
     654:	b580      	push	{r7, lr}
     656:	b084      	sub	sp, #16
     658:	af00      	add	r7, sp, #0
     65a:	6078      	str	r0, [r7, #4]
     65c:	6039      	str	r1, [r7, #0]
    ASSERT(g_ulBase != 0);

    //
    // Send the characters
    //
    for(uIdx = 0; uIdx < ulLen; uIdx++)
     65e:	2300      	movs	r3, #0
     660:	60fb      	str	r3, [r7, #12]
     662:	e059      	b.n	718 <UARTwrite+0xc4>
    {
        //
        // If the character to the UART is \n, then add a \r before it so that
        // \n is translated to \n\r in the output.
        //
        if(pcBuf[uIdx] == '\n')
     664:	687a      	ldr	r2, [r7, #4]
     666:	68fb      	ldr	r3, [r7, #12]
     668:	18d3      	adds	r3, r2, r3
     66a:	781b      	ldrb	r3, [r3, #0]
     66c:	2b0a      	cmp	r3, #10
     66e:	d126      	bne.n	6be <UARTwrite+0x6a>
        {
            if(!TX_BUFFER_FULL)
     670:	f640 4008 	movw	r0, #3080	; 0xc08
     674:	f2c2 0000 	movt	r0, #8192	; 0x2000
     678:	f640 4104 	movw	r1, #3076	; 0xc04
     67c:	f2c2 0100 	movt	r1, #8192	; 0x2000
     680:	f44f 6280 	mov.w	r2, #1024	; 0x400
     684:	f7ff fe5c 	bl	340 <IsBufferFull>
     688:	4603      	mov	r3, r0
     68a:	2b00      	cmp	r3, #0
     68c:	d149      	bne.n	722 <UARTwrite+0xce>
            {
                g_pcUARTTxBuffer[g_ulUARTTxWriteIndex] = '\r';
     68e:	f640 4304 	movw	r3, #3076	; 0xc04
     692:	f2c2 0300 	movt	r3, #8192	; 0x2000
     696:	681a      	ldr	r2, [r3, #0]
     698:	f640 0304 	movw	r3, #2052	; 0x804
     69c:	f2c2 0300 	movt	r3, #8192	; 0x2000
     6a0:	210d      	movs	r1, #13
     6a2:	5499      	strb	r1, [r3, r2]
                ADVANCE_TX_BUFFER_INDEX(g_ulUARTTxWriteIndex);
     6a4:	f640 4304 	movw	r3, #3076	; 0xc04
     6a8:	f2c2 0300 	movt	r3, #8192	; 0x2000
     6ac:	681b      	ldr	r3, [r3, #0]
     6ae:	3301      	adds	r3, #1
     6b0:	f3c3 0209 	ubfx	r2, r3, #0, #10
     6b4:	f640 4304 	movw	r3, #3076	; 0xc04
     6b8:	f2c2 0300 	movt	r3, #8192	; 0x2000
     6bc:	601a      	str	r2, [r3, #0]
        }

        //
        // Send the character to the UART output.
        //
        if(!TX_BUFFER_FULL)
     6be:	f640 4008 	movw	r0, #3080	; 0xc08
     6c2:	f2c2 0000 	movt	r0, #8192	; 0x2000
     6c6:	f640 4104 	movw	r1, #3076	; 0xc04
     6ca:	f2c2 0100 	movt	r1, #8192	; 0x2000
     6ce:	f44f 6280 	mov.w	r2, #1024	; 0x400
     6d2:	f7ff fe35 	bl	340 <IsBufferFull>
     6d6:	4603      	mov	r3, r0
     6d8:	2b00      	cmp	r3, #0
     6da:	d124      	bne.n	726 <UARTwrite+0xd2>
        {
            g_pcUARTTxBuffer[g_ulUARTTxWriteIndex] = pcBuf[uIdx];
     6dc:	f640 4304 	movw	r3, #3076	; 0xc04
     6e0:	f2c2 0300 	movt	r3, #8192	; 0x2000
     6e4:	681a      	ldr	r2, [r3, #0]
     6e6:	6879      	ldr	r1, [r7, #4]
     6e8:	68fb      	ldr	r3, [r7, #12]
     6ea:	18cb      	adds	r3, r1, r3
     6ec:	7819      	ldrb	r1, [r3, #0]
     6ee:	f640 0304 	movw	r3, #2052	; 0x804
     6f2:	f2c2 0300 	movt	r3, #8192	; 0x2000
     6f6:	5499      	strb	r1, [r3, r2]
            ADVANCE_TX_BUFFER_INDEX(g_ulUARTTxWriteIndex);
     6f8:	f640 4304 	movw	r3, #3076	; 0xc04
     6fc:	f2c2 0300 	movt	r3, #8192	; 0x2000
     700:	681b      	ldr	r3, [r3, #0]
     702:	3301      	adds	r3, #1
     704:	f3c3 0209 	ubfx	r2, r3, #0, #10
     708:	f640 4304 	movw	r3, #3076	; 0xc04
     70c:	f2c2 0300 	movt	r3, #8192	; 0x2000
     710:	601a      	str	r2, [r3, #0]
    ASSERT(g_ulBase != 0);

    //
    // Send the characters
    //
    for(uIdx = 0; uIdx < ulLen; uIdx++)
     712:	68fb      	ldr	r3, [r7, #12]
     714:	3301      	adds	r3, #1
     716:	60fb      	str	r3, [r7, #12]
     718:	68fa      	ldr	r2, [r7, #12]
     71a:	683b      	ldr	r3, [r7, #0]
     71c:	429a      	cmp	r2, r3
     71e:	d3a1      	bcc.n	664 <UARTwrite+0x10>
     720:	e002      	b.n	728 <UARTwrite+0xd4>
            else
            {
                //
                // Buffer is full - discard remaining characters and return.
                //
                break;
     722:	bf00      	nop
     724:	e000      	b.n	728 <UARTwrite+0xd4>
        else
        {
            //
            // Buffer is full - discard remaining characters and return.
            //
            break;
     726:	bf00      	nop

    //
    // If we have anything in the buffer, make sure that the UART is set
    // up to transmit it.
    //
    if(!TX_BUFFER_EMPTY)
     728:	f640 4008 	movw	r0, #3080	; 0xc08
     72c:	f2c2 0000 	movt	r0, #8192	; 0x2000
     730:	f640 4104 	movw	r1, #3076	; 0xc04
     734:	f2c2 0100 	movt	r1, #8192	; 0x2000
     738:	f7ff fe24 	bl	384 <IsBufferEmpty>
     73c:	4603      	mov	r3, r0
     73e:	2b00      	cmp	r3, #0
     740:	d116      	bne.n	770 <UARTwrite+0x11c>
    {
        UARTPrimeTransmit(g_ulBase);
     742:	f640 4394 	movw	r3, #3220	; 0xc94
     746:	f2c2 0300 	movt	r3, #8192	; 0x2000
     74a:	681b      	ldr	r3, [r3, #0]
     74c:	4618      	mov	r0, r3
     74e:	f7ff fe51 	bl	3f4 <UARTPrimeTransmit>
        MAP_UARTIntEnable(g_ulBase, UART_INT_TX);
     752:	2314      	movs	r3, #20
     754:	f2c0 1300 	movt	r3, #256	; 0x100
     758:	681b      	ldr	r3, [r3, #0]
     75a:	3344      	adds	r3, #68	; 0x44
     75c:	681b      	ldr	r3, [r3, #0]
     75e:	461a      	mov	r2, r3
     760:	f640 4394 	movw	r3, #3220	; 0xc94
     764:	f2c2 0300 	movt	r3, #8192	; 0x2000
     768:	681b      	ldr	r3, [r3, #0]
     76a:	4618      	mov	r0, r3
     76c:	2120      	movs	r1, #32
     76e:	4790      	blx	r2
    }

    //
    // Return the number of characters written.
    //
    return(uIdx);
     770:	68fb      	ldr	r3, [r7, #12]
    //
    // Return the number of characters written.
    //
    return(uIdx);
#endif
}
     772:	4618      	mov	r0, r3
     774:	f107 0710 	add.w	r7, r7, #16
     778:	46bd      	mov	sp, r7
     77a:	bd80      	pop	{r7, pc}

0000077c <UARTgets>:
//! the trailing 0.
//
//*****************************************************************************
int
UARTgets(char *pcBuf, unsigned long ulLen)
{
     77c:	b580      	push	{r7, lr}
     77e:	b084      	sub	sp, #16
     780:	af00      	add	r7, sp, #0
     782:	6078      	str	r0, [r7, #4]
     784:	6039      	str	r1, [r7, #0]
#ifdef UART_BUFFERED
    unsigned long ulCount = 0;
     786:	2300      	movs	r3, #0
     788:	60fb      	str	r3, [r7, #12]

    //
    // Adjust the length back by 1 to leave space for the trailing
    // null terminator.
    //
    ulLen--;
     78a:	683b      	ldr	r3, [r7, #0]
     78c:	3b01      	subs	r3, #1
     78e:	603b      	str	r3, [r7, #0]
     790:	e000      	b.n	794 <UARTgets+0x18>
                // Increment the count of characters received.
                //
                ulCount++;
            }
        }
    }
     792:	bf00      	nop
    while(1)
    {
        //
        // Read the next character from the receive buffer.
        //
        if(!RX_BUFFER_EMPTY)
     794:	f640 4090 	movw	r0, #3216	; 0xc90
     798:	f2c2 0000 	movt	r0, #8192	; 0x2000
     79c:	f640 418c 	movw	r1, #3212	; 0xc8c
     7a0:	f2c2 0100 	movt	r1, #8192	; 0x2000
     7a4:	f7ff fdee 	bl	384 <IsBufferEmpty>
     7a8:	4603      	mov	r3, r0
     7aa:	2b00      	cmp	r3, #0
     7ac:	d1f1      	bne.n	792 <UARTgets+0x16>
        {
            cChar = g_pcUARTRxBuffer[g_ulUARTRxReadIndex];
     7ae:	f640 4390 	movw	r3, #3216	; 0xc90
     7b2:	f2c2 0300 	movt	r3, #8192	; 0x2000
     7b6:	681a      	ldr	r2, [r3, #0]
     7b8:	f640 430c 	movw	r3, #3084	; 0xc0c
     7bc:	f2c2 0300 	movt	r3, #8192	; 0x2000
     7c0:	5c9b      	ldrb	r3, [r3, r2]
     7c2:	72fb      	strb	r3, [r7, #11]
            ADVANCE_RX_BUFFER_INDEX(g_ulUARTRxReadIndex);
     7c4:	f640 4390 	movw	r3, #3216	; 0xc90
     7c8:	f2c2 0300 	movt	r3, #8192	; 0x2000
     7cc:	681b      	ldr	r3, [r3, #0]
     7ce:	3301      	adds	r3, #1
     7d0:	f003 027f 	and.w	r2, r3, #127	; 0x7f
     7d4:	f640 4390 	movw	r3, #3216	; 0xc90
     7d8:	f2c2 0300 	movt	r3, #8192	; 0x2000
     7dc:	601a      	str	r2, [r3, #0]

            //
            // See if a newline or escape character was received.
            //
            if((cChar == '\r') || (cChar == '\n') || (cChar == 0x1b))
     7de:	7afb      	ldrb	r3, [r7, #11]
     7e0:	2b0d      	cmp	r3, #13
     7e2:	d012      	beq.n	80a <UARTgets+0x8e>
     7e4:	7afb      	ldrb	r3, [r7, #11]
     7e6:	2b0a      	cmp	r3, #10
     7e8:	d00f      	beq.n	80a <UARTgets+0x8e>
     7ea:	7afb      	ldrb	r3, [r7, #11]
     7ec:	2b1b      	cmp	r3, #27
     7ee:	d00c      	beq.n	80a <UARTgets+0x8e>
            // Process the received character as long as we are not at the end
            // of the buffer.  If the end of the buffer has been reached then
            // all additional characters are ignored until a newline is
            // received.
            //
            if(ulCount < ulLen)
     7f0:	68fa      	ldr	r2, [r7, #12]
     7f2:	683b      	ldr	r3, [r7, #0]
     7f4:	429a      	cmp	r2, r3
     7f6:	d2cc      	bcs.n	792 <UARTgets+0x16>
            {
                //
                // Store the character in the caller supplied buffer.
                //
                pcBuf[ulCount] = cChar;
     7f8:	687a      	ldr	r2, [r7, #4]
     7fa:	68fb      	ldr	r3, [r7, #12]
     7fc:	18d3      	adds	r3, r2, r3
     7fe:	7afa      	ldrb	r2, [r7, #11]
     800:	701a      	strb	r2, [r3, #0]

                //
                // Increment the count of characters received.
                //
                ulCount++;
     802:	68fb      	ldr	r3, [r7, #12]
     804:	3301      	adds	r3, #1
     806:	60fb      	str	r3, [r7, #12]
            }
        }
    }
     808:	e7c3      	b.n	792 <UARTgets+0x16>

    //
    // Add a null termination to the string.
    //
    pcBuf[ulCount] = 0;
     80a:	687a      	ldr	r2, [r7, #4]
     80c:	68fb      	ldr	r3, [r7, #12]
     80e:	18d3      	adds	r3, r2, r3
     810:	2200      	movs	r2, #0
     812:	701a      	strb	r2, [r3, #0]

    //
    // Return the count of chars in the buffer, not counting the trailing 0.
    //
    return(ulCount);
     814:	68fb      	ldr	r3, [r7, #12]
    //
    // Return the count of chars in the buffer, not counting the trailing 0.
    //
    return(ulCount);
#endif
}
     816:	4618      	mov	r0, r3
     818:	f107 0710 	add.w	r7, r7, #16
     81c:	46bd      	mov	sp, r7
     81e:	bd80      	pop	{r7, pc}

00000820 <UARTprintf>:
//! \return None.
//
//*****************************************************************************
void
UARTprintf(const char *pcString, ...)
{
     820:	b40f      	push	{r0, r1, r2, r3}
     822:	b580      	push	{r7, lr}
     824:	b08e      	sub	sp, #56	; 0x38
     826:	af00      	add	r7, sp, #0
    ASSERT(pcString != 0);

    //
    // Start the varargs processing.
    //
    va_start(vaArgP, pcString);
     828:	f107 0344 	add.w	r3, r7, #68	; 0x44
     82c:	607b      	str	r3, [r7, #4]

    //
    // Loop while there are more characters in the string.
    //
    while(*pcString)
     82e:	e1f3      	b.n	c18 <UARTprintf+0x3f8>
    {
        //
        // Find the first non-% character, or the end of the string.
        //
        for(ulIdx = 0; (pcString[ulIdx] != '%') && (pcString[ulIdx] != '\0');
     830:	2300      	movs	r3, #0
     832:	637b      	str	r3, [r7, #52]	; 0x34
     834:	e002      	b.n	83c <UARTprintf+0x1c>
            ulIdx++)
     836:	6b7b      	ldr	r3, [r7, #52]	; 0x34
     838:	3301      	adds	r3, #1
     83a:	637b      	str	r3, [r7, #52]	; 0x34
    while(*pcString)
    {
        //
        // Find the first non-% character, or the end of the string.
        //
        for(ulIdx = 0; (pcString[ulIdx] != '%') && (pcString[ulIdx] != '\0');
     83c:	6c3a      	ldr	r2, [r7, #64]	; 0x40
     83e:	6b7b      	ldr	r3, [r7, #52]	; 0x34
     840:	18d3      	adds	r3, r2, r3
     842:	781b      	ldrb	r3, [r3, #0]
     844:	2b25      	cmp	r3, #37	; 0x25
     846:	d005      	beq.n	854 <UARTprintf+0x34>
     848:	6c3a      	ldr	r2, [r7, #64]	; 0x40
     84a:	6b7b      	ldr	r3, [r7, #52]	; 0x34
     84c:	18d3      	adds	r3, r2, r3
     84e:	781b      	ldrb	r3, [r3, #0]
     850:	2b00      	cmp	r3, #0
     852:	d1f0      	bne.n	836 <UARTprintf+0x16>
        }

        //
        // Write this portion of the string.
        //
        UARTwrite(pcString, ulIdx);
     854:	6c38      	ldr	r0, [r7, #64]	; 0x40
     856:	6b79      	ldr	r1, [r7, #52]	; 0x34
     858:	f7ff fefc 	bl	654 <UARTwrite>

        //
        // Skip the portion of the string that was written.
        //
        pcString += ulIdx;
     85c:	6c3a      	ldr	r2, [r7, #64]	; 0x40
     85e:	6b7b      	ldr	r3, [r7, #52]	; 0x34
     860:	18d3      	adds	r3, r2, r3
     862:	643b      	str	r3, [r7, #64]	; 0x40

        //
        // See if the next character is a %.
        //
        if(*pcString == '%')
     864:	6c3b      	ldr	r3, [r7, #64]	; 0x40
     866:	781b      	ldrb	r3, [r3, #0]
     868:	2b25      	cmp	r3, #37	; 0x25
     86a:	f040 81d5 	bne.w	c18 <UARTprintf+0x3f8>
        {
            //
            // Skip the %.
            //
            pcString++;
     86e:	6c3b      	ldr	r3, [r7, #64]	; 0x40
     870:	3301      	adds	r3, #1
     872:	643b      	str	r3, [r7, #64]	; 0x40

            //
            // Set the digit count to zero, and the fill character to space
            // (i.e. to the defaults).
            //
            ulCount = 0;
     874:	2300      	movs	r3, #0
     876:	62fb      	str	r3, [r7, #44]	; 0x2c
            cFill = ' ';
     878:	2320      	movs	r3, #32
     87a:	f887 3023 	strb.w	r3, [r7, #35]	; 0x23
again:

            //
            // Determine how to handle the next character.
            //
            switch(*pcString++)
     87e:	6c3b      	ldr	r3, [r7, #64]	; 0x40
     880:	781b      	ldrb	r3, [r3, #0]
     882:	6c3a      	ldr	r2, [r7, #64]	; 0x40
     884:	3201      	adds	r2, #1
     886:	643a      	str	r2, [r7, #64]	; 0x40
     888:	3b25      	subs	r3, #37	; 0x25
     88a:	2b53      	cmp	r3, #83	; 0x53
     88c:	f200 81bb 	bhi.w	c06 <UARTprintf+0x3e6>
     890:	a201      	add	r2, pc, #4	; (adr r2, 898 <UARTprintf+0x78>)
     892:	f852 f023 	ldr.w	pc, [r2, r3, lsl #2]
     896:	bf00      	nop
     898:	00000bf9 	.word	0x00000bf9
     89c:	00000c07 	.word	0x00000c07
     8a0:	00000c07 	.word	0x00000c07
     8a4:	00000c07 	.word	0x00000c07
     8a8:	00000c07 	.word	0x00000c07
     8ac:	00000c07 	.word	0x00000c07
     8b0:	00000c07 	.word	0x00000c07
     8b4:	00000c07 	.word	0x00000c07
     8b8:	00000c07 	.word	0x00000c07
     8bc:	00000c07 	.word	0x00000c07
     8c0:	00000c07 	.word	0x00000c07
     8c4:	000009e9 	.word	0x000009e9
     8c8:	000009e9 	.word	0x000009e9
     8cc:	000009e9 	.word	0x000009e9
     8d0:	000009e9 	.word	0x000009e9
     8d4:	000009e9 	.word	0x000009e9
     8d8:	000009e9 	.word	0x000009e9
     8dc:	000009e9 	.word	0x000009e9
     8e0:	000009e9 	.word	0x000009e9
     8e4:	000009e9 	.word	0x000009e9
     8e8:	000009e9 	.word	0x000009e9
     8ec:	00000c07 	.word	0x00000c07
     8f0:	00000c07 	.word	0x00000c07
     8f4:	00000c07 	.word	0x00000c07
     8f8:	00000c07 	.word	0x00000c07
     8fc:	00000c07 	.word	0x00000c07
     900:	00000c07 	.word	0x00000c07
     904:	00000c07 	.word	0x00000c07
     908:	00000c07 	.word	0x00000c07
     90c:	00000c07 	.word	0x00000c07
     910:	00000c07 	.word	0x00000c07
     914:	00000c07 	.word	0x00000c07
     918:	00000c07 	.word	0x00000c07
     91c:	00000c07 	.word	0x00000c07
     920:	00000c07 	.word	0x00000c07
     924:	00000c07 	.word	0x00000c07
     928:	00000c07 	.word	0x00000c07
     92c:	00000c07 	.word	0x00000c07
     930:	00000c07 	.word	0x00000c07
     934:	00000c07 	.word	0x00000c07
     938:	00000c07 	.word	0x00000c07
     93c:	00000c07 	.word	0x00000c07
     940:	00000c07 	.word	0x00000c07
     944:	00000c07 	.word	0x00000c07
     948:	00000c07 	.word	0x00000c07
     94c:	00000c07 	.word	0x00000c07
     950:	00000c07 	.word	0x00000c07
     954:	00000c07 	.word	0x00000c07
     958:	00000c07 	.word	0x00000c07
     95c:	00000c07 	.word	0x00000c07
     960:	00000c07 	.word	0x00000c07
     964:	00000adb 	.word	0x00000adb
     968:	00000c07 	.word	0x00000c07
     96c:	00000c07 	.word	0x00000c07
     970:	00000c07 	.word	0x00000c07
     974:	00000c07 	.word	0x00000c07
     978:	00000c07 	.word	0x00000c07
     97c:	00000c07 	.word	0x00000c07
     980:	00000c07 	.word	0x00000c07
     984:	00000c07 	.word	0x00000c07
     988:	00000c07 	.word	0x00000c07
     98c:	00000c07 	.word	0x00000c07
     990:	00000a1d 	.word	0x00000a1d
     994:	00000a35 	.word	0x00000a35
     998:	00000c07 	.word	0x00000c07
     99c:	00000c07 	.word	0x00000c07
     9a0:	00000c07 	.word	0x00000c07
     9a4:	00000c07 	.word	0x00000c07
     9a8:	00000a35 	.word	0x00000a35
     9ac:	00000c07 	.word	0x00000c07
     9b0:	00000c07 	.word	0x00000c07
     9b4:	00000c07 	.word	0x00000c07
     9b8:	00000c07 	.word	0x00000c07
     9bc:	00000c07 	.word	0x00000c07
     9c0:	00000c07 	.word	0x00000c07
     9c4:	00000adb 	.word	0x00000adb
     9c8:	00000c07 	.word	0x00000c07
     9cc:	00000c07 	.word	0x00000c07
     9d0:	00000a5f 	.word	0x00000a5f
     9d4:	00000c07 	.word	0x00000c07
     9d8:	00000ac3 	.word	0x00000ac3
     9dc:	00000c07 	.word	0x00000c07
     9e0:	00000c07 	.word	0x00000c07
     9e4:	00000adb 	.word	0x00000adb
                {
                    //
                    // If this is a zero, and it is the first digit, then the
                    // fill character is a zero instead of a space.
                    //
                    if((pcString[-1] == '0') && (ulCount == 0))
     9e8:	6c3b      	ldr	r3, [r7, #64]	; 0x40
     9ea:	3b01      	subs	r3, #1
     9ec:	781b      	ldrb	r3, [r3, #0]
     9ee:	2b30      	cmp	r3, #48	; 0x30
     9f0:	d105      	bne.n	9fe <UARTprintf+0x1de>
     9f2:	6afb      	ldr	r3, [r7, #44]	; 0x2c
     9f4:	2b00      	cmp	r3, #0
     9f6:	d102      	bne.n	9fe <UARTprintf+0x1de>
                    {
                        cFill = '0';
     9f8:	2330      	movs	r3, #48	; 0x30
     9fa:	f887 3023 	strb.w	r3, [r7, #35]	; 0x23
                    }

                    //
                    // Update the digit count.
                    //
                    ulCount *= 10;
     9fe:	6afa      	ldr	r2, [r7, #44]	; 0x2c
     a00:	4613      	mov	r3, r2
     a02:	009b      	lsls	r3, r3, #2
     a04:	189b      	adds	r3, r3, r2
     a06:	005b      	lsls	r3, r3, #1
     a08:	62fb      	str	r3, [r7, #44]	; 0x2c
                    ulCount += pcString[-1] - '0';
     a0a:	6c3b      	ldr	r3, [r7, #64]	; 0x40
     a0c:	3b01      	subs	r3, #1
     a0e:	781b      	ldrb	r3, [r3, #0]
     a10:	461a      	mov	r2, r3
     a12:	6afb      	ldr	r3, [r7, #44]	; 0x2c
     a14:	18d3      	adds	r3, r2, r3
     a16:	3b30      	subs	r3, #48	; 0x30
     a18:	62fb      	str	r3, [r7, #44]	; 0x2c

                    //
                    // Get the next character.
                    //
                    goto again;
     a1a:	e730      	b.n	87e <UARTprintf+0x5e>
                case 'c':
                {
                    //
                    // Get the value from the varargs.
                    //
                    ulValue = va_arg(vaArgP, unsigned long);
     a1c:	687b      	ldr	r3, [r7, #4]
     a1e:	1d1a      	adds	r2, r3, #4
     a20:	607a      	str	r2, [r7, #4]
     a22:	681b      	ldr	r3, [r3, #0]
     a24:	61bb      	str	r3, [r7, #24]

                    //
                    // Print out the character.
                    //
                    UARTwrite((char *)&ulValue, 1);
     a26:	f107 0318 	add.w	r3, r7, #24
     a2a:	4618      	mov	r0, r3
     a2c:	2101      	movs	r1, #1
     a2e:	f7ff fe11 	bl	654 <UARTwrite>

                    //
                    // This command has been handled.
                    //
                    break;
     a32:	e0f1      	b.n	c18 <UARTprintf+0x3f8>
                case 'i':
                {
                    //
                    // Get the value from the varargs.
                    //
                    ulValue = va_arg(vaArgP, unsigned long);
     a34:	687b      	ldr	r3, [r7, #4]
     a36:	1d1a      	adds	r2, r3, #4
     a38:	607a      	str	r2, [r7, #4]
     a3a:	681b      	ldr	r3, [r3, #0]
     a3c:	61bb      	str	r3, [r7, #24]

                    //
                    // Reset the buffer position.
                    //
                    ulPos = 0;
     a3e:	2300      	movs	r3, #0
     a40:	633b      	str	r3, [r7, #48]	; 0x30

                    //
                    // If the value is negative, make it positive and indicate
                    // that a minus sign is needed.
                    //
                    if((long)ulValue < 0)
     a42:	69bb      	ldr	r3, [r7, #24]
     a44:	2b00      	cmp	r3, #0
     a46:	da05      	bge.n	a54 <UARTprintf+0x234>
                    {
                        //
                        // Make the value positive.
                        //
                        ulValue = -(long)ulValue;
     a48:	69bb      	ldr	r3, [r7, #24]
     a4a:	425b      	negs	r3, r3
     a4c:	61bb      	str	r3, [r7, #24]

                        //
                        // Indicate that the value is negative.
                        //
                        ulNeg = 1;
     a4e:	2301      	movs	r3, #1
     a50:	627b      	str	r3, [r7, #36]	; 0x24
     a52:	e001      	b.n	a58 <UARTprintf+0x238>
                    {
                        //
                        // Indicate that the value is positive so that a minus
                        // sign isn't inserted.
                        //
                        ulNeg = 0;
     a54:	2300      	movs	r3, #0
     a56:	627b      	str	r3, [r7, #36]	; 0x24
                    }

                    //
                    // Set the base to 10.
                    //
                    ulBase = 10;
     a58:	230a      	movs	r3, #10
     a5a:	62bb      	str	r3, [r7, #40]	; 0x28

                    //
                    // Convert the value to ASCII.
                    //
                    goto convert;
     a5c:	e048      	b.n	af0 <UARTprintf+0x2d0>
                case 's':
                {
                    //
                    // Get the string pointer from the varargs.
                    //
                    pcStr = va_arg(vaArgP, char *);
     a5e:	687b      	ldr	r3, [r7, #4]
     a60:	1d1a      	adds	r2, r3, #4
     a62:	607a      	str	r2, [r7, #4]
     a64:	681b      	ldr	r3, [r3, #0]
     a66:	61fb      	str	r3, [r7, #28]

                    //
                    // Determine the length of the string.
                    //
                    for(ulIdx = 0; pcStr[ulIdx] != '\0'; ulIdx++)
     a68:	2300      	movs	r3, #0
     a6a:	637b      	str	r3, [r7, #52]	; 0x34
     a6c:	e002      	b.n	a74 <UARTprintf+0x254>
     a6e:	6b7b      	ldr	r3, [r7, #52]	; 0x34
     a70:	3301      	adds	r3, #1
     a72:	637b      	str	r3, [r7, #52]	; 0x34
     a74:	69fa      	ldr	r2, [r7, #28]
     a76:	6b7b      	ldr	r3, [r7, #52]	; 0x34
     a78:	18d3      	adds	r3, r2, r3
     a7a:	781b      	ldrb	r3, [r3, #0]
     a7c:	2b00      	cmp	r3, #0
     a7e:	d1f6      	bne.n	a6e <UARTprintf+0x24e>
                    }

                    //
                    // Write the string.
                    //
                    UARTwrite(pcStr, ulIdx);
     a80:	69f8      	ldr	r0, [r7, #28]
     a82:	6b79      	ldr	r1, [r7, #52]	; 0x34
     a84:	f7ff fde6 	bl	654 <UARTwrite>

                    //
                    // Write any required padding spaces
                    //
                    if(ulCount > ulIdx)
     a88:	6afa      	ldr	r2, [r7, #44]	; 0x2c
     a8a:	6b7b      	ldr	r3, [r7, #52]	; 0x34
     a8c:	429a      	cmp	r2, r3
     a8e:	f240 80c2 	bls.w	c16 <UARTprintf+0x3f6>
                    {
                        ulCount -= ulIdx;
     a92:	6afa      	ldr	r2, [r7, #44]	; 0x2c
     a94:	6b7b      	ldr	r3, [r7, #52]	; 0x34
     a96:	1ad3      	subs	r3, r2, r3
     a98:	62fb      	str	r3, [r7, #44]	; 0x2c
                        while(ulCount--)
     a9a:	e006      	b.n	aaa <UARTprintf+0x28a>
                        {
                            UARTwrite(" ", 1);
     a9c:	f242 3024 	movw	r0, #8996	; 0x2324
     aa0:	f2c0 0000 	movt	r0, #0
     aa4:	2101      	movs	r1, #1
     aa6:	f7ff fdd5 	bl	654 <UARTwrite>
                    // Write any required padding spaces
                    //
                    if(ulCount > ulIdx)
                    {
                        ulCount -= ulIdx;
                        while(ulCount--)
     aaa:	6afb      	ldr	r3, [r7, #44]	; 0x2c
     aac:	2b00      	cmp	r3, #0
     aae:	bf0c      	ite	eq
     ab0:	2300      	moveq	r3, #0
     ab2:	2301      	movne	r3, #1
     ab4:	b2db      	uxtb	r3, r3
     ab6:	6afa      	ldr	r2, [r7, #44]	; 0x2c
     ab8:	3a01      	subs	r2, #1
     aba:	62fa      	str	r2, [r7, #44]	; 0x2c
     abc:	2b00      	cmp	r3, #0
     abe:	d1ed      	bne.n	a9c <UARTprintf+0x27c>
                        }
                    }
                    //
                    // This command has been handled.
                    //
                    break;
     ac0:	e0a9      	b.n	c16 <UARTprintf+0x3f6>
                case 'u':
                {
                    //
                    // Get the value from the varargs.
                    //
                    ulValue = va_arg(vaArgP, unsigned long);
     ac2:	687b      	ldr	r3, [r7, #4]
     ac4:	1d1a      	adds	r2, r3, #4
     ac6:	607a      	str	r2, [r7, #4]
     ac8:	681b      	ldr	r3, [r3, #0]
     aca:	61bb      	str	r3, [r7, #24]

                    //
                    // Reset the buffer position.
                    //
                    ulPos = 0;
     acc:	2300      	movs	r3, #0
     ace:	633b      	str	r3, [r7, #48]	; 0x30

                    //
                    // Set the base to 10.
                    //
                    ulBase = 10;
     ad0:	230a      	movs	r3, #10
     ad2:	62bb      	str	r3, [r7, #40]	; 0x28

                    //
                    // Indicate that the value is positive so that a minus sign
                    // isn't inserted.
                    //
                    ulNeg = 0;
     ad4:	2300      	movs	r3, #0
     ad6:	627b      	str	r3, [r7, #36]	; 0x24

                    //
                    // Convert the value to ASCII.
                    //
                    goto convert;
     ad8:	e00a      	b.n	af0 <UARTprintf+0x2d0>
                case 'p':
                {
                    //
                    // Get the value from the varargs.
                    //
                    ulValue = va_arg(vaArgP, unsigned long);
     ada:	687b      	ldr	r3, [r7, #4]
     adc:	1d1a      	adds	r2, r3, #4
     ade:	607a      	str	r2, [r7, #4]
     ae0:	681b      	ldr	r3, [r3, #0]
     ae2:	61bb      	str	r3, [r7, #24]

                    //
                    // Reset the buffer position.
                    //
                    ulPos = 0;
     ae4:	2300      	movs	r3, #0
     ae6:	633b      	str	r3, [r7, #48]	; 0x30

                    //
                    // Set the base to 16.
                    //
                    ulBase = 16;
     ae8:	2310      	movs	r3, #16
     aea:	62bb      	str	r3, [r7, #40]	; 0x28

                    //
                    // Indicate that the value is positive so that a minus sign
                    // isn't inserted.
                    //
                    ulNeg = 0;
     aec:	2300      	movs	r3, #0
     aee:	627b      	str	r3, [r7, #36]	; 0x24
                    //
                    // Determine the number of digits in the string version of
                    // the value.
                    //
convert:
                    for(ulIdx = 1;
     af0:	2301      	movs	r3, #1
     af2:	637b      	str	r3, [r7, #52]	; 0x34
     af4:	e007      	b.n	b06 <UARTprintf+0x2e6>
                        (((ulIdx * ulBase) <= ulValue) &&
                         (((ulIdx * ulBase) / ulBase) == ulIdx));
                        ulIdx *= ulBase, ulCount--)
     af6:	6b7b      	ldr	r3, [r7, #52]	; 0x34
     af8:	6aba      	ldr	r2, [r7, #40]	; 0x28
     afa:	fb02 f303 	mul.w	r3, r2, r3
     afe:	637b      	str	r3, [r7, #52]	; 0x34
     b00:	6afb      	ldr	r3, [r7, #44]	; 0x2c
     b02:	3b01      	subs	r3, #1
     b04:	62fb      	str	r3, [r7, #44]	; 0x2c
                    // Determine the number of digits in the string version of
                    // the value.
                    //
convert:
                    for(ulIdx = 1;
                        (((ulIdx * ulBase) <= ulValue) &&
     b06:	6b7b      	ldr	r3, [r7, #52]	; 0x34
     b08:	6aba      	ldr	r2, [r7, #40]	; 0x28
     b0a:	fb02 f203 	mul.w	r2, r2, r3
     b0e:	69bb      	ldr	r3, [r7, #24]
                    //
                    // Determine the number of digits in the string version of
                    // the value.
                    //
convert:
                    for(ulIdx = 1;
     b10:	429a      	cmp	r2, r3
     b12:	d809      	bhi.n	b28 <UARTprintf+0x308>
                        (((ulIdx * ulBase) <= ulValue) &&
                         (((ulIdx * ulBase) / ulBase) == ulIdx));
     b14:	6b7b      	ldr	r3, [r7, #52]	; 0x34
     b16:	6aba      	ldr	r2, [r7, #40]	; 0x28
     b18:	fb02 f203 	mul.w	r2, r2, r3
     b1c:	6abb      	ldr	r3, [r7, #40]	; 0x28
     b1e:	fbb2 f2f3 	udiv	r2, r2, r3
                    // Determine the number of digits in the string version of
                    // the value.
                    //
convert:
                    for(ulIdx = 1;
                        (((ulIdx * ulBase) <= ulValue) &&
     b22:	6b7b      	ldr	r3, [r7, #52]	; 0x34
     b24:	429a      	cmp	r2, r3
     b26:	d0e6      	beq.n	af6 <UARTprintf+0x2d6>

                    //
                    // If the value is negative, reduce the count of padding
                    // characters needed.
                    //
                    if(ulNeg)
     b28:	6a7b      	ldr	r3, [r7, #36]	; 0x24
     b2a:	2b00      	cmp	r3, #0
     b2c:	d002      	beq.n	b34 <UARTprintf+0x314>
                    {
                        ulCount--;
     b2e:	6afb      	ldr	r3, [r7, #44]	; 0x2c
     b30:	3b01      	subs	r3, #1
     b32:	62fb      	str	r3, [r7, #44]	; 0x2c

                    //
                    // If the value is negative and the value is padded with
                    // zeros, then place the minus sign before the padding.
                    //
                    if(ulNeg && (cFill == '0'))
     b34:	6a7b      	ldr	r3, [r7, #36]	; 0x24
     b36:	2b00      	cmp	r3, #0
     b38:	d00e      	beq.n	b58 <UARTprintf+0x338>
     b3a:	f897 3023 	ldrb.w	r3, [r7, #35]	; 0x23
     b3e:	2b30      	cmp	r3, #48	; 0x30
     b40:	d10a      	bne.n	b58 <UARTprintf+0x338>
                    {
                        //
                        // Place the minus sign in the output buffer.
                        //
                        pcBuf[ulPos++] = '-';
     b42:	f107 0208 	add.w	r2, r7, #8
     b46:	6b3b      	ldr	r3, [r7, #48]	; 0x30
     b48:	18d3      	adds	r3, r2, r3
     b4a:	222d      	movs	r2, #45	; 0x2d
     b4c:	701a      	strb	r2, [r3, #0]
     b4e:	6b3b      	ldr	r3, [r7, #48]	; 0x30
     b50:	3301      	adds	r3, #1
     b52:	633b      	str	r3, [r7, #48]	; 0x30

                        //
                        // The minus sign has been placed, so turn off the
                        // negative flag.
                        //
                        ulNeg = 0;
     b54:	2300      	movs	r3, #0
     b56:	627b      	str	r3, [r7, #36]	; 0x24

                    //
                    // Provide additional padding at the beginning of the
                    // string conversion if needed.
                    //
                    if((ulCount > 1) && (ulCount < 16))
     b58:	6afb      	ldr	r3, [r7, #44]	; 0x2c
     b5a:	2b01      	cmp	r3, #1
     b5c:	d916      	bls.n	b8c <UARTprintf+0x36c>
     b5e:	6afb      	ldr	r3, [r7, #44]	; 0x2c
     b60:	2b0f      	cmp	r3, #15
     b62:	d813      	bhi.n	b8c <UARTprintf+0x36c>
                    {
                        for(ulCount--; ulCount; ulCount--)
     b64:	6afb      	ldr	r3, [r7, #44]	; 0x2c
     b66:	3b01      	subs	r3, #1
     b68:	62fb      	str	r3, [r7, #44]	; 0x2c
     b6a:	e00c      	b.n	b86 <UARTprintf+0x366>
                        {
                            pcBuf[ulPos++] = cFill;
     b6c:	f107 0208 	add.w	r2, r7, #8
     b70:	6b3b      	ldr	r3, [r7, #48]	; 0x30
     b72:	18d3      	adds	r3, r2, r3
     b74:	f897 2023 	ldrb.w	r2, [r7, #35]	; 0x23
     b78:	701a      	strb	r2, [r3, #0]
     b7a:	6b3b      	ldr	r3, [r7, #48]	; 0x30
     b7c:	3301      	adds	r3, #1
     b7e:	633b      	str	r3, [r7, #48]	; 0x30
                    // Provide additional padding at the beginning of the
                    // string conversion if needed.
                    //
                    if((ulCount > 1) && (ulCount < 16))
                    {
                        for(ulCount--; ulCount; ulCount--)
     b80:	6afb      	ldr	r3, [r7, #44]	; 0x2c
     b82:	3b01      	subs	r3, #1
     b84:	62fb      	str	r3, [r7, #44]	; 0x2c
     b86:	6afb      	ldr	r3, [r7, #44]	; 0x2c
     b88:	2b00      	cmp	r3, #0
     b8a:	d1ef      	bne.n	b6c <UARTprintf+0x34c>

                    //
                    // If the value is negative, then place the minus sign
                    // before the number.
                    //
                    if(ulNeg)
     b8c:	6a7b      	ldr	r3, [r7, #36]	; 0x24
     b8e:	2b00      	cmp	r3, #0
     b90:	d028      	beq.n	be4 <UARTprintf+0x3c4>
                    {
                        //
                        // Place the minus sign in the output buffer.
                        //
                        pcBuf[ulPos++] = '-';
     b92:	f107 0208 	add.w	r2, r7, #8
     b96:	6b3b      	ldr	r3, [r7, #48]	; 0x30
     b98:	18d3      	adds	r3, r2, r3
     b9a:	222d      	movs	r2, #45	; 0x2d
     b9c:	701a      	strb	r2, [r3, #0]
     b9e:	6b3b      	ldr	r3, [r7, #48]	; 0x30
     ba0:	3301      	adds	r3, #1
     ba2:	633b      	str	r3, [r7, #48]	; 0x30
                    }

                    //
                    // Convert the value into a string.
                    //
                    for(; ulIdx; ulIdx /= ulBase)
     ba4:	e01e      	b.n	be4 <UARTprintf+0x3c4>
                    {
                        pcBuf[ulPos++] = g_pcHex[(ulValue / ulIdx) % ulBase];
     ba6:	f242 1384 	movw	r3, #8580	; 0x2184
     baa:	f2c0 0300 	movt	r3, #0
     bae:	681a      	ldr	r2, [r3, #0]
     bb0:	69b9      	ldr	r1, [r7, #24]
     bb2:	6b7b      	ldr	r3, [r7, #52]	; 0x34
     bb4:	fbb1 f3f3 	udiv	r3, r1, r3
     bb8:	6ab9      	ldr	r1, [r7, #40]	; 0x28
     bba:	fbb3 f1f1 	udiv	r1, r3, r1
     bbe:	6ab8      	ldr	r0, [r7, #40]	; 0x28
     bc0:	fb00 f101 	mul.w	r1, r0, r1
     bc4:	1a5b      	subs	r3, r3, r1
     bc6:	18d3      	adds	r3, r2, r3
     bc8:	781a      	ldrb	r2, [r3, #0]
     bca:	f107 0108 	add.w	r1, r7, #8
     bce:	6b3b      	ldr	r3, [r7, #48]	; 0x30
     bd0:	18cb      	adds	r3, r1, r3
     bd2:	701a      	strb	r2, [r3, #0]
     bd4:	6b3b      	ldr	r3, [r7, #48]	; 0x30
     bd6:	3301      	adds	r3, #1
     bd8:	633b      	str	r3, [r7, #48]	; 0x30
                    }

                    //
                    // Convert the value into a string.
                    //
                    for(; ulIdx; ulIdx /= ulBase)
     bda:	6b7a      	ldr	r2, [r7, #52]	; 0x34
     bdc:	6abb      	ldr	r3, [r7, #40]	; 0x28
     bde:	fbb2 f3f3 	udiv	r3, r2, r3
     be2:	637b      	str	r3, [r7, #52]	; 0x34
     be4:	6b7b      	ldr	r3, [r7, #52]	; 0x34
     be6:	2b00      	cmp	r3, #0
     be8:	d1dd      	bne.n	ba6 <UARTprintf+0x386>
                    }

                    //
                    // Write the string.
                    //
                    UARTwrite(pcBuf, ulPos);
     bea:	f107 0308 	add.w	r3, r7, #8
     bee:	4618      	mov	r0, r3
     bf0:	6b39      	ldr	r1, [r7, #48]	; 0x30
     bf2:	f7ff fd2f 	bl	654 <UARTwrite>

                    //
                    // This command has been handled.
                    //
                    break;
     bf6:	e00f      	b.n	c18 <UARTprintf+0x3f8>
                case '%':
                {
                    //
                    // Simply write a single %.
                    //
                    UARTwrite(pcString - 1, 1);
     bf8:	6c3b      	ldr	r3, [r7, #64]	; 0x40
     bfa:	3b01      	subs	r3, #1
     bfc:	4618      	mov	r0, r3
     bfe:	2101      	movs	r1, #1
     c00:	f7ff fd28 	bl	654 <UARTwrite>

                    //
                    // This command has been handled.
                    //
                    break;
     c04:	e008      	b.n	c18 <UARTprintf+0x3f8>
                default:
                {
                    //
                    // Indicate an error.
                    //
                    UARTwrite("ERROR", 5);
     c06:	f242 3028 	movw	r0, #9000	; 0x2328
     c0a:	f2c0 0000 	movt	r0, #0
     c0e:	2105      	movs	r1, #5
     c10:	f7ff fd20 	bl	654 <UARTwrite>

                    //
                    // This command has been handled.
                    //
                    break;
     c14:	e000      	b.n	c18 <UARTprintf+0x3f8>
                        }
                    }
                    //
                    // This command has been handled.
                    //
                    break;
     c16:	bf00      	nop
    va_start(vaArgP, pcString);

    //
    // Loop while there are more characters in the string.
    //
    while(*pcString)
     c18:	6c3b      	ldr	r3, [r7, #64]	; 0x40
     c1a:	781b      	ldrb	r3, [r3, #0]
     c1c:	2b00      	cmp	r3, #0
     c1e:	f47f ae07 	bne.w	830 <UARTprintf+0x10>

    //
    // End the varargs processing.
    //
    va_end(vaArgP);
}
     c22:	f107 0738 	add.w	r7, r7, #56	; 0x38
     c26:	46bd      	mov	sp, r7
     c28:	e8bd 4080 	ldmia.w	sp!, {r7, lr}
     c2c:	b004      	add	sp, #16
     c2e:	4770      	bx	lr

00000c30 <UARTPeek>:
//
//*****************************************************************************
#if defined(UART_BUFFERED) || defined(DOXYGEN)
int
UARTPeek(unsigned char ucChar)
{
     c30:	b580      	push	{r7, lr}
     c32:	b086      	sub	sp, #24
     c34:	af00      	add	r7, sp, #0
     c36:	4603      	mov	r3, r0
     c38:	71fb      	strb	r3, [r7, #7]
    unsigned long ulReadIndex;

    //
    // How many characters are there in the receive buffer?
    //
    iAvail = (int)RX_BUFFER_USED;
     c3a:	f640 4090 	movw	r0, #3216	; 0xc90
     c3e:	f2c2 0000 	movt	r0, #8192	; 0x2000
     c42:	f640 418c 	movw	r1, #3212	; 0xc8c
     c46:	f2c2 0100 	movt	r1, #8192	; 0x2000
     c4a:	2280      	movs	r2, #128	; 0x80
     c4c:	f7ff fbb2 	bl	3b4 <GetBufferCount>
     c50:	4603      	mov	r3, r0
     c52:	60fb      	str	r3, [r7, #12]
    ulReadIndex = g_ulUARTRxReadIndex;
     c54:	f640 4390 	movw	r3, #3216	; 0xc90
     c58:	f2c2 0300 	movt	r3, #8192	; 0x2000
     c5c:	681b      	ldr	r3, [r3, #0]
     c5e:	613b      	str	r3, [r7, #16]

    //
    // Check all the unread characters looking for the one passed.
    //
    for(iCount = 0; iCount < iAvail; iCount++)
     c60:	2300      	movs	r3, #0
     c62:	617b      	str	r3, [r7, #20]
     c64:	e013      	b.n	c8e <UARTPeek+0x5e>
    {
        if(g_pcUARTRxBuffer[ulReadIndex] == ucChar)
     c66:	f640 430c 	movw	r3, #3084	; 0xc0c
     c6a:	f2c2 0300 	movt	r3, #8192	; 0x2000
     c6e:	693a      	ldr	r2, [r7, #16]
     c70:	189b      	adds	r3, r3, r2
     c72:	781b      	ldrb	r3, [r3, #0]
     c74:	79fa      	ldrb	r2, [r7, #7]
     c76:	429a      	cmp	r2, r3
     c78:	d101      	bne.n	c7e <UARTPeek+0x4e>
        {
            //
            // We found it so return the index
            //
            return(iCount);
     c7a:	697b      	ldr	r3, [r7, #20]
     c7c:	e00d      	b.n	c9a <UARTPeek+0x6a>
        else
        {
            //
            // This one didn't match so move on to the next character.
            //
            ADVANCE_RX_BUFFER_INDEX(ulReadIndex);
     c7e:	693b      	ldr	r3, [r7, #16]
     c80:	3301      	adds	r3, #1
     c82:	f003 037f 	and.w	r3, r3, #127	; 0x7f
     c86:	613b      	str	r3, [r7, #16]
    ulReadIndex = g_ulUARTRxReadIndex;

    //
    // Check all the unread characters looking for the one passed.
    //
    for(iCount = 0; iCount < iAvail; iCount++)
     c88:	697b      	ldr	r3, [r7, #20]
     c8a:	3301      	adds	r3, #1
     c8c:	617b      	str	r3, [r7, #20]
     c8e:	697a      	ldr	r2, [r7, #20]
     c90:	68fb      	ldr	r3, [r7, #12]
     c92:	429a      	cmp	r2, r3
     c94:	dbe7      	blt.n	c66 <UARTPeek+0x36>

    //
    // If we drop out of the loop, we didn't find the character in the receive
    // buffer.
    //
    return(-1);
     c96:	f04f 33ff 	mov.w	r3, #4294967295	; 0xffffffff
}
     c9a:	4618      	mov	r0, r3
     c9c:	f107 0718 	add.w	r7, r7, #24
     ca0:	46bd      	mov	sp, r7
     ca2:	bd80      	pop	{r7, pc}

00000ca4 <UARTFlushRx>:
//
//*****************************************************************************
#if defined(UART_BUFFERED) || defined(DOXYGEN)
void
UARTFlushRx(void)
{
     ca4:	b580      	push	{r7, lr}
     ca6:	b082      	sub	sp, #8
     ca8:	af00      	add	r7, sp, #0
    unsigned long ulInt;

    //
    // Temporarily turn off interrupts.
    //
    ulInt = MAP_IntMasterDisable();
     caa:	2348      	movs	r3, #72	; 0x48
     cac:	f2c0 1300 	movt	r3, #256	; 0x100
     cb0:	681b      	ldr	r3, [r3, #0]
     cb2:	3308      	adds	r3, #8
     cb4:	681b      	ldr	r3, [r3, #0]
     cb6:	4798      	blx	r3
     cb8:	4603      	mov	r3, r0
     cba:	607b      	str	r3, [r7, #4]

    //
    // Flush the receive buffer.
    //
    g_ulUARTRxReadIndex = 0;
     cbc:	f640 4390 	movw	r3, #3216	; 0xc90
     cc0:	f2c2 0300 	movt	r3, #8192	; 0x2000
     cc4:	2200      	movs	r2, #0
     cc6:	601a      	str	r2, [r3, #0]
    g_ulUARTRxWriteIndex = 0;
     cc8:	f640 438c 	movw	r3, #3212	; 0xc8c
     ccc:	f2c2 0300 	movt	r3, #8192	; 0x2000
     cd0:	2200      	movs	r2, #0
     cd2:	601a      	str	r2, [r3, #0]

    //
    // If interrupts were enabled when we turned them off, turn them
    // back on again.
    //
    if(!ulInt)
     cd4:	687b      	ldr	r3, [r7, #4]
     cd6:	2b00      	cmp	r3, #0
     cd8:	d106      	bne.n	ce8 <UARTFlushRx+0x44>
    {
        MAP_IntMasterEnable();
     cda:	2348      	movs	r3, #72	; 0x48
     cdc:	f2c0 1300 	movt	r3, #256	; 0x100
     ce0:	681b      	ldr	r3, [r3, #0]
     ce2:	3304      	adds	r3, #4
     ce4:	681b      	ldr	r3, [r3, #0]
     ce6:	4798      	blx	r3
    }
}
     ce8:	f107 0708 	add.w	r7, r7, #8
     cec:	46bd      	mov	sp, r7
     cee:	bd80      	pop	{r7, pc}

00000cf0 <UARTFlushTx>:
//
//*****************************************************************************
#if defined(UART_BUFFERED) || defined(DOXYGEN)
void
UARTFlushTx(tBoolean bDiscard)
{
     cf0:	b580      	push	{r7, lr}
     cf2:	b084      	sub	sp, #16
     cf4:	af00      	add	r7, sp, #0
     cf6:	4603      	mov	r3, r0
     cf8:	71fb      	strb	r3, [r7, #7]
    unsigned long ulInt;

    //
    // Should the remaining data be discarded or transmitted?
    //
    if(bDiscard)
     cfa:	79fb      	ldrb	r3, [r7, #7]
     cfc:	2b00      	cmp	r3, #0
     cfe:	d01f      	beq.n	d40 <UARTFlushTx+0x50>
    {
        //
        // The remaining data should be discarded, so temporarily turn off
        // interrupts.
        //
        ulInt = MAP_IntMasterDisable();
     d00:	2348      	movs	r3, #72	; 0x48
     d02:	f2c0 1300 	movt	r3, #256	; 0x100
     d06:	681b      	ldr	r3, [r3, #0]
     d08:	3308      	adds	r3, #8
     d0a:	681b      	ldr	r3, [r3, #0]
     d0c:	4798      	blx	r3
     d0e:	4603      	mov	r3, r0
     d10:	60fb      	str	r3, [r7, #12]

        //
        // Flush the transmit buffer.
        //
        g_ulUARTTxReadIndex = 0;
     d12:	f640 4308 	movw	r3, #3080	; 0xc08
     d16:	f2c2 0300 	movt	r3, #8192	; 0x2000
     d1a:	2200      	movs	r2, #0
     d1c:	601a      	str	r2, [r3, #0]
        g_ulUARTTxWriteIndex = 0;
     d1e:	f640 4304 	movw	r3, #3076	; 0xc04
     d22:	f2c2 0300 	movt	r3, #8192	; 0x2000
     d26:	2200      	movs	r2, #0
     d28:	601a      	str	r2, [r3, #0]

        //
        // If interrupts were enabled when we turned them off, turn them
        // back on again.
        //
        if(!ulInt)
     d2a:	68fb      	ldr	r3, [r7, #12]
     d2c:	2b00      	cmp	r3, #0
     d2e:	d115      	bne.n	d5c <UARTFlushTx+0x6c>
        {
            MAP_IntMasterEnable();
     d30:	2348      	movs	r3, #72	; 0x48
     d32:	f2c0 1300 	movt	r3, #256	; 0x100
     d36:	681b      	ldr	r3, [r3, #0]
     d38:	3304      	adds	r3, #4
     d3a:	681b      	ldr	r3, [r3, #0]
     d3c:	4798      	blx	r3
     d3e:	e00d      	b.n	d5c <UARTFlushTx+0x6c>
    else
    {
        //
        // Wait for all remaining data to be transmitted before returning.
        //
        while(!TX_BUFFER_EMPTY)
     d40:	bf00      	nop
     d42:	f640 4008 	movw	r0, #3080	; 0xc08
     d46:	f2c2 0000 	movt	r0, #8192	; 0x2000
     d4a:	f640 4104 	movw	r1, #3076	; 0xc04
     d4e:	f2c2 0100 	movt	r1, #8192	; 0x2000
     d52:	f7ff fb17 	bl	384 <IsBufferEmpty>
     d56:	4603      	mov	r3, r0
     d58:	2b00      	cmp	r3, #0
     d5a:	d0f2      	beq.n	d42 <UARTFlushTx+0x52>
        {
        }
    }
}
     d5c:	f107 0710 	add.w	r7, r7, #16
     d60:	46bd      	mov	sp, r7
     d62:	bd80      	pop	{r7, pc}

00000d64 <UARTStdioIntHandler>:
//
//*****************************************************************************
#if defined(UART_BUFFERED) || defined(DOXYGEN)
void
UARTStdioIntHandler(void)
{
     d64:	b580      	push	{r7, lr}
     d66:	b084      	sub	sp, #16
     d68:	af00      	add	r7, sp, #0
    static tBoolean bLastWasCR = false;

    //
    // Get and clear the current interrupt source(s)
    //
    ulInts = MAP_UARTIntStatus(g_ulBase, true);
     d6a:	2314      	movs	r3, #20
     d6c:	f2c0 1300 	movt	r3, #256	; 0x100
     d70:	681b      	ldr	r3, [r3, #0]
     d72:	334c      	adds	r3, #76	; 0x4c
     d74:	681b      	ldr	r3, [r3, #0]
     d76:	461a      	mov	r2, r3
     d78:	f640 4394 	movw	r3, #3220	; 0xc94
     d7c:	f2c2 0300 	movt	r3, #8192	; 0x2000
     d80:	681b      	ldr	r3, [r3, #0]
     d82:	4618      	mov	r0, r3
     d84:	2101      	movs	r1, #1
     d86:	4790      	blx	r2
     d88:	60f8      	str	r0, [r7, #12]
    MAP_UARTIntClear(g_ulBase, ulInts);
     d8a:	2314      	movs	r3, #20
     d8c:	f2c0 1300 	movt	r3, #256	; 0x100
     d90:	681b      	ldr	r3, [r3, #0]
     d92:	3350      	adds	r3, #80	; 0x50
     d94:	681b      	ldr	r3, [r3, #0]
     d96:	461a      	mov	r2, r3
     d98:	f640 4394 	movw	r3, #3220	; 0xc94
     d9c:	f2c2 0300 	movt	r3, #8192	; 0x2000
     da0:	681b      	ldr	r3, [r3, #0]
     da2:	4618      	mov	r0, r3
     da4:	68f9      	ldr	r1, [r7, #12]
     da6:	4790      	blx	r2

    //
    // Are we being interrupted because the TX FIFO has space available?
    //
    if(ulInts & UART_INT_TX)
     da8:	68fb      	ldr	r3, [r7, #12]
     daa:	f003 0320 	and.w	r3, r3, #32
     dae:	2b00      	cmp	r3, #0
     db0:	d023      	beq.n	dfa <UARTStdioIntHandler+0x96>
    {
        //
        // Move as many bytes as we can into the transmit FIFO.
        //
        UARTPrimeTransmit(g_ulBase);
     db2:	f640 4394 	movw	r3, #3220	; 0xc94
     db6:	f2c2 0300 	movt	r3, #8192	; 0x2000
     dba:	681b      	ldr	r3, [r3, #0]
     dbc:	4618      	mov	r0, r3
     dbe:	f7ff fb19 	bl	3f4 <UARTPrimeTransmit>

        //
        // If the output buffer is empty, turn off the transmit interrupt.
        //
        if(TX_BUFFER_EMPTY)
     dc2:	f640 4008 	movw	r0, #3080	; 0xc08
     dc6:	f2c2 0000 	movt	r0, #8192	; 0x2000
     dca:	f640 4104 	movw	r1, #3076	; 0xc04
     dce:	f2c2 0100 	movt	r1, #8192	; 0x2000
     dd2:	f7ff fad7 	bl	384 <IsBufferEmpty>
     dd6:	4603      	mov	r3, r0
     dd8:	2b00      	cmp	r3, #0
     dda:	d00e      	beq.n	dfa <UARTStdioIntHandler+0x96>
        {
            MAP_UARTIntDisable(g_ulBase, UART_INT_TX);
     ddc:	2314      	movs	r3, #20
     dde:	f2c0 1300 	movt	r3, #256	; 0x100
     de2:	681b      	ldr	r3, [r3, #0]
     de4:	3348      	adds	r3, #72	; 0x48
     de6:	681b      	ldr	r3, [r3, #0]
     de8:	461a      	mov	r2, r3
     dea:	f640 4394 	movw	r3, #3220	; 0xc94
     dee:	f2c2 0300 	movt	r3, #8192	; 0x2000
     df2:	681b      	ldr	r3, [r3, #0]
     df4:	4618      	mov	r0, r3
     df6:	2120      	movs	r1, #32
     df8:	4790      	blx	r2
    }

    //
    // Are we being interrupted due to a received character?
    //
    if(ulInts & (UART_INT_RX | UART_INT_RT))
     dfa:	68fb      	ldr	r3, [r7, #12]
     dfc:	f003 0350 	and.w	r3, r3, #80	; 0x50
     e00:	2b00      	cmp	r3, #0
     e02:	f000 80d6 	beq.w	fb2 <UARTStdioIntHandler+0x24e>
    {
        //
        // Get all the available characters from the UART.
        //
        while(MAP_UARTCharsAvail(g_ulBase))
     e06:	e0ab      	b.n	f60 <UARTStdioIntHandler+0x1fc>
        {
            //
            // Read a character
            //
            lChar = MAP_UARTCharGetNonBlocking(g_ulBase);
     e08:	2314      	movs	r3, #20
     e0a:	f2c0 1300 	movt	r3, #256	; 0x100
     e0e:	681b      	ldr	r3, [r3, #0]
     e10:	3334      	adds	r3, #52	; 0x34
     e12:	681b      	ldr	r3, [r3, #0]
     e14:	461a      	mov	r2, r3
     e16:	f640 4394 	movw	r3, #3220	; 0xc94
     e1a:	f2c2 0300 	movt	r3, #8192	; 0x2000
     e1e:	681b      	ldr	r3, [r3, #0]
     e20:	4618      	mov	r0, r3
     e22:	4790      	blx	r2
     e24:	60b8      	str	r0, [r7, #8]
            cChar = (unsigned char)(lChar & 0xFF);
     e26:	68bb      	ldr	r3, [r7, #8]
     e28:	b2db      	uxtb	r3, r3
     e2a:	71fb      	strb	r3, [r7, #7]
            //
            // If echo is disabled, we skip the various text filtering
            // operations that would typically be required when supporting a
            // command line.
            //
            if(!g_bDisableEcho)
     e2c:	f640 0300 	movw	r3, #2048	; 0x800
     e30:	f2c2 0300 	movt	r3, #8192	; 0x2000
     e34:	781b      	ldrb	r3, [r3, #0]
     e36:	2b00      	cmp	r3, #0
     e38:	d15d      	bne.n	ef6 <UARTStdioIntHandler+0x192>
            {
                //
                // Handle backspace by erasing the last character in the buffer.
                //
                if(cChar == '\b')
     e3a:	79fb      	ldrb	r3, [r7, #7]
     e3c:	2b08      	cmp	r3, #8
     e3e:	d12e      	bne.n	e9e <UARTStdioIntHandler+0x13a>
                {
                    //
                    // If there are any characters already in the buffer, then
                    // delete the last.
                    //
                    if(!RX_BUFFER_EMPTY)
     e40:	f640 4090 	movw	r0, #3216	; 0xc90
     e44:	f2c2 0000 	movt	r0, #8192	; 0x2000
     e48:	f640 418c 	movw	r1, #3212	; 0xc8c
     e4c:	f2c2 0100 	movt	r1, #8192	; 0x2000
     e50:	f7ff fa98 	bl	384 <IsBufferEmpty>
     e54:	4603      	mov	r3, r0
     e56:	2b00      	cmp	r3, #0
     e58:	f040 8081 	bne.w	f5e <UARTStdioIntHandler+0x1fa>
                    {
                        //
                        // Rub out the previous character on the users terminal.
                        //
                        UARTwrite("\b \b", 3);
     e5c:	f242 3030 	movw	r0, #9008	; 0x2330
     e60:	f2c0 0000 	movt	r0, #0
     e64:	2103      	movs	r1, #3
     e66:	f7ff fbf5 	bl	654 <UARTwrite>

                        //
                        // Decrement the number of characters in the buffer.
                        //
                        if(g_ulUARTRxWriteIndex == 0)
     e6a:	f640 438c 	movw	r3, #3212	; 0xc8c
     e6e:	f2c2 0300 	movt	r3, #8192	; 0x2000
     e72:	681b      	ldr	r3, [r3, #0]
     e74:	2b00      	cmp	r3, #0
     e76:	d106      	bne.n	e86 <UARTStdioIntHandler+0x122>
                        {
                            g_ulUARTRxWriteIndex = UART_RX_BUFFER_SIZE - 1;
     e78:	f640 438c 	movw	r3, #3212	; 0xc8c
     e7c:	f2c2 0300 	movt	r3, #8192	; 0x2000
     e80:	227f      	movs	r2, #127	; 0x7f
     e82:	601a      	str	r2, [r3, #0]
                    }

                    //
                    // Skip ahead to read the next character.
                    //
                    continue;
     e84:	e06b      	b.n	f5e <UARTStdioIntHandler+0x1fa>
                        {
                            g_ulUARTRxWriteIndex = UART_RX_BUFFER_SIZE - 1;
                        }
                        else
                        {
                            g_ulUARTRxWriteIndex--;
     e86:	f640 438c 	movw	r3, #3212	; 0xc8c
     e8a:	f2c2 0300 	movt	r3, #8192	; 0x2000
     e8e:	681b      	ldr	r3, [r3, #0]
     e90:	1e5a      	subs	r2, r3, #1
     e92:	f640 438c 	movw	r3, #3212	; 0xc8c
     e96:	f2c2 0300 	movt	r3, #8192	; 0x2000
     e9a:	601a      	str	r2, [r3, #0]
                    }

                    //
                    // Skip ahead to read the next character.
                    //
                    continue;
     e9c:	e05f      	b.n	f5e <UARTStdioIntHandler+0x1fa>
                // If this character is LF and last was CR, then just gobble up
                // the character since we already echoed the previous CR and we
                // don't want to store 2 characters in the buffer if we don't
                // need to.
                //
                if((cChar == '\n') && bLastWasCR)
     e9e:	79fb      	ldrb	r3, [r7, #7]
     ea0:	2b0a      	cmp	r3, #10
     ea2:	d10d      	bne.n	ec0 <UARTStdioIntHandler+0x15c>
     ea4:	f640 43a4 	movw	r3, #3236	; 0xca4
     ea8:	f2c2 0300 	movt	r3, #8192	; 0x2000
     eac:	781b      	ldrb	r3, [r3, #0]
     eae:	2b00      	cmp	r3, #0
     eb0:	d006      	beq.n	ec0 <UARTStdioIntHandler+0x15c>
                {
                    bLastWasCR = false;
     eb2:	f640 43a4 	movw	r3, #3236	; 0xca4
     eb6:	f2c2 0300 	movt	r3, #8192	; 0x2000
     eba:	2200      	movs	r2, #0
     ebc:	701a      	strb	r2, [r3, #0]
                    continue;
     ebe:	e04f      	b.n	f60 <UARTStdioIntHandler+0x1fc>
                }

                //
                // See if a newline or escape character was received.
                //
                if((cChar == '\r') || (cChar == '\n') || (cChar == 0x1b))
     ec0:	79fb      	ldrb	r3, [r7, #7]
     ec2:	2b0d      	cmp	r3, #13
     ec4:	d005      	beq.n	ed2 <UARTStdioIntHandler+0x16e>
     ec6:	79fb      	ldrb	r3, [r7, #7]
     ec8:	2b0a      	cmp	r3, #10
     eca:	d002      	beq.n	ed2 <UARTStdioIntHandler+0x16e>
     ecc:	79fb      	ldrb	r3, [r7, #7]
     ece:	2b1b      	cmp	r3, #27
     ed0:	d111      	bne.n	ef6 <UARTStdioIntHandler+0x192>
                    //
                    // If the character is a CR, then it may be followed by an
                    // LF which should be paired with the CR.  So remember that
                    // a CR was received.
                    //
                    if(cChar == '\r')
     ed2:	79fb      	ldrb	r3, [r7, #7]
     ed4:	2b0d      	cmp	r3, #13
     ed6:	d105      	bne.n	ee4 <UARTStdioIntHandler+0x180>
                    {
                        bLastWasCR = 1;
     ed8:	f640 43a4 	movw	r3, #3236	; 0xca4
     edc:	f2c2 0300 	movt	r3, #8192	; 0x2000
     ee0:	2201      	movs	r2, #1
     ee2:	701a      	strb	r2, [r3, #0]
                    // put a CR in the receive buffer as a marker telling
                    // UARTgets() where the line ends.  We also send an
                    // additional LF to ensure that the local terminal echo
                    // receives both CR and LF.
                    //
                    cChar = '\r';
     ee4:	230d      	movs	r3, #13
     ee6:	71fb      	strb	r3, [r7, #7]
                    UARTwrite("\n", 1);
     ee8:	f242 3034 	movw	r0, #9012	; 0x2334
     eec:	f2c0 0000 	movt	r0, #0
     ef0:	2101      	movs	r1, #1
     ef2:	f7ff fbaf 	bl	654 <UARTwrite>

            //
            // If there is space in the receive buffer, put the character
            // there, otherwise throw it away.
            //
            if(!RX_BUFFER_FULL)
     ef6:	f640 4090 	movw	r0, #3216	; 0xc90
     efa:	f2c2 0000 	movt	r0, #8192	; 0x2000
     efe:	f640 418c 	movw	r1, #3212	; 0xc8c
     f02:	f2c2 0100 	movt	r1, #8192	; 0x2000
     f06:	2280      	movs	r2, #128	; 0x80
     f08:	f7ff fa1a 	bl	340 <IsBufferFull>
     f0c:	4603      	mov	r3, r0
     f0e:	2b00      	cmp	r3, #0
     f10:	d126      	bne.n	f60 <UARTStdioIntHandler+0x1fc>
            {
                //
                // Store the new character in the receive buffer
                //
                g_pcUARTRxBuffer[g_ulUARTRxWriteIndex] =
     f12:	f640 438c 	movw	r3, #3212	; 0xc8c
     f16:	f2c2 0300 	movt	r3, #8192	; 0x2000
     f1a:	681a      	ldr	r2, [r3, #0]
                    (unsigned char)(lChar & 0xFF);
     f1c:	68bb      	ldr	r3, [r7, #8]
     f1e:	b2d9      	uxtb	r1, r3
            if(!RX_BUFFER_FULL)
            {
                //
                // Store the new character in the receive buffer
                //
                g_pcUARTRxBuffer[g_ulUARTRxWriteIndex] =
     f20:	f640 430c 	movw	r3, #3084	; 0xc0c
     f24:	f2c2 0300 	movt	r3, #8192	; 0x2000
     f28:	5499      	strb	r1, [r3, r2]
                    (unsigned char)(lChar & 0xFF);
                ADVANCE_RX_BUFFER_INDEX(g_ulUARTRxWriteIndex);
     f2a:	f640 438c 	movw	r3, #3212	; 0xc8c
     f2e:	f2c2 0300 	movt	r3, #8192	; 0x2000
     f32:	681b      	ldr	r3, [r3, #0]
     f34:	3301      	adds	r3, #1
     f36:	f003 027f 	and.w	r2, r3, #127	; 0x7f
     f3a:	f640 438c 	movw	r3, #3212	; 0xc8c
     f3e:	f2c2 0300 	movt	r3, #8192	; 0x2000
     f42:	601a      	str	r2, [r3, #0]

                //
                // If echo is enabled, write the character to the transmit
                // buffer so that the user gets some immediate feedback.
                //
                if(!g_bDisableEcho)
     f44:	f640 0300 	movw	r3, #2048	; 0x800
     f48:	f2c2 0300 	movt	r3, #8192	; 0x2000
     f4c:	781b      	ldrb	r3, [r3, #0]
     f4e:	2b00      	cmp	r3, #0
     f50:	d106      	bne.n	f60 <UARTStdioIntHandler+0x1fc>
                {
                    UARTwrite(&cChar, 1);
     f52:	1dfb      	adds	r3, r7, #7
     f54:	4618      	mov	r0, r3
     f56:	2101      	movs	r1, #1
     f58:	f7ff fb7c 	bl	654 <UARTwrite>
     f5c:	e000      	b.n	f60 <UARTStdioIntHandler+0x1fc>
                    }

                    //
                    // Skip ahead to read the next character.
                    //
                    continue;
     f5e:	bf00      	nop
    if(ulInts & (UART_INT_RX | UART_INT_RT))
    {
        //
        // Get all the available characters from the UART.
        //
        while(MAP_UARTCharsAvail(g_ulBase))
     f60:	2314      	movs	r3, #20
     f62:	f2c0 1300 	movt	r3, #256	; 0x100
     f66:	681b      	ldr	r3, [r3, #0]
     f68:	332c      	adds	r3, #44	; 0x2c
     f6a:	681b      	ldr	r3, [r3, #0]
     f6c:	461a      	mov	r2, r3
     f6e:	f640 4394 	movw	r3, #3220	; 0xc94
     f72:	f2c2 0300 	movt	r3, #8192	; 0x2000
     f76:	681b      	ldr	r3, [r3, #0]
     f78:	4618      	mov	r0, r3
     f7a:	4790      	blx	r2
     f7c:	4603      	mov	r3, r0
     f7e:	2b00      	cmp	r3, #0
     f80:	f47f af42 	bne.w	e08 <UARTStdioIntHandler+0xa4>

        //
        // If we wrote anything to the transmit buffer, make sure it actually
        // gets transmitted.
        //
        UARTPrimeTransmit(g_ulBase);
     f84:	f640 4394 	movw	r3, #3220	; 0xc94
     f88:	f2c2 0300 	movt	r3, #8192	; 0x2000
     f8c:	681b      	ldr	r3, [r3, #0]
     f8e:	4618      	mov	r0, r3
     f90:	f7ff fa30 	bl	3f4 <UARTPrimeTransmit>
        MAP_UARTIntEnable(g_ulBase, UART_INT_TX);
     f94:	2314      	movs	r3, #20
     f96:	f2c0 1300 	movt	r3, #256	; 0x100
     f9a:	681b      	ldr	r3, [r3, #0]
     f9c:	3344      	adds	r3, #68	; 0x44
     f9e:	681b      	ldr	r3, [r3, #0]
     fa0:	461a      	mov	r2, r3
     fa2:	f640 4394 	movw	r3, #3220	; 0xc94
     fa6:	f2c2 0300 	movt	r3, #8192	; 0x2000
     faa:	681b      	ldr	r3, [r3, #0]
     fac:	4618      	mov	r0, r3
     fae:	2120      	movs	r1, #32
     fb0:	4790      	blx	r2
    }
}
     fb2:	f107 0710 	add.w	r7, r7, #16
     fb6:	46bd      	mov	sp, r7
     fb8:	bd80      	pop	{r7, pc}
     fba:	bf00      	nop

00000fbc <initUART>:
static unsigned long countToDelay = 10;


void pwmTimerIsr(void);

void initUART() {
     fbc:	b580      	push	{r7, lr}
     fbe:	af00      	add	r7, sp, #0
	SysCtlPeripheralEnable(SYSCTL_PERIPH_GPIOA);
     fc0:	2001      	movs	r0, #1
     fc2:	f2c2 0000 	movt	r0, #8192	; 0x2000
     fc6:	f000 fbe1 	bl	178c <SysCtlPeripheralEnable>
	GPIOPinConfigure(GPIO_PA0_U0RX);
     fca:	2001      	movs	r0, #1
     fcc:	f000 faf0 	bl	15b0 <GPIOPinConfigure>
	GPIOPinConfigure(GPIO_PA1_U0TX);
     fd0:	f240 4001 	movw	r0, #1025	; 0x401
     fd4:	f000 faec 	bl	15b0 <GPIOPinConfigure>
	GPIOPinTypeUART(GPIO_PORTA_BASE, GPIO_PIN_0 | GPIO_PIN_1);
     fd8:	f04f 2040 	mov.w	r0, #1073758208	; 0x40004000
     fdc:	2103      	movs	r1, #3
     fde:	f000 facf 	bl	1580 <GPIOPinTypeUART>
	UARTStdioInit(0);
     fe2:	2000      	movs	r0, #0
     fe4:	f7ff fb20 	bl	628 <UARTStdioInit>
}
     fe8:	bd80      	pop	{r7, pc}
     fea:	bf00      	nop

00000fec <loopUART_cmd>:
char cmd[128];
void loopUART_cmd() {
     fec:	b580      	push	{r7, lr}
     fee:	af00      	add	r7, sp, #0
	while (1) {
		UARTprintf("\n>");
     ff0:	f242 3038 	movw	r0, #9016	; 0x2338
     ff4:	f2c0 0000 	movt	r0, #0
     ff8:	f7ff fc12 	bl	820 <UARTprintf>
		while (UARTPeek('\r') == -1) {
     ffc:	e010      	b.n	1020 <loopUART_cmd+0x34>
			SysCtlDelay(10 * (SysCtlClockGet() / 1000));
     ffe:	f000 fd61 	bl	1ac4 <SysCtlClockGet>
    1002:	4602      	mov	r2, r0
    1004:	f644 53d3 	movw	r3, #19923	; 0x4dd3
    1008:	f2c1 0362 	movt	r3, #4194	; 0x1062
    100c:	fba3 1302 	umull	r1, r3, r3, r2
    1010:	099a      	lsrs	r2, r3, #6
    1012:	4613      	mov	r3, r2
    1014:	009b      	lsls	r3, r3, #2
    1016:	189b      	adds	r3, r3, r2
    1018:	005b      	lsls	r3, r3, #1
    101a:	4618      	mov	r0, r3
    101c:	f000 fc02 	bl	1824 <SysCtlDelay>
}
char cmd[128];
void loopUART_cmd() {
	while (1) {
		UARTprintf("\n>");
		while (UARTPeek('\r') == -1) {
    1020:	200d      	movs	r0, #13
    1022:	f7ff fe05 	bl	c30 <UARTPeek>
    1026:	4603      	mov	r3, r0
    1028:	f1b3 3fff 	cmp.w	r3, #4294967295	; 0xffffffff
    102c:	d0e7      	beq.n	ffe <loopUART_cmd+0x12>
			SysCtlDelay(10 * (SysCtlClockGet() / 1000));
		}
		UARTgets(cmd, sizeof(cmd));
    102e:	f640 40a8 	movw	r0, #3240	; 0xca8
    1032:	f2c2 0000 	movt	r0, #8192	; 0x2000
    1036:	2180      	movs	r1, #128	; 0x80
    1038:	f7ff fba0 	bl	77c <UARTgets>
		UARTprintf("%s\n", cmd);
    103c:	f242 303c 	movw	r0, #9020	; 0x233c
    1040:	f2c0 0000 	movt	r0, #0
    1044:	f640 41a8 	movw	r1, #3240	; 0xca8
    1048:	f2c2 0100 	movt	r1, #8192	; 0x2000
    104c:	f7ff fbe8 	bl	820 <UARTprintf>
	}
    1050:	e7ce      	b.n	ff0 <loopUART_cmd+0x4>
    1052:	bf00      	nop

00001054 <initPWM>:
}

void initPWM() {
    1054:	b580      	push	{r7, lr}
    1056:	af00      	add	r7, sp, #0
	pwm_period = SysCtlClockGet() / PWM_FREQUENCY;
    1058:	f000 fd34 	bl	1ac4 <SysCtlClockGet>
    105c:	4602      	mov	r2, r0
    105e:	f241 7359 	movw	r3, #5977	; 0x1759
    1062:	f2cd 13b7 	movt	r3, #53687	; 0xd1b7
    1066:	fba3 1302 	umull	r1, r3, r3, r2
    106a:	0bda      	lsrs	r2, r3, #15
    106c:	f640 439c 	movw	r3, #3228	; 0xc9c
    1070:	f2c2 0300 	movt	r3, #8192	; 0x2000
    1074:	601a      	str	r2, [r3, #0]
	SysCtlPeripheralEnable(PWM_TIMER_PERIPH);
    1076:	2004      	movs	r0, #4
    1078:	f2c1 0010 	movt	r0, #4112	; 0x1010
    107c:	f000 fb86 	bl	178c <SysCtlPeripheralEnable>
//	SysCtlPeripheralEnable(CTRL_TIMER_PERIPH);
	SysCtlPeripheralEnable(PWM_TIMER_A_PIN_PERIPH);
    1080:	2002      	movs	r0, #2
    1082:	f2c2 0000 	movt	r0, #8192	; 0x2000
    1086:	f000 fb81 	bl	178c <SysCtlPeripheralEnable>
	SysCtlPeripheralEnable(PWM_TIMER_B_PIN_PERIPH);
    108a:	2002      	movs	r0, #2
    108c:	f2c2 0000 	movt	r0, #8192	; 0x2000
    1090:	f000 fb7c 	bl	178c <SysCtlPeripheralEnable>
	TimerConfigure(PWM_TIMER_BASE,
    1094:	f44f 5000 	mov.w	r0, #8192	; 0x2000
    1098:	f2c4 0003 	movt	r0, #16387	; 0x4003
    109c:	f640 210a 	movw	r1, #2570	; 0xa0a
    10a0:	f2c0 4100 	movt	r1, #1024	; 0x400
    10a4:	f000 ff50 	bl	1f48 <TimerConfigure>
			TIMER_CFG_SPLIT_PAIR | TIMER_CFG_A_PWM | TIMER_CFG_B_PWM);
//	TimerConfigure(CTRL_TIMER_BASE,
//			TIMER_CFG_SPLIT_PAIR | TIMER_CFG_A_PERIODIC);
	TimerControlStall(PWM_TIMER_BASE, TIMER_BOTH, true);
    10a8:	f44f 5000 	mov.w	r0, #8192	; 0x2000
    10ac:	f2c4 0003 	movt	r0, #16387	; 0x4003
    10b0:	f64f 71ff 	movw	r1, #65535	; 0xffff
    10b4:	2201      	movs	r2, #1
    10b6:	f000 ff8d 	bl	1fd4 <TimerControlStall>
//	TimerControlStall(CTRL_TIMER_BASE,TIMER_A,true);
	TimerLoadSet(PWM_TIMER_BASE, TIMER_BOTH, pwm_period - 1);
    10ba:	f640 439c 	movw	r3, #3228	; 0xc9c
    10be:	f2c2 0300 	movt	r3, #8192	; 0x2000
    10c2:	681b      	ldr	r3, [r3, #0]
    10c4:	3b01      	subs	r3, #1
    10c6:	f44f 5000 	mov.w	r0, #8192	; 0x2000
    10ca:	f2c4 0003 	movt	r0, #16387	; 0x4003
    10ce:	f64f 71ff 	movw	r1, #65535	; 0xffff
    10d2:	461a      	mov	r2, r3
    10d4:	f000 ffa2 	bl	201c <TimerLoadSet>
//	TimerLoadSet(CTRL_TIMER_BASE, TIMER_A, pwm_period - 1);
	TimerMatchSet(PWM_TIMER_BASE, TIMER_BOTH, pwm_period / 2 - 1);
    10d8:	f640 439c 	movw	r3, #3228	; 0xc9c
    10dc:	f2c2 0300 	movt	r3, #8192	; 0x2000
    10e0:	681b      	ldr	r3, [r3, #0]
    10e2:	085b      	lsrs	r3, r3, #1
    10e4:	3b01      	subs	r3, #1
    10e6:	f44f 5000 	mov.w	r0, #8192	; 0x2000
    10ea:	f2c4 0003 	movt	r0, #16387	; 0x4003
    10ee:	f64f 71ff 	movw	r1, #65535	; 0xffff
    10f2:	461a      	mov	r2, r3
    10f4:	f000 ffae 	bl	2054 <TimerMatchSet>
	TimerControlEvent(PWM_TIMER_BASE, TIMER_BOTH, TIMER_EVENT_NEG_EDGE);
    10f8:	f44f 5000 	mov.w	r0, #8192	; 0x2000
    10fc:	f2c4 0003 	movt	r0, #16387	; 0x4003
    1100:	f64f 71ff 	movw	r1, #65535	; 0xffff
    1104:	f240 4204 	movw	r2, #1028	; 0x404
    1108:	f000 ff46 	bl	1f98 <TimerControlEvent>
	TimerIntRegister(PWM_TIMER_BASE, TIMER_BOTH, pwmTimerIsr);
    110c:	f44f 5000 	mov.w	r0, #8192	; 0x2000
    1110:	f2c4 0003 	movt	r0, #16387	; 0x4003
    1114:	f64f 71ff 	movw	r1, #65535	; 0xffff
    1118:	f241 12ed 	movw	r2, #4589	; 0x11ed
    111c:	f2c0 0200 	movt	r2, #0
    1120:	f000 ffca 	bl	20b8 <TimerIntRegister>
	TimerIntEnable(PWM_TIMER_BASE, TIMER_CAPA_EVENT | TIMER_CAPB_EVENT); //TIMER_TIMA_MATCH | TIMER_TIMB_MATCH
    1124:	f44f 5000 	mov.w	r0, #8192	; 0x2000
    1128:	f2c4 0003 	movt	r0, #16387	; 0x4003
    112c:	f240 4104 	movw	r1, #1028	; 0x404
    1130:	f000 ffec 	bl	210c <TimerIntEnable>
	GPIOPinConfigure(PWM_TIMER_A_PIN_CFG);
    1134:	2007      	movs	r0, #7
    1136:	f2c0 0001 	movt	r0, #1
    113a:	f000 fa39 	bl	15b0 <GPIOPinConfigure>
	GPIOPinTypeTimer(PWM_TIMER_A_PIN_BASE, PWM_TIMER_A_PIN);
    113e:	f44f 40a0 	mov.w	r0, #20480	; 0x5000
    1142:	f2c4 0000 	movt	r0, #16384	; 0x4000
    1146:	2101      	movs	r1, #1
    1148:	f000 fa02 	bl	1550 <GPIOPinTypeTimer>
	GPIOPadConfigSet(PWM_TIMER_A_PIN_BASE, PWM_TIMER_A_PIN,
    114c:	f44f 40a0 	mov.w	r0, #20480	; 0x5000
    1150:	f2c4 0000 	movt	r0, #16384	; 0x4000
    1154:	2101      	movs	r1, #1
    1156:	220c      	movs	r2, #12
    1158:	2308      	movs	r3, #8
    115a:	f000 f915 	bl	1388 <GPIOPadConfigSet>
			GPIO_STRENGTH_8MA_SC, GPIO_PIN_TYPE_STD);
	GPIOPinConfigure(PWM_TIMER_B_PIN_CFG);
    115e:	f240 4007 	movw	r0, #1031	; 0x407
    1162:	f2c0 0001 	movt	r0, #1
    1166:	f000 fa23 	bl	15b0 <GPIOPinConfigure>
	GPIOPinTypeTimer(PWM_TIMER_B_PIN_BASE, PWM_TIMER_B_PIN);
    116a:	f44f 40a0 	mov.w	r0, #20480	; 0x5000
    116e:	f2c4 0000 	movt	r0, #16384	; 0x4000
    1172:	2102      	movs	r1, #2
    1174:	f000 f9ec 	bl	1550 <GPIOPinTypeTimer>
	GPIOPadConfigSet(PWM_TIMER_B_PIN_BASE, PWM_TIMER_B_PIN,
    1178:	f44f 40a0 	mov.w	r0, #20480	; 0x5000
    117c:	f2c4 0000 	movt	r0, #16384	; 0x4000
    1180:	2102      	movs	r1, #2
    1182:	220c      	movs	r2, #12
    1184:	2308      	movs	r3, #8
    1186:	f000 f8ff 	bl	1388 <GPIOPadConfigSet>
			GPIO_STRENGTH_8MA_SC, GPIO_PIN_TYPE_STD);
//	TimerEnable(CTRL_TIMER_BASE, TIMER_A);
	TimerEnable(PWM_TIMER_BASE, TIMER_BOTH);
    118a:	f44f 5000 	mov.w	r0, #8192	; 0x2000
    118e:	f2c4 0003 	movt	r0, #16387	; 0x4003
    1192:	f64f 71ff 	movw	r1, #65535	; 0xffff
    1196:	f000 fec1 	bl	1f1c <TimerEnable>
	//TimerSynchronize(TIMER0_BASE,PWM_TIMER_A_SYNC|PWM_TIMER_B_SYNC|CTRL_TIMER_SYNC);
}
    119a:	bd80      	pop	{r7, pc}

0000119c <main>:

// main function.
int main(void) {
    119c:	b580      	push	{r7, lr}
    119e:	af00      	add	r7, sp, #0
	FPUEnable();
    11a0:	f000 f890 	bl	12c4 <FPUEnable>
	FPUStackingEnable();
    11a4:	f000 f8a0 	bl	12e8 <FPUStackingEnable>
	SysCtlClockSet(
    11a8:	f44f 60a8 	mov.w	r0, #1344	; 0x540
    11ac:	f2cc 1000 	movt	r0, #49408	; 0xc100
    11b0:	f000 fb3c 	bl	182c <SysCtlClockSet>
			SYSCTL_SYSDIV_2_5 | SYSCTL_USE_PLL | SYSCTL_OSC_MAIN
					| SYSCTL_XTAL_16MHZ);
	initUART();
    11b4:	f7ff ff02 	bl	fbc <initUART>
	initPWM();
    11b8:	f7ff ff4c 	bl	1054 <initPWM>
	SysTickPeriodSet(SysCtlClockGet() / SYSTICKS_PER_SEC);
    11bc:	f000 fc82 	bl	1ac4 <SysCtlClockGet>
    11c0:	4602      	mov	r2, r0
    11c2:	f248 531f 	movw	r3, #34079	; 0x851f
    11c6:	f2c5 13eb 	movt	r3, #20971	; 0x51eb
    11ca:	fba3 1302 	umull	r1, r3, r3, r2
    11ce:	095b      	lsrs	r3, r3, #5
    11d0:	4618      	mov	r0, r3
    11d2:	f000 fe6b 	bl	1eac <SysTickPeriodSet>
	SysTickEnable();
    11d6:	f000 fe45 	bl	1e64 <SysTickEnable>
	SysTickIntEnable();
    11da:	f000 fe55 	bl	1e88 <SysTickIntEnable>
	IntMasterEnable();
    11de:	f000 fa2d 	bl	163c <IntMasterEnable>

	loopUART_cmd();
    11e2:	f7ff ff03 	bl	fec <loopUART_cmd>
}
    11e6:	4618      	mov	r0, r3
    11e8:	bd80      	pop	{r7, pc}
    11ea:	bf00      	nop

000011ec <pwmTimerIsr>:

// The interrupt function definition.
void pwmTimerIsr(void) {
    11ec:	b580      	push	{r7, lr}
    11ee:	b082      	sub	sp, #8
    11f0:	af00      	add	r7, sp, #0
	unsigned long status = TimerIntStatus(PWM_TIMER_BASE, true);
    11f2:	f44f 5000 	mov.w	r0, #8192	; 0x2000
    11f6:	f2c4 0003 	movt	r0, #16387	; 0x4003
    11fa:	2101      	movs	r1, #1
    11fc:	f000 ff98 	bl	2130 <TimerIntStatus>
    1200:	6038      	str	r0, [r7, #0]
	TimerIntClear(PWM_TIMER_BASE, PWM_TIMER_INT_TRIGGER);
    1202:	f44f 5000 	mov.w	r0, #8192	; 0x2000
    1206:	f2c4 0003 	movt	r0, #16387	; 0x4003
    120a:	f240 4104 	movw	r1, #1028	; 0x404
    120e:	f000 ffa5 	bl	215c <TimerIntClear>
	if (status & PWM_TIMER_B_INT_TRIGGER) {
    1212:	683b      	ldr	r3, [r7, #0]
    1214:	f403 6380 	and.w	r3, r3, #1024	; 0x400
    1218:	2b00      	cmp	r3, #0
    121a:	d049      	beq.n	12b0 <pwmTimerIsr+0xc4>
		if (++count >= countToDelay) {
    121c:	f640 43a0 	movw	r3, #3232	; 0xca0
    1220:	f2c2 0300 	movt	r3, #8192	; 0x2000
    1224:	681b      	ldr	r3, [r3, #0]
    1226:	1c5a      	adds	r2, r3, #1
    1228:	f640 43a0 	movw	r3, #3232	; 0xca0
    122c:	f2c2 0300 	movt	r3, #8192	; 0x2000
    1230:	601a      	str	r2, [r3, #0]
    1232:	f640 43a0 	movw	r3, #3232	; 0xca0
    1236:	f2c2 0300 	movt	r3, #8192	; 0x2000
    123a:	681a      	ldr	r2, [r3, #0]
    123c:	f240 0304 	movw	r3, #4
    1240:	f2c2 0300 	movt	r3, #8192	; 0x2000
    1244:	681b      	ldr	r3, [r3, #0]
    1246:	429a      	cmp	r2, r3
    1248:	d332      	bcc.n	12b0 <pwmTimerIsr+0xc4>
			count = 0;
    124a:	f640 43a0 	movw	r3, #3232	; 0xca0
    124e:	f2c2 0300 	movt	r3, #8192	; 0x2000
    1252:	2200      	movs	r2, #0
    1254:	601a      	str	r2, [r3, #0]
			unsigned long m = TimerMatchGet(PWM_TIMER_BASE, TIMER_B) - step;
    1256:	f44f 5000 	mov.w	r0, #8192	; 0x2000
    125a:	f2c4 0003 	movt	r0, #16387	; 0x4003
    125e:	f44f 417f 	mov.w	r1, #65280	; 0xff00
    1262:	f000 ff13 	bl	208c <TimerMatchGet>
    1266:	4602      	mov	r2, r0
    1268:	f240 0300 	movw	r3, #0
    126c:	f2c2 0300 	movt	r3, #8192	; 0x2000
    1270:	681b      	ldr	r3, [r3, #0]
    1272:	1ad3      	subs	r3, r2, r3
    1274:	607b      	str	r3, [r7, #4]
			while (m < 0)
    1276:	bf00      	nop
				m += pwm_period - 2;
			while (m >= pwm_period-1)
    1278:	e008      	b.n	128c <pwmTimerIsr+0xa0>
				m -= pwm_period - 2;
    127a:	f640 439c 	movw	r3, #3228	; 0xc9c
    127e:	f2c2 0300 	movt	r3, #8192	; 0x2000
    1282:	681b      	ldr	r3, [r3, #0]
    1284:	687a      	ldr	r2, [r7, #4]
    1286:	1ad3      	subs	r3, r2, r3
    1288:	3302      	adds	r3, #2
    128a:	607b      	str	r3, [r7, #4]
		if (++count >= countToDelay) {
			count = 0;
			unsigned long m = TimerMatchGet(PWM_TIMER_BASE, TIMER_B) - step;
			while (m < 0)
				m += pwm_period - 2;
			while (m >= pwm_period-1)
    128c:	f640 439c 	movw	r3, #3228	; 0xc9c
    1290:	f2c2 0300 	movt	r3, #8192	; 0x2000
    1294:	681b      	ldr	r3, [r3, #0]
    1296:	1e5a      	subs	r2, r3, #1
    1298:	687b      	ldr	r3, [r7, #4]
    129a:	429a      	cmp	r2, r3
    129c:	d9ed      	bls.n	127a <pwmTimerIsr+0x8e>
				m -= pwm_period - 2;
			TimerMatchSet(PWM_TIMER_BASE, TIMER_B, m);
    129e:	f44f 5000 	mov.w	r0, #8192	; 0x2000
    12a2:	f2c4 0003 	movt	r0, #16387	; 0x4003
    12a6:	f44f 417f 	mov.w	r1, #65280	; 0xff00
    12aa:	687a      	ldr	r2, [r7, #4]
    12ac:	f000 fed2 	bl	2054 <TimerMatchSet>
		}
	}
}
    12b0:	f107 0708 	add.w	r7, r7, #8
    12b4:	46bd      	mov	sp, r7
    12b6:	bd80      	pop	{r7, pc}

000012b8 <SysTickIntHandler>:
void SysTickIntHandler() {
    12b8:	b480      	push	{r7}
    12ba:	af00      	add	r7, sp, #0

}
    12bc:	46bd      	mov	sp, r7
    12be:	bc80      	pop	{r7}
    12c0:	4770      	bx	lr
    12c2:	bf00      	nop

000012c4 <FPUEnable>:
//! \return None.
//
//*****************************************************************************
void
FPUEnable(void)
{
    12c4:	b480      	push	{r7}
    12c6:	af00      	add	r7, sp, #0
    //
    // Enable the coprocessors used by the floating-point unit.
    //
    HWREG(NVIC_CPAC) = ((HWREG(NVIC_CPAC) &
    12c8:	f64e 5388 	movw	r3, #60808	; 0xed88
    12cc:	f2ce 0300 	movt	r3, #57344	; 0xe000
    12d0:	f64e 5288 	movw	r2, #60808	; 0xed88
    12d4:	f2ce 0200 	movt	r2, #57344	; 0xe000
    12d8:	6812      	ldr	r2, [r2, #0]
                         ~(NVIC_CPAC_CP10_M | NVIC_CPAC_CP11_M)) |
                        NVIC_CPAC_CP10_FULL | NVIC_CPAC_CP11_FULL);
    12da:	f442 0270 	orr.w	r2, r2, #15728640	; 0xf00000
FPUEnable(void)
{
    //
    // Enable the coprocessors used by the floating-point unit.
    //
    HWREG(NVIC_CPAC) = ((HWREG(NVIC_CPAC) &
    12de:	601a      	str	r2, [r3, #0]
                         ~(NVIC_CPAC_CP10_M | NVIC_CPAC_CP11_M)) |
                        NVIC_CPAC_CP10_FULL | NVIC_CPAC_CP11_FULL);
}
    12e0:	46bd      	mov	sp, r7
    12e2:	bc80      	pop	{r7}
    12e4:	4770      	bx	lr
    12e6:	bf00      	nop

000012e8 <FPUStackingEnable>:
//! \return None.
//
//*****************************************************************************
void
FPUStackingEnable(void)
{
    12e8:	b480      	push	{r7}
    12ea:	af00      	add	r7, sp, #0
    //
    // Enable automatic state preservation for the floating-point unit, and
    // disable lazy state preservation (meaning that the floating-point state
    // is always stacked when floating-point instructions are used).
    //
    HWREG(NVIC_FPCC) = (HWREG(NVIC_FPCC) & ~NVIC_FPCC_LSPEN) | NVIC_FPCC_ASPEN;
    12ec:	f64e 7334 	movw	r3, #61236	; 0xef34
    12f0:	f2ce 0300 	movt	r3, #57344	; 0xe000
    12f4:	f64e 7234 	movw	r2, #61236	; 0xef34
    12f8:	f2ce 0200 	movt	r2, #57344	; 0xe000
    12fc:	6812      	ldr	r2, [r2, #0]
    12fe:	f022 4240 	bic.w	r2, r2, #3221225472	; 0xc0000000
    1302:	f042 4200 	orr.w	r2, r2, #2147483648	; 0x80000000
    1306:	601a      	str	r2, [r3, #0]
}
    1308:	46bd      	mov	sp, r7
    130a:	bc80      	pop	{r7}
    130c:	4770      	bx	lr
    130e:	bf00      	nop

00001310 <GPIODirModeSet>:
//
//*****************************************************************************
void
GPIODirModeSet(unsigned long ulPort, unsigned char ucPins,
               unsigned long ulPinIO)
{
    1310:	b480      	push	{r7}
    1312:	b085      	sub	sp, #20
    1314:	af00      	add	r7, sp, #0
    1316:	60f8      	str	r0, [r7, #12]
    1318:	460b      	mov	r3, r1
    131a:	607a      	str	r2, [r7, #4]
    131c:	72fb      	strb	r3, [r7, #11]
           (ulPinIO == GPIO_DIR_MODE_HW));

    //
    // Set the pin direction and mode.
    //
    HWREG(ulPort + GPIO_O_DIR) = ((ulPinIO & 1) ?
    131e:	68fb      	ldr	r3, [r7, #12]
    1320:	f503 6380 	add.w	r3, r3, #1024	; 0x400
    1324:	461a      	mov	r2, r3
    1326:	687b      	ldr	r3, [r7, #4]
    1328:	f003 0301 	and.w	r3, r3, #1
                                  (HWREG(ulPort + GPIO_O_DIR) | ucPins) :
    132c:	2b00      	cmp	r3, #0
    132e:	d006      	beq.n	133e <GPIODirModeSet+0x2e>
    1330:	68fb      	ldr	r3, [r7, #12]
    1332:	f503 6380 	add.w	r3, r3, #1024	; 0x400
    1336:	6819      	ldr	r1, [r3, #0]
    1338:	7afb      	ldrb	r3, [r7, #11]
    133a:	430b      	orrs	r3, r1
    133c:	e006      	b.n	134c <GPIODirModeSet+0x3c>
                                  (HWREG(ulPort + GPIO_O_DIR) & ~(ucPins)));
    133e:	68fb      	ldr	r3, [r7, #12]
    1340:	f503 6380 	add.w	r3, r3, #1024	; 0x400
    1344:	6819      	ldr	r1, [r3, #0]
    1346:	7afb      	ldrb	r3, [r7, #11]
    1348:	43db      	mvns	r3, r3

    //
    // Set the pin direction and mode.
    //
    HWREG(ulPort + GPIO_O_DIR) = ((ulPinIO & 1) ?
                                  (HWREG(ulPort + GPIO_O_DIR) | ucPins) :
    134a:	400b      	ands	r3, r1
           (ulPinIO == GPIO_DIR_MODE_HW));

    //
    // Set the pin direction and mode.
    //
    HWREG(ulPort + GPIO_O_DIR) = ((ulPinIO & 1) ?
    134c:	6013      	str	r3, [r2, #0]
                                  (HWREG(ulPort + GPIO_O_DIR) | ucPins) :
                                  (HWREG(ulPort + GPIO_O_DIR) & ~(ucPins)));
    HWREG(ulPort + GPIO_O_AFSEL) = ((ulPinIO & 2) ?
    134e:	68fb      	ldr	r3, [r7, #12]
    1350:	f503 6384 	add.w	r3, r3, #1056	; 0x420
    1354:	461a      	mov	r2, r3
    1356:	687b      	ldr	r3, [r7, #4]
    1358:	f003 0302 	and.w	r3, r3, #2
                                    (HWREG(ulPort + GPIO_O_AFSEL) | ucPins) :
    135c:	2b00      	cmp	r3, #0
    135e:	d006      	beq.n	136e <GPIODirModeSet+0x5e>
    1360:	68fb      	ldr	r3, [r7, #12]
    1362:	f503 6384 	add.w	r3, r3, #1056	; 0x420
    1366:	6819      	ldr	r1, [r3, #0]
    1368:	7afb      	ldrb	r3, [r7, #11]
    136a:	430b      	orrs	r3, r1
    136c:	e006      	b.n	137c <GPIODirModeSet+0x6c>
                                    (HWREG(ulPort + GPIO_O_AFSEL) &
    136e:	68fb      	ldr	r3, [r7, #12]
    1370:	f503 6384 	add.w	r3, r3, #1056	; 0x420
    1374:	6819      	ldr	r1, [r3, #0]
                                     ~(ucPins)));
    1376:	7afb      	ldrb	r3, [r7, #11]
    1378:	43db      	mvns	r3, r3
    //
    HWREG(ulPort + GPIO_O_DIR) = ((ulPinIO & 1) ?
                                  (HWREG(ulPort + GPIO_O_DIR) | ucPins) :
                                  (HWREG(ulPort + GPIO_O_DIR) & ~(ucPins)));
    HWREG(ulPort + GPIO_O_AFSEL) = ((ulPinIO & 2) ?
                                    (HWREG(ulPort + GPIO_O_AFSEL) | ucPins) :
    137a:	400b      	ands	r3, r1
    // Set the pin direction and mode.
    //
    HWREG(ulPort + GPIO_O_DIR) = ((ulPinIO & 1) ?
                                  (HWREG(ulPort + GPIO_O_DIR) | ucPins) :
                                  (HWREG(ulPort + GPIO_O_DIR) & ~(ucPins)));
    HWREG(ulPort + GPIO_O_AFSEL) = ((ulPinIO & 2) ?
    137c:	6013      	str	r3, [r2, #0]
                                    (HWREG(ulPort + GPIO_O_AFSEL) | ucPins) :
                                    (HWREG(ulPort + GPIO_O_AFSEL) &
                                     ~(ucPins)));
}
    137e:	f107 0714 	add.w	r7, r7, #20
    1382:	46bd      	mov	sp, r7
    1384:	bc80      	pop	{r7}
    1386:	4770      	bx	lr

00001388 <GPIOPadConfigSet>:
//
//*****************************************************************************
void
GPIOPadConfigSet(unsigned long ulPort, unsigned char ucPins,
                 unsigned long ulStrength, unsigned long ulPinType)
{
    1388:	b480      	push	{r7}
    138a:	b085      	sub	sp, #20
    138c:	af00      	add	r7, sp, #0
    138e:	60f8      	str	r0, [r7, #12]
    1390:	607a      	str	r2, [r7, #4]
    1392:	603b      	str	r3, [r7, #0]
    1394:	460b      	mov	r3, r1
    1396:	72fb      	strb	r3, [r7, #11]
           (ulPinType == GPIO_PIN_TYPE_ANALOG));

    //
    // Set the output drive strength.
    //
    HWREG(ulPort + GPIO_O_DR2R) = ((ulStrength & 1) ?
    1398:	68fb      	ldr	r3, [r7, #12]
    139a:	f503 63a0 	add.w	r3, r3, #1280	; 0x500
    139e:	461a      	mov	r2, r3
    13a0:	687b      	ldr	r3, [r7, #4]
    13a2:	f003 0301 	and.w	r3, r3, #1
                                   (HWREG(ulPort + GPIO_O_DR2R) | ucPins) :
    13a6:	2b00      	cmp	r3, #0
    13a8:	d006      	beq.n	13b8 <GPIOPadConfigSet+0x30>
    13aa:	68fb      	ldr	r3, [r7, #12]
    13ac:	f503 63a0 	add.w	r3, r3, #1280	; 0x500
    13b0:	6819      	ldr	r1, [r3, #0]
    13b2:	7afb      	ldrb	r3, [r7, #11]
    13b4:	430b      	orrs	r3, r1
    13b6:	e006      	b.n	13c6 <GPIOPadConfigSet+0x3e>
                                   (HWREG(ulPort + GPIO_O_DR2R) & ~(ucPins)));
    13b8:	68fb      	ldr	r3, [r7, #12]
    13ba:	f503 63a0 	add.w	r3, r3, #1280	; 0x500
    13be:	6819      	ldr	r1, [r3, #0]
    13c0:	7afb      	ldrb	r3, [r7, #11]
    13c2:	43db      	mvns	r3, r3

    //
    // Set the output drive strength.
    //
    HWREG(ulPort + GPIO_O_DR2R) = ((ulStrength & 1) ?
                                   (HWREG(ulPort + GPIO_O_DR2R) | ucPins) :
    13c4:	400b      	ands	r3, r1
           (ulPinType == GPIO_PIN_TYPE_ANALOG));

    //
    // Set the output drive strength.
    //
    HWREG(ulPort + GPIO_O_DR2R) = ((ulStrength & 1) ?
    13c6:	6013      	str	r3, [r2, #0]
                                   (HWREG(ulPort + GPIO_O_DR2R) | ucPins) :
                                   (HWREG(ulPort + GPIO_O_DR2R) & ~(ucPins)));
    HWREG(ulPort + GPIO_O_DR4R) = ((ulStrength & 2) ?
    13c8:	68fb      	ldr	r3, [r7, #12]
    13ca:	f203 5304 	addw	r3, r3, #1284	; 0x504
    13ce:	461a      	mov	r2, r3
    13d0:	687b      	ldr	r3, [r7, #4]
    13d2:	f003 0302 	and.w	r3, r3, #2
                                   (HWREG(ulPort + GPIO_O_DR4R) | ucPins) :
    13d6:	2b00      	cmp	r3, #0
    13d8:	d006      	beq.n	13e8 <GPIOPadConfigSet+0x60>
    13da:	68fb      	ldr	r3, [r7, #12]
    13dc:	f203 5304 	addw	r3, r3, #1284	; 0x504
    13e0:	6819      	ldr	r1, [r3, #0]
    13e2:	7afb      	ldrb	r3, [r7, #11]
    13e4:	430b      	orrs	r3, r1
    13e6:	e006      	b.n	13f6 <GPIOPadConfigSet+0x6e>
                                   (HWREG(ulPort + GPIO_O_DR4R) & ~(ucPins)));
    13e8:	68fb      	ldr	r3, [r7, #12]
    13ea:	f203 5304 	addw	r3, r3, #1284	; 0x504
    13ee:	6819      	ldr	r1, [r3, #0]
    13f0:	7afb      	ldrb	r3, [r7, #11]
    13f2:	43db      	mvns	r3, r3
    //
    HWREG(ulPort + GPIO_O_DR2R) = ((ulStrength & 1) ?
                                   (HWREG(ulPort + GPIO_O_DR2R) | ucPins) :
                                   (HWREG(ulPort + GPIO_O_DR2R) & ~(ucPins)));
    HWREG(ulPort + GPIO_O_DR4R) = ((ulStrength & 2) ?
                                   (HWREG(ulPort + GPIO_O_DR4R) | ucPins) :
    13f4:	400b      	ands	r3, r1
    // Set the output drive strength.
    //
    HWREG(ulPort + GPIO_O_DR2R) = ((ulStrength & 1) ?
                                   (HWREG(ulPort + GPIO_O_DR2R) | ucPins) :
                                   (HWREG(ulPort + GPIO_O_DR2R) & ~(ucPins)));
    HWREG(ulPort + GPIO_O_DR4R) = ((ulStrength & 2) ?
    13f6:	6013      	str	r3, [r2, #0]
                                   (HWREG(ulPort + GPIO_O_DR4R) | ucPins) :
                                   (HWREG(ulPort + GPIO_O_DR4R) & ~(ucPins)));
    HWREG(ulPort + GPIO_O_DR8R) = ((ulStrength & 4) ?
    13f8:	68fb      	ldr	r3, [r7, #12]
    13fa:	f503 63a1 	add.w	r3, r3, #1288	; 0x508
    13fe:	461a      	mov	r2, r3
    1400:	687b      	ldr	r3, [r7, #4]
    1402:	f003 0304 	and.w	r3, r3, #4
                                   (HWREG(ulPort + GPIO_O_DR8R) | ucPins) :
    1406:	2b00      	cmp	r3, #0
    1408:	d006      	beq.n	1418 <GPIOPadConfigSet+0x90>
    140a:	68fb      	ldr	r3, [r7, #12]
    140c:	f503 63a1 	add.w	r3, r3, #1288	; 0x508
    1410:	6819      	ldr	r1, [r3, #0]
    1412:	7afb      	ldrb	r3, [r7, #11]
    1414:	430b      	orrs	r3, r1
    1416:	e006      	b.n	1426 <GPIOPadConfigSet+0x9e>
                                   (HWREG(ulPort + GPIO_O_DR8R) & ~(ucPins)));
    1418:	68fb      	ldr	r3, [r7, #12]
    141a:	f503 63a1 	add.w	r3, r3, #1288	; 0x508
    141e:	6819      	ldr	r1, [r3, #0]
    1420:	7afb      	ldrb	r3, [r7, #11]
    1422:	43db      	mvns	r3, r3
                                   (HWREG(ulPort + GPIO_O_DR2R) & ~(ucPins)));
    HWREG(ulPort + GPIO_O_DR4R) = ((ulStrength & 2) ?
                                   (HWREG(ulPort + GPIO_O_DR4R) | ucPins) :
                                   (HWREG(ulPort + GPIO_O_DR4R) & ~(ucPins)));
    HWREG(ulPort + GPIO_O_DR8R) = ((ulStrength & 4) ?
                                   (HWREG(ulPort + GPIO_O_DR8R) | ucPins) :
    1424:	400b      	ands	r3, r1
                                   (HWREG(ulPort + GPIO_O_DR2R) | ucPins) :
                                   (HWREG(ulPort + GPIO_O_DR2R) & ~(ucPins)));
    HWREG(ulPort + GPIO_O_DR4R) = ((ulStrength & 2) ?
                                   (HWREG(ulPort + GPIO_O_DR4R) | ucPins) :
                                   (HWREG(ulPort + GPIO_O_DR4R) & ~(ucPins)));
    HWREG(ulPort + GPIO_O_DR8R) = ((ulStrength & 4) ?
    1426:	6013      	str	r3, [r2, #0]
                                   (HWREG(ulPort + GPIO_O_DR8R) | ucPins) :
                                   (HWREG(ulPort + GPIO_O_DR8R) & ~(ucPins)));
    HWREG(ulPort + GPIO_O_SLR) = ((ulStrength & 8) ?
    1428:	68fb      	ldr	r3, [r7, #12]
    142a:	f503 63a3 	add.w	r3, r3, #1304	; 0x518
    142e:	461a      	mov	r2, r3
    1430:	687b      	ldr	r3, [r7, #4]
    1432:	f003 0308 	and.w	r3, r3, #8
                                  (HWREG(ulPort + GPIO_O_SLR) | ucPins) :
    1436:	2b00      	cmp	r3, #0
    1438:	d006      	beq.n	1448 <GPIOPadConfigSet+0xc0>
    143a:	68fb      	ldr	r3, [r7, #12]
    143c:	f503 63a3 	add.w	r3, r3, #1304	; 0x518
    1440:	6819      	ldr	r1, [r3, #0]
    1442:	7afb      	ldrb	r3, [r7, #11]
    1444:	430b      	orrs	r3, r1
    1446:	e006      	b.n	1456 <GPIOPadConfigSet+0xce>
                                  (HWREG(ulPort + GPIO_O_SLR) & ~(ucPins)));
    1448:	68fb      	ldr	r3, [r7, #12]
    144a:	f503 63a3 	add.w	r3, r3, #1304	; 0x518
    144e:	6819      	ldr	r1, [r3, #0]
    1450:	7afb      	ldrb	r3, [r7, #11]
    1452:	43db      	mvns	r3, r3
                                   (HWREG(ulPort + GPIO_O_DR4R) & ~(ucPins)));
    HWREG(ulPort + GPIO_O_DR8R) = ((ulStrength & 4) ?
                                   (HWREG(ulPort + GPIO_O_DR8R) | ucPins) :
                                   (HWREG(ulPort + GPIO_O_DR8R) & ~(ucPins)));
    HWREG(ulPort + GPIO_O_SLR) = ((ulStrength & 8) ?
                                  (HWREG(ulPort + GPIO_O_SLR) | ucPins) :
    1454:	400b      	ands	r3, r1
                                   (HWREG(ulPort + GPIO_O_DR4R) | ucPins) :
                                   (HWREG(ulPort + GPIO_O_DR4R) & ~(ucPins)));
    HWREG(ulPort + GPIO_O_DR8R) = ((ulStrength & 4) ?
                                   (HWREG(ulPort + GPIO_O_DR8R) | ucPins) :
                                   (HWREG(ulPort + GPIO_O_DR8R) & ~(ucPins)));
    HWREG(ulPort + GPIO_O_SLR) = ((ulStrength & 8) ?
    1456:	6013      	str	r3, [r2, #0]
                                  (HWREG(ulPort + GPIO_O_SLR) & ~(ucPins)));

    //
    // Set the pin type.
    //
    HWREG(ulPort + GPIO_O_ODR) = ((ulPinType & 1) ?
    1458:	68fb      	ldr	r3, [r7, #12]
    145a:	f203 530c 	addw	r3, r3, #1292	; 0x50c
    145e:	461a      	mov	r2, r3
    1460:	683b      	ldr	r3, [r7, #0]
    1462:	f003 0301 	and.w	r3, r3, #1
                                  (HWREG(ulPort + GPIO_O_ODR) | ucPins) :
    1466:	2b00      	cmp	r3, #0
    1468:	d006      	beq.n	1478 <GPIOPadConfigSet+0xf0>
    146a:	68fb      	ldr	r3, [r7, #12]
    146c:	f203 530c 	addw	r3, r3, #1292	; 0x50c
    1470:	6819      	ldr	r1, [r3, #0]
    1472:	7afb      	ldrb	r3, [r7, #11]
    1474:	430b      	orrs	r3, r1
    1476:	e006      	b.n	1486 <GPIOPadConfigSet+0xfe>
                                  (HWREG(ulPort + GPIO_O_ODR) & ~(ucPins)));
    1478:	68fb      	ldr	r3, [r7, #12]
    147a:	f203 530c 	addw	r3, r3, #1292	; 0x50c
    147e:	6819      	ldr	r1, [r3, #0]
    1480:	7afb      	ldrb	r3, [r7, #11]
    1482:	43db      	mvns	r3, r3

    //
    // Set the pin type.
    //
    HWREG(ulPort + GPIO_O_ODR) = ((ulPinType & 1) ?
                                  (HWREG(ulPort + GPIO_O_ODR) | ucPins) :
    1484:	400b      	ands	r3, r1
                                  (HWREG(ulPort + GPIO_O_SLR) & ~(ucPins)));

    //
    // Set the pin type.
    //
    HWREG(ulPort + GPIO_O_ODR) = ((ulPinType & 1) ?
    1486:	6013      	str	r3, [r2, #0]
                                  (HWREG(ulPort + GPIO_O_ODR) | ucPins) :
                                  (HWREG(ulPort + GPIO_O_ODR) & ~(ucPins)));
    HWREG(ulPort + GPIO_O_PUR) = ((ulPinType & 2) ?
    1488:	68fb      	ldr	r3, [r7, #12]
    148a:	f503 63a2 	add.w	r3, r3, #1296	; 0x510
    148e:	461a      	mov	r2, r3
    1490:	683b      	ldr	r3, [r7, #0]
    1492:	f003 0302 	and.w	r3, r3, #2
                                  (HWREG(ulPort + GPIO_O_PUR) | ucPins) :
    1496:	2b00      	cmp	r3, #0
    1498:	d006      	beq.n	14a8 <GPIOPadConfigSet+0x120>
    149a:	68fb      	ldr	r3, [r7, #12]
    149c:	f503 63a2 	add.w	r3, r3, #1296	; 0x510
    14a0:	6819      	ldr	r1, [r3, #0]
    14a2:	7afb      	ldrb	r3, [r7, #11]
    14a4:	430b      	orrs	r3, r1
    14a6:	e006      	b.n	14b6 <GPIOPadConfigSet+0x12e>
                                  (HWREG(ulPort + GPIO_O_PUR) & ~(ucPins)));
    14a8:	68fb      	ldr	r3, [r7, #12]
    14aa:	f503 63a2 	add.w	r3, r3, #1296	; 0x510
    14ae:	6819      	ldr	r1, [r3, #0]
    14b0:	7afb      	ldrb	r3, [r7, #11]
    14b2:	43db      	mvns	r3, r3
    //
    HWREG(ulPort + GPIO_O_ODR) = ((ulPinType & 1) ?
                                  (HWREG(ulPort + GPIO_O_ODR) | ucPins) :
                                  (HWREG(ulPort + GPIO_O_ODR) & ~(ucPins)));
    HWREG(ulPort + GPIO_O_PUR) = ((ulPinType & 2) ?
                                  (HWREG(ulPort + GPIO_O_PUR) | ucPins) :
    14b4:	400b      	ands	r3, r1
    // Set the pin type.
    //
    HWREG(ulPort + GPIO_O_ODR) = ((ulPinType & 1) ?
                                  (HWREG(ulPort + GPIO_O_ODR) | ucPins) :
                                  (HWREG(ulPort + GPIO_O_ODR) & ~(ucPins)));
    HWREG(ulPort + GPIO_O_PUR) = ((ulPinType & 2) ?
    14b6:	6013      	str	r3, [r2, #0]
                                  (HWREG(ulPort + GPIO_O_PUR) | ucPins) :
                                  (HWREG(ulPort + GPIO_O_PUR) & ~(ucPins)));
    HWREG(ulPort + GPIO_O_PDR) = ((ulPinType & 4) ?
    14b8:	68fb      	ldr	r3, [r7, #12]
    14ba:	f203 5314 	addw	r3, r3, #1300	; 0x514
    14be:	461a      	mov	r2, r3
    14c0:	683b      	ldr	r3, [r7, #0]
    14c2:	f003 0304 	and.w	r3, r3, #4
                                  (HWREG(ulPort + GPIO_O_PDR) | ucPins) :
    14c6:	2b00      	cmp	r3, #0
    14c8:	d006      	beq.n	14d8 <GPIOPadConfigSet+0x150>
    14ca:	68fb      	ldr	r3, [r7, #12]
    14cc:	f203 5314 	addw	r3, r3, #1300	; 0x514
    14d0:	6819      	ldr	r1, [r3, #0]
    14d2:	7afb      	ldrb	r3, [r7, #11]
    14d4:	430b      	orrs	r3, r1
    14d6:	e006      	b.n	14e6 <GPIOPadConfigSet+0x15e>
                                  (HWREG(ulPort + GPIO_O_PDR) & ~(ucPins)));
    14d8:	68fb      	ldr	r3, [r7, #12]
    14da:	f203 5314 	addw	r3, r3, #1300	; 0x514
    14de:	6819      	ldr	r1, [r3, #0]
    14e0:	7afb      	ldrb	r3, [r7, #11]
    14e2:	43db      	mvns	r3, r3
                                  (HWREG(ulPort + GPIO_O_ODR) & ~(ucPins)));
    HWREG(ulPort + GPIO_O_PUR) = ((ulPinType & 2) ?
                                  (HWREG(ulPort + GPIO_O_PUR) | ucPins) :
                                  (HWREG(ulPort + GPIO_O_PUR) & ~(ucPins)));
    HWREG(ulPort + GPIO_O_PDR) = ((ulPinType & 4) ?
                                  (HWREG(ulPort + GPIO_O_PDR) | ucPins) :
    14e4:	400b      	ands	r3, r1
                                  (HWREG(ulPort + GPIO_O_ODR) | ucPins) :
                                  (HWREG(ulPort + GPIO_O_ODR) & ~(ucPins)));
    HWREG(ulPort + GPIO_O_PUR) = ((ulPinType & 2) ?
                                  (HWREG(ulPort + GPIO_O_PUR) | ucPins) :
                                  (HWREG(ulPort + GPIO_O_PUR) & ~(ucPins)));
    HWREG(ulPort + GPIO_O_PDR) = ((ulPinType & 4) ?
    14e6:	6013      	str	r3, [r2, #0]
                                  (HWREG(ulPort + GPIO_O_PDR) | ucPins) :
                                  (HWREG(ulPort + GPIO_O_PDR) & ~(ucPins)));
    HWREG(ulPort + GPIO_O_DEN) = ((ulPinType & 8) ?
    14e8:	68fb      	ldr	r3, [r7, #12]
    14ea:	f203 531c 	addw	r3, r3, #1308	; 0x51c
    14ee:	461a      	mov	r2, r3
    14f0:	683b      	ldr	r3, [r7, #0]
    14f2:	f003 0308 	and.w	r3, r3, #8
                                  (HWREG(ulPort + GPIO_O_DEN) | ucPins) :
    14f6:	2b00      	cmp	r3, #0
    14f8:	d006      	beq.n	1508 <GPIOPadConfigSet+0x180>
    14fa:	68fb      	ldr	r3, [r7, #12]
    14fc:	f203 531c 	addw	r3, r3, #1308	; 0x51c
    1500:	6819      	ldr	r1, [r3, #0]
    1502:	7afb      	ldrb	r3, [r7, #11]
    1504:	430b      	orrs	r3, r1
    1506:	e006      	b.n	1516 <GPIOPadConfigSet+0x18e>
                                  (HWREG(ulPort + GPIO_O_DEN) & ~(ucPins)));
    1508:	68fb      	ldr	r3, [r7, #12]
    150a:	f203 531c 	addw	r3, r3, #1308	; 0x51c
    150e:	6819      	ldr	r1, [r3, #0]
    1510:	7afb      	ldrb	r3, [r7, #11]
    1512:	43db      	mvns	r3, r3
                                  (HWREG(ulPort + GPIO_O_PUR) & ~(ucPins)));
    HWREG(ulPort + GPIO_O_PDR) = ((ulPinType & 4) ?
                                  (HWREG(ulPort + GPIO_O_PDR) | ucPins) :
                                  (HWREG(ulPort + GPIO_O_PDR) & ~(ucPins)));
    HWREG(ulPort + GPIO_O_DEN) = ((ulPinType & 8) ?
                                  (HWREG(ulPort + GPIO_O_DEN) | ucPins) :
    1514:	400b      	ands	r3, r1
                                  (HWREG(ulPort + GPIO_O_PUR) | ucPins) :
                                  (HWREG(ulPort + GPIO_O_PUR) & ~(ucPins)));
    HWREG(ulPort + GPIO_O_PDR) = ((ulPinType & 4) ?
                                  (HWREG(ulPort + GPIO_O_PDR) | ucPins) :
                                  (HWREG(ulPort + GPIO_O_PDR) & ~(ucPins)));
    HWREG(ulPort + GPIO_O_DEN) = ((ulPinType & 8) ?
    1516:	6013      	str	r3, [r2, #0]
    //
    // Set the analog mode select register.  This register only appears in
    // DustDevil-class (and later) devices, but is a harmless write on
    // Sandstorm- and Fury-class devices.
    //
    HWREG(ulPort + GPIO_O_AMSEL) =
    1518:	68fb      	ldr	r3, [r7, #12]
    151a:	f503 63a5 	add.w	r3, r3, #1320	; 0x528
    151e:	461a      	mov	r2, r3
        ((ulPinType == GPIO_PIN_TYPE_ANALOG) ?
         (HWREG(ulPort + GPIO_O_AMSEL) | ucPins) :
    1520:	683b      	ldr	r3, [r7, #0]
    1522:	2b00      	cmp	r3, #0
    1524:	d106      	bne.n	1534 <GPIOPadConfigSet+0x1ac>
    1526:	68fb      	ldr	r3, [r7, #12]
    1528:	f503 63a5 	add.w	r3, r3, #1320	; 0x528
    152c:	6819      	ldr	r1, [r3, #0]
    152e:	7afb      	ldrb	r3, [r7, #11]
    1530:	430b      	orrs	r3, r1
    1532:	e006      	b.n	1542 <GPIOPadConfigSet+0x1ba>
         (HWREG(ulPort + GPIO_O_AMSEL) & ~(ucPins)));
    1534:	68fb      	ldr	r3, [r7, #12]
    1536:	f503 63a5 	add.w	r3, r3, #1320	; 0x528
    153a:	6819      	ldr	r1, [r3, #0]
    153c:	7afb      	ldrb	r3, [r7, #11]
    153e:	43db      	mvns	r3, r3
    // DustDevil-class (and later) devices, but is a harmless write on
    // Sandstorm- and Fury-class devices.
    //
    HWREG(ulPort + GPIO_O_AMSEL) =
        ((ulPinType == GPIO_PIN_TYPE_ANALOG) ?
         (HWREG(ulPort + GPIO_O_AMSEL) | ucPins) :
    1540:	400b      	ands	r3, r1
    //
    // Set the analog mode select register.  This register only appears in
    // DustDevil-class (and later) devices, but is a harmless write on
    // Sandstorm- and Fury-class devices.
    //
    HWREG(ulPort + GPIO_O_AMSEL) =
    1542:	6013      	str	r3, [r2, #0]
        ((ulPinType == GPIO_PIN_TYPE_ANALOG) ?
         (HWREG(ulPort + GPIO_O_AMSEL) | ucPins) :
         (HWREG(ulPort + GPIO_O_AMSEL) & ~(ucPins)));
}
    1544:	f107 0714 	add.w	r7, r7, #20
    1548:	46bd      	mov	sp, r7
    154a:	bc80      	pop	{r7}
    154c:	4770      	bx	lr
    154e:	bf00      	nop

00001550 <GPIOPinTypeTimer>:
//! \return None.
//
//*****************************************************************************
void
GPIOPinTypeTimer(unsigned long ulPort, unsigned char ucPins)
{
    1550:	b580      	push	{r7, lr}
    1552:	b082      	sub	sp, #8
    1554:	af00      	add	r7, sp, #0
    1556:	6078      	str	r0, [r7, #4]
    1558:	460b      	mov	r3, r1
    155a:	70fb      	strb	r3, [r7, #3]
    ASSERT(GPIOBaseValid(ulPort));

    //
    // Make the pin(s) be peripheral controlled.
    //
    GPIODirModeSet(ulPort, ucPins, GPIO_DIR_MODE_HW);
    155c:	78fb      	ldrb	r3, [r7, #3]
    155e:	6878      	ldr	r0, [r7, #4]
    1560:	4619      	mov	r1, r3
    1562:	2202      	movs	r2, #2
    1564:	f7ff fed4 	bl	1310 <GPIODirModeSet>

    //
    // Set the pad(s) for standard push-pull operation.
    //
    GPIOPadConfigSet(ulPort, ucPins, GPIO_STRENGTH_2MA, GPIO_PIN_TYPE_STD);
    1568:	78fb      	ldrb	r3, [r7, #3]
    156a:	6878      	ldr	r0, [r7, #4]
    156c:	4619      	mov	r1, r3
    156e:	2201      	movs	r2, #1
    1570:	2308      	movs	r3, #8
    1572:	f7ff ff09 	bl	1388 <GPIOPadConfigSet>
}
    1576:	f107 0708 	add.w	r7, r7, #8
    157a:	46bd      	mov	sp, r7
    157c:	bd80      	pop	{r7, pc}
    157e:	bf00      	nop

00001580 <GPIOPinTypeUART>:
//! \return None.
//
//*****************************************************************************
void
GPIOPinTypeUART(unsigned long ulPort, unsigned char ucPins)
{
    1580:	b580      	push	{r7, lr}
    1582:	b082      	sub	sp, #8
    1584:	af00      	add	r7, sp, #0
    1586:	6078      	str	r0, [r7, #4]
    1588:	460b      	mov	r3, r1
    158a:	70fb      	strb	r3, [r7, #3]
    ASSERT(GPIOBaseValid(ulPort));

    //
    // Make the pin(s) be peripheral controlled.
    //
    GPIODirModeSet(ulPort, ucPins, GPIO_DIR_MODE_HW);
    158c:	78fb      	ldrb	r3, [r7, #3]
    158e:	6878      	ldr	r0, [r7, #4]
    1590:	4619      	mov	r1, r3
    1592:	2202      	movs	r2, #2
    1594:	f7ff febc 	bl	1310 <GPIODirModeSet>

    //
    // Set the pad(s) for standard push-pull operation.
    //
    GPIOPadConfigSet(ulPort, ucPins, GPIO_STRENGTH_2MA, GPIO_PIN_TYPE_STD);
    1598:	78fb      	ldrb	r3, [r7, #3]
    159a:	6878      	ldr	r0, [r7, #4]
    159c:	4619      	mov	r1, r3
    159e:	2201      	movs	r2, #1
    15a0:	2308      	movs	r3, #8
    15a2:	f7ff fef1 	bl	1388 <GPIOPadConfigSet>
}
    15a6:	f107 0708 	add.w	r7, r7, #8
    15aa:	46bd      	mov	sp, r7
    15ac:	bd80      	pop	{r7, pc}
    15ae:	bf00      	nop

000015b0 <GPIOPinConfigure>:
//! \return None.
//
//*****************************************************************************
void
GPIOPinConfigure(unsigned long ulPinConfig)
{
    15b0:	b480      	push	{r7}
    15b2:	b085      	sub	sp, #20
    15b4:	af00      	add	r7, sp, #0
    15b6:	6078      	str	r0, [r7, #4]
    ASSERT(((ulPinConfig >> 8) & 0xe3) == 0);

    //
    // Extract the base address index from the input value.
    //
    ulBase = (ulPinConfig >> 16) & 0xff;
    15b8:	687b      	ldr	r3, [r7, #4]
    15ba:	0c1b      	lsrs	r3, r3, #16
    15bc:	b2db      	uxtb	r3, r3
    15be:	60fb      	str	r3, [r7, #12]

    //
    // Get the base address of the GPIO module, selecting either the APB or the
    // AHB aperture as appropriate.
    //
    if(HWREG(SYSCTL_GPIOHBCTL) & (1 << ulBase))
    15c0:	f24e 036c 	movw	r3, #57452	; 0xe06c
    15c4:	f2c4 030f 	movt	r3, #16399	; 0x400f
    15c8:	681a      	ldr	r2, [r3, #0]
    15ca:	68fb      	ldr	r3, [r7, #12]
    15cc:	2101      	movs	r1, #1
    15ce:	fa01 f303 	lsl.w	r3, r1, r3
    15d2:	4013      	ands	r3, r2
    15d4:	2b00      	cmp	r3, #0
    15d6:	d00a      	beq.n	15ee <GPIOPinConfigure+0x3e>
    {
        ulBase = g_pulGPIOBaseAddrs[(ulBase << 1) + 1];
    15d8:	68fb      	ldr	r3, [r7, #12]
    15da:	005b      	lsls	r3, r3, #1
    15dc:	1c5a      	adds	r2, r3, #1
    15de:	f242 13ac 	movw	r3, #8620	; 0x21ac
    15e2:	f2c0 0300 	movt	r3, #0
    15e6:	f853 3022 	ldr.w	r3, [r3, r2, lsl #2]
    15ea:	60fb      	str	r3, [r7, #12]
    15ec:	e008      	b.n	1600 <GPIOPinConfigure+0x50>
    }
    else
    {
        ulBase = g_pulGPIOBaseAddrs[ulBase << 1];
    15ee:	68fb      	ldr	r3, [r7, #12]
    15f0:	005a      	lsls	r2, r3, #1
    15f2:	f242 13ac 	movw	r3, #8620	; 0x21ac
    15f6:	f2c0 0300 	movt	r3, #0
    15fa:	f853 3022 	ldr.w	r3, [r3, r2, lsl #2]
    15fe:	60fb      	str	r3, [r7, #12]
    }

    //
    // Extract the shift from the input value.
    //
    ulShift = (ulPinConfig >> 8) & 0xff;
    1600:	687b      	ldr	r3, [r7, #4]
    1602:	0a1b      	lsrs	r3, r3, #8
    1604:	b2db      	uxtb	r3, r3
    1606:	60bb      	str	r3, [r7, #8]

    //
    // Write the requested pin muxing value for this GPIO pin.
    //
    HWREG(ulBase + GPIO_O_PCTL) = ((HWREG(ulBase + GPIO_O_PCTL) &
    1608:	68fb      	ldr	r3, [r7, #12]
    160a:	f203 532c 	addw	r3, r3, #1324	; 0x52c
    160e:	68fa      	ldr	r2, [r7, #12]
    1610:	f202 522c 	addw	r2, r2, #1324	; 0x52c
    1614:	6811      	ldr	r1, [r2, #0]
                                    ~(0xf << ulShift)) |
    1616:	68ba      	ldr	r2, [r7, #8]
    1618:	200f      	movs	r0, #15
    161a:	fa00 f202 	lsl.w	r2, r0, r2
    161e:	43d2      	mvns	r2, r2
    ulShift = (ulPinConfig >> 8) & 0xff;

    //
    // Write the requested pin muxing value for this GPIO pin.
    //
    HWREG(ulBase + GPIO_O_PCTL) = ((HWREG(ulBase + GPIO_O_PCTL) &
    1620:	4011      	ands	r1, r2
                                    ~(0xf << ulShift)) |
                                   ((ulPinConfig & 0xf) << ulShift));
    1622:	687a      	ldr	r2, [r7, #4]
    1624:	f002 000f 	and.w	r0, r2, #15
    1628:	68ba      	ldr	r2, [r7, #8]
    162a:	fa00 f202 	lsl.w	r2, r0, r2

    //
    // Write the requested pin muxing value for this GPIO pin.
    //
    HWREG(ulBase + GPIO_O_PCTL) = ((HWREG(ulBase + GPIO_O_PCTL) &
                                    ~(0xf << ulShift)) |
    162e:	430a      	orrs	r2, r1
    ulShift = (ulPinConfig >> 8) & 0xff;

    //
    // Write the requested pin muxing value for this GPIO pin.
    //
    HWREG(ulBase + GPIO_O_PCTL) = ((HWREG(ulBase + GPIO_O_PCTL) &
    1630:	601a      	str	r2, [r3, #0]
                                    ~(0xf << ulShift)) |
                                   ((ulPinConfig & 0xf) << ulShift));
}
    1632:	f107 0714 	add.w	r7, r7, #20
    1636:	46bd      	mov	sp, r7
    1638:	bc80      	pop	{r7}
    163a:	4770      	bx	lr

0000163c <IntMasterEnable>:
//! called or \b false if they were initially enabled.
//
//*****************************************************************************
tBoolean
IntMasterEnable(void)
{
    163c:	b580      	push	{r7, lr}
    163e:	af00      	add	r7, sp, #0
    //
    // Enable processor interrupts.
    //
    return(CPUcpsie());
    1640:	f000 fd9a 	bl	2178 <CPUcpsie>
    1644:	4603      	mov	r3, r0
    1646:	b2db      	uxtb	r3, r3
}
    1648:	4618      	mov	r0, r3
    164a:	bd80      	pop	{r7, pc}

0000164c <IntRegister>:
//! \return None.
//
//*****************************************************************************
void
IntRegister(unsigned long ulInterrupt, void (*pfnHandler)(void))
{
    164c:	b480      	push	{r7}
    164e:	b085      	sub	sp, #20
    1650:	af00      	add	r7, sp, #0
    1652:	6078      	str	r0, [r7, #4]
    1654:	6039      	str	r1, [r7, #0]
    ASSERT(((unsigned long)g_pfnRAMVectors & 0x000003ff) == 0);

    //
    // See if the RAM vector table has been initialized.
    //
    if(HWREG(NVIC_VTABLE) != (unsigned long)g_pfnRAMVectors)
    1656:	f64e 5308 	movw	r3, #60680	; 0xed08
    165a:	f2ce 0300 	movt	r3, #57344	; 0xe000
    165e:	681a      	ldr	r2, [r3, #0]
    1660:	f240 4300 	movw	r3, #1024	; 0x400
    1664:	f2c2 0300 	movt	r3, #8192	; 0x2000
    1668:	429a      	cmp	r2, r3
    166a:	d024      	beq.n	16b6 <IntRegister+0x6a>
    {
        //
        // Copy the vector table from the beginning of FLASH to the RAM vector
        // table.
        //
        ulValue = HWREG(NVIC_VTABLE);
    166c:	f64e 5308 	movw	r3, #60680	; 0xed08
    1670:	f2ce 0300 	movt	r3, #57344	; 0xe000
    1674:	681b      	ldr	r3, [r3, #0]
    1676:	60bb      	str	r3, [r7, #8]
        for(ulIdx = 0; ulIdx < NUM_INTERRUPTS; ulIdx++)
    1678:	2300      	movs	r3, #0
    167a:	60fb      	str	r3, [r7, #12]
    167c:	e00f      	b.n	169e <IntRegister+0x52>
        {
            g_pfnRAMVectors[ulIdx] = (void (*)(void))HWREG((ulIdx * 4) +
    167e:	68fb      	ldr	r3, [r7, #12]
    1680:	009a      	lsls	r2, r3, #2
    1682:	68bb      	ldr	r3, [r7, #8]
    1684:	18d3      	adds	r3, r2, r3
    1686:	681b      	ldr	r3, [r3, #0]
    1688:	4619      	mov	r1, r3
    168a:	f240 4300 	movw	r3, #1024	; 0x400
    168e:	f2c2 0300 	movt	r3, #8192	; 0x2000
    1692:	68fa      	ldr	r2, [r7, #12]
    1694:	f843 1022 	str.w	r1, [r3, r2, lsl #2]
        //
        // Copy the vector table from the beginning of FLASH to the RAM vector
        // table.
        //
        ulValue = HWREG(NVIC_VTABLE);
        for(ulIdx = 0; ulIdx < NUM_INTERRUPTS; ulIdx++)
    1698:	68fb      	ldr	r3, [r7, #12]
    169a:	3301      	adds	r3, #1
    169c:	60fb      	str	r3, [r7, #12]
    169e:	68fb      	ldr	r3, [r7, #12]
    16a0:	2b9a      	cmp	r3, #154	; 0x9a
    16a2:	d9ec      	bls.n	167e <IntRegister+0x32>
        }

        //
        // Point the NVIC at the RAM vector table.
        //
        HWREG(NVIC_VTABLE) = (unsigned long)g_pfnRAMVectors;
    16a4:	f64e 5308 	movw	r3, #60680	; 0xed08
    16a8:	f2ce 0300 	movt	r3, #57344	; 0xe000
    16ac:	f240 4200 	movw	r2, #1024	; 0x400
    16b0:	f2c2 0200 	movt	r2, #8192	; 0x2000
    16b4:	601a      	str	r2, [r3, #0]
    }

    //
    // Save the interrupt handler.
    //
    g_pfnRAMVectors[ulInterrupt] = pfnHandler;
    16b6:	f240 4300 	movw	r3, #1024	; 0x400
    16ba:	f2c2 0300 	movt	r3, #8192	; 0x2000
    16be:	687a      	ldr	r2, [r7, #4]
    16c0:	6839      	ldr	r1, [r7, #0]
    16c2:	f843 1022 	str.w	r1, [r3, r2, lsl #2]
}
    16c6:	f107 0714 	add.w	r7, r7, #20
    16ca:	46bd      	mov	sp, r7
    16cc:	bc80      	pop	{r7}
    16ce:	4770      	bx	lr

000016d0 <IntEnable>:
//! \return None.
//
//*****************************************************************************
void
IntEnable(unsigned long ulInterrupt)
{
    16d0:	b480      	push	{r7}
    16d2:	b083      	sub	sp, #12
    16d4:	af00      	add	r7, sp, #0
    16d6:	6078      	str	r0, [r7, #4]
    ASSERT(ulInterrupt < NUM_INTERRUPTS);

    //
    // Determine the interrupt to enable.
    //
    if(ulInterrupt == FAULT_MPU)
    16d8:	687b      	ldr	r3, [r7, #4]
    16da:	2b04      	cmp	r3, #4
    16dc:	d10c      	bne.n	16f8 <IntEnable+0x28>
    {
        //
        // Enable the MemManage interrupt.
        //
        HWREG(NVIC_SYS_HND_CTRL) |= NVIC_SYS_HND_CTRL_MEM;
    16de:	f64e 5324 	movw	r3, #60708	; 0xed24
    16e2:	f2ce 0300 	movt	r3, #57344	; 0xe000
    16e6:	f64e 5224 	movw	r2, #60708	; 0xed24
    16ea:	f2ce 0200 	movt	r2, #57344	; 0xe000
    16ee:	6812      	ldr	r2, [r2, #0]
    16f0:	f442 3280 	orr.w	r2, r2, #65536	; 0x10000
    16f4:	601a      	str	r2, [r3, #0]
    16f6:	e043      	b.n	1780 <IntEnable+0xb0>
    }
    else if(ulInterrupt == FAULT_BUS)
    16f8:	687b      	ldr	r3, [r7, #4]
    16fa:	2b05      	cmp	r3, #5
    16fc:	d10c      	bne.n	1718 <IntEnable+0x48>
    {
        //
        // Enable the bus fault interrupt.
        //
        HWREG(NVIC_SYS_HND_CTRL) |= NVIC_SYS_HND_CTRL_BUS;
    16fe:	f64e 5324 	movw	r3, #60708	; 0xed24
    1702:	f2ce 0300 	movt	r3, #57344	; 0xe000
    1706:	f64e 5224 	movw	r2, #60708	; 0xed24
    170a:	f2ce 0200 	movt	r2, #57344	; 0xe000
    170e:	6812      	ldr	r2, [r2, #0]
    1710:	f442 3200 	orr.w	r2, r2, #131072	; 0x20000
    1714:	601a      	str	r2, [r3, #0]
    1716:	e033      	b.n	1780 <IntEnable+0xb0>
    }
    else if(ulInterrupt == FAULT_USAGE)
    1718:	687b      	ldr	r3, [r7, #4]
    171a:	2b06      	cmp	r3, #6
    171c:	d10c      	bne.n	1738 <IntEnable+0x68>
    {
        //
        // Enable the usage fault interrupt.
        //
        HWREG(NVIC_SYS_HND_CTRL) |= NVIC_SYS_HND_CTRL_USAGE;
    171e:	f64e 5324 	movw	r3, #60708	; 0xed24
    1722:	f2ce 0300 	movt	r3, #57344	; 0xe000
    1726:	f64e 5224 	movw	r2, #60708	; 0xed24
    172a:	f2ce 0200 	movt	r2, #57344	; 0xe000
    172e:	6812      	ldr	r2, [r2, #0]
    1730:	f442 2280 	orr.w	r2, r2, #262144	; 0x40000
    1734:	601a      	str	r2, [r3, #0]
    1736:	e023      	b.n	1780 <IntEnable+0xb0>
    }
    else if(ulInterrupt == FAULT_SYSTICK)
    1738:	687b      	ldr	r3, [r7, #4]
    173a:	2b0f      	cmp	r3, #15
    173c:	d10c      	bne.n	1758 <IntEnable+0x88>
    {
        //
        // Enable the System Tick interrupt.
        //
        HWREG(NVIC_ST_CTRL) |= NVIC_ST_CTRL_INTEN;
    173e:	f24e 0310 	movw	r3, #57360	; 0xe010
    1742:	f2ce 0300 	movt	r3, #57344	; 0xe000
    1746:	f24e 0210 	movw	r2, #57360	; 0xe010
    174a:	f2ce 0200 	movt	r2, #57344	; 0xe000
    174e:	6812      	ldr	r2, [r2, #0]
    1750:	f042 0202 	orr.w	r2, r2, #2
    1754:	601a      	str	r2, [r3, #0]
    1756:	e013      	b.n	1780 <IntEnable+0xb0>
    }
    else if(ulInterrupt >= 16)
    1758:	687b      	ldr	r3, [r7, #4]
    175a:	2b0f      	cmp	r3, #15
    175c:	d910      	bls.n	1780 <IntEnable+0xb0>
    {
        //
        // Enable the general interrupt.
        //
        HWREG(g_pulEnRegs[(ulInterrupt - 16) / 32]) =
    175e:	687b      	ldr	r3, [r7, #4]
    1760:	3b10      	subs	r3, #16
    1762:	095a      	lsrs	r2, r3, #5
    1764:	f242 2324 	movw	r3, #8740	; 0x2224
    1768:	f2c0 0300 	movt	r3, #0
    176c:	f853 3022 	ldr.w	r3, [r3, r2, lsl #2]
            1 << ((ulInterrupt - 16) & 31);
    1770:	687a      	ldr	r2, [r7, #4]
    1772:	3a10      	subs	r2, #16
    1774:	f002 021f 	and.w	r2, r2, #31
    1778:	2101      	movs	r1, #1
    177a:	fa01 f202 	lsl.w	r2, r1, r2
    else if(ulInterrupt >= 16)
    {
        //
        // Enable the general interrupt.
        //
        HWREG(g_pulEnRegs[(ulInterrupt - 16) / 32]) =
    177e:	601a      	str	r2, [r3, #0]
            1 << ((ulInterrupt - 16) & 31);
    }
}
    1780:	f107 070c 	add.w	r7, r7, #12
    1784:	46bd      	mov	sp, r7
    1786:	bc80      	pop	{r7}
    1788:	4770      	bx	lr
    178a:	bf00      	nop

0000178c <SysCtlPeripheralEnable>:
//! \return None.
//
//*****************************************************************************
void
SysCtlPeripheralEnable(unsigned long ulPeripheral)
{
    178c:	b480      	push	{r7}
    178e:	b083      	sub	sp, #12
    1790:	af00      	add	r7, sp, #0
    1792:	6078      	str	r0, [r7, #4]

    //
    // See if the peripheral index is 15, indicating a peripheral that is
    // accessed via the SYSCTL_RCGCperiph registers.
    //
    if((ulPeripheral & 0xf0000000) == 0xf0000000)
    1794:	687b      	ldr	r3, [r7, #4]
    1796:	f003 4370 	and.w	r3, r3, #4026531840	; 0xf0000000
    179a:	f1b3 4f70 	cmp.w	r3, #4026531840	; 0xf0000000
    179e:	d120      	bne.n	17e2 <SysCtlPeripheralEnable+0x56>
    {
        //
        // Enable this peripheral.
        //
        HWREGBITW(SYSCTL_RCGCBASE + ((ulPeripheral & 0xff00) >> 8),
    17a0:	687b      	ldr	r3, [r7, #4]
    17a2:	f403 437f 	and.w	r3, r3, #65280	; 0xff00
    17a6:	0a1a      	lsrs	r2, r3, #8
    17a8:	f44f 4366 	mov.w	r3, #58880	; 0xe600
    17ac:	f2c4 030f 	movt	r3, #16399	; 0x400f
    17b0:	18d3      	adds	r3, r2, r3
    17b2:	f003 4270 	and.w	r2, r3, #4026531840	; 0xf0000000
    17b6:	687b      	ldr	r3, [r7, #4]
    17b8:	f403 437f 	and.w	r3, r3, #65280	; 0xff00
    17bc:	0a19      	lsrs	r1, r3, #8
    17be:	f44f 4366 	mov.w	r3, #58880	; 0xe600
    17c2:	f2c4 030f 	movt	r3, #16399	; 0x400f
    17c6:	18cb      	adds	r3, r1, r3
    17c8:	f3c3 0313 	ubfx	r3, r3, #0, #20
    17cc:	015b      	lsls	r3, r3, #5
    17ce:	431a      	orrs	r2, r3
    17d0:	687b      	ldr	r3, [r7, #4]
    17d2:	b2db      	uxtb	r3, r3
    17d4:	009b      	lsls	r3, r3, #2
    17d6:	4313      	orrs	r3, r2
    17d8:	f043 7300 	orr.w	r3, r3, #33554432	; 0x2000000
                  ulPeripheral & 0xff) = 1;
    17dc:	2201      	movs	r2, #1
    17de:	601a      	str	r2, [r3, #0]
    17e0:	e01b      	b.n	181a <SysCtlPeripheralEnable+0x8e>
    else
    {
        //
        // Enable this peripheral.
        //
        HWREG(g_pulRCGCRegs[SYSCTL_PERIPH_INDEX(ulPeripheral)]) |=
    17e2:	687b      	ldr	r3, [r7, #4]
    17e4:	0f1a      	lsrs	r2, r3, #28
    17e6:	f242 2338 	movw	r3, #8760	; 0x2238
    17ea:	f2c0 0300 	movt	r3, #0
    17ee:	f853 3022 	ldr.w	r3, [r3, r2, lsl #2]
    17f2:	461a      	mov	r2, r3
    17f4:	687b      	ldr	r3, [r7, #4]
    17f6:	0f19      	lsrs	r1, r3, #28
    17f8:	f242 2338 	movw	r3, #8760	; 0x2238
    17fc:	f2c0 0300 	movt	r3, #0
    1800:	f853 3021 	ldr.w	r3, [r3, r1, lsl #2]
    1804:	6819      	ldr	r1, [r3, #0]
            SYSCTL_PERIPH_MASK(ulPeripheral);
    1806:	687b      	ldr	r3, [r7, #4]
    1808:	b298      	uxth	r0, r3
    180a:	687b      	ldr	r3, [r7, #4]
    180c:	f403 13f8 	and.w	r3, r3, #2031616	; 0x1f0000
    1810:	0c1b      	lsrs	r3, r3, #16
    1812:	fa00 f303 	lsl.w	r3, r0, r3
    else
    {
        //
        // Enable this peripheral.
        //
        HWREG(g_pulRCGCRegs[SYSCTL_PERIPH_INDEX(ulPeripheral)]) |=
    1816:	430b      	orrs	r3, r1
    1818:	6013      	str	r3, [r2, #0]
            SYSCTL_PERIPH_MASK(ulPeripheral);
    }
}
    181a:	f107 070c 	add.w	r7, r7, #12
    181e:	46bd      	mov	sp, r7
    1820:	bc80      	pop	{r7}
    1822:	4770      	bx	lr

00001824 <SysCtlDelay>:
#endif
#if defined(codered) || defined(gcc) || defined(sourcerygxx)
void __attribute__((naked))
SysCtlDelay(unsigned long ulCount)
{
    __asm("    subs    r0, #1\n"
    1824:	3801      	subs	r0, #1
    1826:	f47f affd 	bne.w	1824 <SysCtlDelay>
    182a:	4770      	bx	lr

0000182c <SysCtlClockSet>:
//! \return None.
//
//*****************************************************************************
void
SysCtlClockSet(unsigned long ulConfig)
{
    182c:	b580      	push	{r7, lr}
    182e:	b086      	sub	sp, #24
    1830:	af00      	add	r7, sp, #0
    1832:	6078      	str	r0, [r7, #4]

    //
    // See if this is a Sandstorm-class device and clocking features from newer
    // devices were requested.
    //
    if(CLASS_IS_SANDSTORM && (ulConfig & SYSCTL_RCC2_USERCC2))
    1834:	f44f 4360 	mov.w	r3, #57344	; 0xe000
    1838:	f2c4 030f 	movt	r3, #16399	; 0x400f
    183c:	681b      	ldr	r3, [r3, #0]
    183e:	f003 43e0 	and.w	r3, r3, #1879048192	; 0x70000000
    1842:	2b00      	cmp	r3, #0
    1844:	d00b      	beq.n	185e <SysCtlClockSet+0x32>
    1846:	f44f 4360 	mov.w	r3, #57344	; 0xe000
    184a:	f2c4 030f 	movt	r3, #16399	; 0x400f
    184e:	681a      	ldr	r2, [r3, #0]
    1850:	2300      	movs	r3, #0
    1852:	f2c7 03ff 	movt	r3, #28927	; 0x70ff
    1856:	4013      	ands	r3, r2
    1858:	f1b3 5f80 	cmp.w	r3, #268435456	; 0x10000000
    185c:	d103      	bne.n	1866 <SysCtlClockSet+0x3a>
    185e:	687b      	ldr	r3, [r7, #4]
    1860:	2b00      	cmp	r3, #0
    1862:	f2c0 812a 	blt.w	1aba <SysCtlClockSet+0x28e>
    //
    // Get the current value of the RCC and RCC2 registers.  If using a
    // Sandstorm-class device, the RCC2 register reads back as zero and the
    // writes to it from within this function are ignored.
    //
    ulRCC = HWREG(SYSCTL_RCC);
    1866:	f24e 0360 	movw	r3, #57440	; 0xe060
    186a:	f2c4 030f 	movt	r3, #16399	; 0x400f
    186e:	681b      	ldr	r3, [r3, #0]
    1870:	613b      	str	r3, [r7, #16]
    ulRCC2 = HWREG(SYSCTL_RCC2);
    1872:	f24e 0370 	movw	r3, #57456	; 0xe070
    1876:	f2c4 030f 	movt	r3, #16399	; 0x400f
    187a:	681b      	ldr	r3, [r3, #0]
    187c:	60fb      	str	r3, [r7, #12]

    //
    // Bypass the PLL and system clock dividers for now.
    //
    ulRCC |= SYSCTL_RCC_BYPASS;
    187e:	693b      	ldr	r3, [r7, #16]
    1880:	f443 6300 	orr.w	r3, r3, #2048	; 0x800
    1884:	613b      	str	r3, [r7, #16]
    ulRCC &= ~(SYSCTL_RCC_USESYSDIV);
    1886:	693b      	ldr	r3, [r7, #16]
    1888:	f423 0380 	bic.w	r3, r3, #4194304	; 0x400000
    188c:	613b      	str	r3, [r7, #16]
    ulRCC2 |= SYSCTL_RCC2_BYPASS2;
    188e:	68fb      	ldr	r3, [r7, #12]
    1890:	f443 6300 	orr.w	r3, r3, #2048	; 0x800
    1894:	60fb      	str	r3, [r7, #12]

    //
    // Write the new RCC value.
    //
    HWREG(SYSCTL_RCC) = ulRCC;
    1896:	f24e 0360 	movw	r3, #57440	; 0xe060
    189a:	f2c4 030f 	movt	r3, #16399	; 0x400f
    189e:	693a      	ldr	r2, [r7, #16]
    18a0:	601a      	str	r2, [r3, #0]
    HWREG(SYSCTL_RCC2) = ulRCC2;
    18a2:	f24e 0370 	movw	r3, #57456	; 0xe070
    18a6:	f2c4 030f 	movt	r3, #16399	; 0x400f
    18aa:	68fa      	ldr	r2, [r7, #12]
    18ac:	601a      	str	r2, [r3, #0]

    //
    // See if either oscillator needs to be enabled.
    //
    if(((ulRCC & SYSCTL_RCC_IOSCDIS) && !(ulConfig & SYSCTL_RCC_IOSCDIS)) ||
    18ae:	693b      	ldr	r3, [r7, #16]
    18b0:	f003 0302 	and.w	r3, r3, #2
    18b4:	2b00      	cmp	r3, #0
    18b6:	d004      	beq.n	18c2 <SysCtlClockSet+0x96>
    18b8:	687b      	ldr	r3, [r7, #4]
    18ba:	f003 0302 	and.w	r3, r3, #2
    18be:	2b00      	cmp	r3, #0
    18c0:	d009      	beq.n	18d6 <SysCtlClockSet+0xaa>
       ((ulRCC & SYSCTL_RCC_MOSCDIS) && !(ulConfig & SYSCTL_RCC_MOSCDIS)))
    18c2:	693b      	ldr	r3, [r7, #16]
    18c4:	f003 0301 	and.w	r3, r3, #1
    HWREG(SYSCTL_RCC2) = ulRCC2;

    //
    // See if either oscillator needs to be enabled.
    //
    if(((ulRCC & SYSCTL_RCC_IOSCDIS) && !(ulConfig & SYSCTL_RCC_IOSCDIS)) ||
    18c8:	2b00      	cmp	r3, #0
    18ca:	d02e      	beq.n	192a <SysCtlClockSet+0xfe>
       ((ulRCC & SYSCTL_RCC_MOSCDIS) && !(ulConfig & SYSCTL_RCC_MOSCDIS)))
    18cc:	687b      	ldr	r3, [r7, #4]
    18ce:	f003 0301 	and.w	r3, r3, #1
    18d2:	2b00      	cmp	r3, #0
    18d4:	d129      	bne.n	192a <SysCtlClockSet+0xfe>
        //
        // Make sure that the required oscillators are enabled.  For now, the
        // previously enabled oscillators must be enabled along with the newly
        // requested oscillators.
        //
        ulRCC &= (~(SYSCTL_RCC_IOSCDIS | SYSCTL_RCC_MOSCDIS) |
    18d6:	687b      	ldr	r3, [r7, #4]
    18d8:	f063 0303 	orn	r3, r3, #3
    18dc:	693a      	ldr	r2, [r7, #16]
    18de:	4013      	ands	r3, r2
    18e0:	613b      	str	r3, [r7, #16]
                  (ulConfig & (SYSCTL_RCC_IOSCDIS | SYSCTL_RCC_MOSCDIS)));

        //
        // Write the new RCC value.
        //
        HWREG(SYSCTL_RCC) = ulRCC;
    18e2:	f24e 0360 	movw	r3, #57440	; 0xe060
    18e6:	f2c4 030f 	movt	r3, #16399	; 0x400f
    18ea:	693a      	ldr	r2, [r7, #16]
    18ec:	601a      	str	r2, [r3, #0]
        //
        // Wait for a bit, giving the oscillator time to stabilize.  The number
        // of iterations is adjusted based on the current clock source; a
        // smaller number of iterations is required for slower clock rates.
        //
        if(((ulRCC2 & SYSCTL_RCC2_USERCC2) &&
    18ee:	68fb      	ldr	r3, [r7, #12]
    18f0:	2b00      	cmp	r3, #0
    18f2:	da09      	bge.n	1908 <SysCtlClockSet+0xdc>
            (((ulRCC2 & SYSCTL_RCC2_OSCSRC2_M) == SYSCTL_RCC2_OSCSRC2_30) ||
    18f4:	68fb      	ldr	r3, [r7, #12]
    18f6:	f003 0370 	and.w	r3, r3, #112	; 0x70
        //
        // Wait for a bit, giving the oscillator time to stabilize.  The number
        // of iterations is adjusted based on the current clock source; a
        // smaller number of iterations is required for slower clock rates.
        //
        if(((ulRCC2 & SYSCTL_RCC2_USERCC2) &&
    18fa:	2b30      	cmp	r3, #48	; 0x30
    18fc:	d00c      	beq.n	1918 <SysCtlClockSet+0xec>
            (((ulRCC2 & SYSCTL_RCC2_OSCSRC2_M) == SYSCTL_RCC2_OSCSRC2_30) ||
             ((ulRCC2 & SYSCTL_RCC2_OSCSRC2_M) == SYSCTL_RCC2_OSCSRC2_32))) ||
    18fe:	68fb      	ldr	r3, [r7, #12]
    1900:	f003 0370 	and.w	r3, r3, #112	; 0x70
        // Wait for a bit, giving the oscillator time to stabilize.  The number
        // of iterations is adjusted based on the current clock source; a
        // smaller number of iterations is required for slower clock rates.
        //
        if(((ulRCC2 & SYSCTL_RCC2_USERCC2) &&
            (((ulRCC2 & SYSCTL_RCC2_OSCSRC2_M) == SYSCTL_RCC2_OSCSRC2_30) ||
    1904:	2b70      	cmp	r3, #112	; 0x70
    1906:	d007      	beq.n	1918 <SysCtlClockSet+0xec>
             ((ulRCC2 & SYSCTL_RCC2_OSCSRC2_M) == SYSCTL_RCC2_OSCSRC2_32))) ||
           (!(ulRCC2 & SYSCTL_RCC2_USERCC2) &&
    1908:	68fb      	ldr	r3, [r7, #12]
        // of iterations is adjusted based on the current clock source; a
        // smaller number of iterations is required for slower clock rates.
        //
        if(((ulRCC2 & SYSCTL_RCC2_USERCC2) &&
            (((ulRCC2 & SYSCTL_RCC2_OSCSRC2_M) == SYSCTL_RCC2_OSCSRC2_30) ||
             ((ulRCC2 & SYSCTL_RCC2_OSCSRC2_M) == SYSCTL_RCC2_OSCSRC2_32))) ||
    190a:	2b00      	cmp	r3, #0
    190c:	db09      	blt.n	1922 <SysCtlClockSet+0xf6>
           (!(ulRCC2 & SYSCTL_RCC2_USERCC2) &&
            ((ulRCC & SYSCTL_RCC_OSCSRC_M) == SYSCTL_RCC_OSCSRC_30)))
    190e:	693b      	ldr	r3, [r7, #16]
    1910:	f003 0330 	and.w	r3, r3, #48	; 0x30
        // smaller number of iterations is required for slower clock rates.
        //
        if(((ulRCC2 & SYSCTL_RCC2_USERCC2) &&
            (((ulRCC2 & SYSCTL_RCC2_OSCSRC2_M) == SYSCTL_RCC2_OSCSRC2_30) ||
             ((ulRCC2 & SYSCTL_RCC2_OSCSRC2_M) == SYSCTL_RCC2_OSCSRC2_32))) ||
           (!(ulRCC2 & SYSCTL_RCC2_USERCC2) &&
    1914:	2b30      	cmp	r3, #48	; 0x30
    1916:	d104      	bne.n	1922 <SysCtlClockSet+0xf6>
            ((ulRCC & SYSCTL_RCC_OSCSRC_M) == SYSCTL_RCC_OSCSRC_30)))
        {
            //
            // Delay for 4096 iterations.
            //
            SysCtlDelay(4096);
    1918:	f44f 5080 	mov.w	r0, #4096	; 0x1000
    191c:	f7ff ff82 	bl	1824 <SysCtlDelay>
    1920:	e003      	b.n	192a <SysCtlClockSet+0xfe>
        else
        {
            //
            // Delay for 524,288 iterations.
            //
            SysCtlDelay(524288);
    1922:	f44f 2000 	mov.w	r0, #524288	; 0x80000
    1926:	f7ff ff7d 	bl	1824 <SysCtlDelay>
    //
    // Set the new crystal value and oscillator source.  Because the OSCSRC2
    // field in RCC2 overlaps the XTAL field in RCC, the OSCSRC field has a
    // special encoding within ulConfig to avoid the overlap.
    //
    ulRCC &= ~(SYSCTL_RCC_XTAL_M | SYSCTL_RCC_OSCSRC_M);
    192a:	693b      	ldr	r3, [r7, #16]
    192c:	f423 63fe 	bic.w	r3, r3, #2032	; 0x7f0
    1930:	613b      	str	r3, [r7, #16]
    ulRCC |= ulConfig & (SYSCTL_RCC_XTAL_M | SYSCTL_RCC_OSCSRC_M);
    1932:	687b      	ldr	r3, [r7, #4]
    1934:	f403 63fe 	and.w	r3, r3, #2032	; 0x7f0
    1938:	693a      	ldr	r2, [r7, #16]
    193a:	4313      	orrs	r3, r2
    193c:	613b      	str	r3, [r7, #16]
    ulRCC2 &= ~(SYSCTL_RCC2_USERCC2 | SYSCTL_RCC2_OSCSRC2_M);
    193e:	68fb      	ldr	r3, [r7, #12]
    1940:	f023 4300 	bic.w	r3, r3, #2147483648	; 0x80000000
    1944:	f023 0370 	bic.w	r3, r3, #112	; 0x70
    1948:	60fb      	str	r3, [r7, #12]
    ulRCC2 |= ulConfig & (SYSCTL_RCC2_USERCC2 | SYSCTL_RCC_OSCSRC_M);
    194a:	687a      	ldr	r2, [r7, #4]
    194c:	2330      	movs	r3, #48	; 0x30
    194e:	f2c8 0300 	movt	r3, #32768	; 0x8000
    1952:	4013      	ands	r3, r2
    1954:	68fa      	ldr	r2, [r7, #12]
    1956:	4313      	orrs	r3, r2
    1958:	60fb      	str	r3, [r7, #12]
    ulRCC2 |= (ulConfig & 0x00000008) << 3;
    195a:	687b      	ldr	r3, [r7, #4]
    195c:	f003 0308 	and.w	r3, r3, #8
    1960:	00db      	lsls	r3, r3, #3
    1962:	68fa      	ldr	r2, [r7, #12]
    1964:	4313      	orrs	r3, r2
    1966:	60fb      	str	r3, [r7, #12]

    //
    // Write the new RCC value.
    //
    HWREG(SYSCTL_RCC) = ulRCC;
    1968:	f24e 0360 	movw	r3, #57440	; 0xe060
    196c:	f2c4 030f 	movt	r3, #16399	; 0x400f
    1970:	693a      	ldr	r2, [r7, #16]
    1972:	601a      	str	r2, [r3, #0]
    HWREG(SYSCTL_RCC2) = ulRCC2;
    1974:	f24e 0370 	movw	r3, #57456	; 0xe070
    1978:	f2c4 030f 	movt	r3, #16399	; 0x400f
    197c:	68fa      	ldr	r2, [r7, #12]
    197e:	601a      	str	r2, [r3, #0]

    //
    // Wait for a bit so that new crystal value and oscillator source can take
    // effect.
    //
    SysCtlDelay(16);
    1980:	2010      	movs	r0, #16
    1982:	f7ff ff4f 	bl	1824 <SysCtlDelay>

    //
    // Set the PLL configuration.
    //
    ulRCC &= ~(SYSCTL_RCC_PWRDN | SYSCTL_RCC_OEN);
    1986:	693b      	ldr	r3, [r7, #16]
    1988:	f423 5340 	bic.w	r3, r3, #12288	; 0x3000
    198c:	613b      	str	r3, [r7, #16]
    ulRCC |= ulConfig & (SYSCTL_RCC_PWRDN | SYSCTL_RCC_OEN);
    198e:	687b      	ldr	r3, [r7, #4]
    1990:	f403 5340 	and.w	r3, r3, #12288	; 0x3000
    1994:	693a      	ldr	r2, [r7, #16]
    1996:	4313      	orrs	r3, r2
    1998:	613b      	str	r3, [r7, #16]
    ulRCC2 &= ~(SYSCTL_RCC2_PWRDN2);
    199a:	68fb      	ldr	r3, [r7, #12]
    199c:	f423 5300 	bic.w	r3, r3, #8192	; 0x2000
    19a0:	60fb      	str	r3, [r7, #12]
    ulRCC2 |= ulConfig & SYSCTL_RCC2_PWRDN2;
    19a2:	687b      	ldr	r3, [r7, #4]
    19a4:	f403 5300 	and.w	r3, r3, #8192	; 0x2000
    19a8:	68fa      	ldr	r2, [r7, #12]
    19aa:	4313      	orrs	r3, r2
    19ac:	60fb      	str	r3, [r7, #12]

    //
    // Clear the PLL lock interrupt.
    //
    HWREG(SYSCTL_MISC) = SYSCTL_INT_PLL_LOCK;
    19ae:	f24e 0358 	movw	r3, #57432	; 0xe058
    19b2:	f2c4 030f 	movt	r3, #16399	; 0x400f
    19b6:	2240      	movs	r2, #64	; 0x40
    19b8:	601a      	str	r2, [r3, #0]

    //
    // Write the new RCC value.
    //
    if(ulRCC2 & SYSCTL_RCC2_USERCC2)
    19ba:	68fb      	ldr	r3, [r7, #12]
    19bc:	2b00      	cmp	r3, #0
    19be:	da0c      	bge.n	19da <SysCtlClockSet+0x1ae>
    {
        HWREG(SYSCTL_RCC2) = ulRCC2;
    19c0:	f24e 0370 	movw	r3, #57456	; 0xe070
    19c4:	f2c4 030f 	movt	r3, #16399	; 0x400f
    19c8:	68fa      	ldr	r2, [r7, #12]
    19ca:	601a      	str	r2, [r3, #0]
        HWREG(SYSCTL_RCC) = ulRCC;
    19cc:	f24e 0360 	movw	r3, #57440	; 0xe060
    19d0:	f2c4 030f 	movt	r3, #16399	; 0x400f
    19d4:	693a      	ldr	r2, [r7, #16]
    19d6:	601a      	str	r2, [r3, #0]
    19d8:	e00b      	b.n	19f2 <SysCtlClockSet+0x1c6>
    }
    else
    {
        HWREG(SYSCTL_RCC) = ulRCC;
    19da:	f24e 0360 	movw	r3, #57440	; 0xe060
    19de:	f2c4 030f 	movt	r3, #16399	; 0x400f
    19e2:	693a      	ldr	r2, [r7, #16]
    19e4:	601a      	str	r2, [r3, #0]
        HWREG(SYSCTL_RCC2) = ulRCC2;
    19e6:	f24e 0370 	movw	r3, #57456	; 0xe070
    19ea:	f2c4 030f 	movt	r3, #16399	; 0x400f
    19ee:	68fa      	ldr	r2, [r7, #12]
    19f0:	601a      	str	r2, [r3, #0]

    //
    // Set the requested system divider and disable the appropriate
    // oscillators.  This value is not written immediately.
    //
    ulRCC &= ~(SYSCTL_RCC_SYSDIV_M | SYSCTL_RCC_USESYSDIV |
    19f2:	693b      	ldr	r3, [r7, #16]
    19f4:	f023 63f8 	bic.w	r3, r3, #130023424	; 0x7c00000
    19f8:	f023 0303 	bic.w	r3, r3, #3
    19fc:	613b      	str	r3, [r7, #16]
               SYSCTL_RCC_IOSCDIS | SYSCTL_RCC_MOSCDIS);
    ulRCC |= ulConfig & (SYSCTL_RCC_SYSDIV_M | SYSCTL_RCC_USESYSDIV |
    19fe:	687a      	ldr	r2, [r7, #4]
    1a00:	2303      	movs	r3, #3
    1a02:	f2c0 73c0 	movt	r3, #1984	; 0x7c0
    1a06:	4013      	ands	r3, r2
    1a08:	693a      	ldr	r2, [r7, #16]
    1a0a:	4313      	orrs	r3, r2
    1a0c:	613b      	str	r3, [r7, #16]
                         SYSCTL_RCC_IOSCDIS | SYSCTL_RCC_MOSCDIS);
    ulRCC2 &= ~(SYSCTL_RCC2_SYSDIV2_M);
    1a0e:	68fb      	ldr	r3, [r7, #12]
    1a10:	f023 53fc 	bic.w	r3, r3, #528482304	; 0x1f800000
    1a14:	60fb      	str	r3, [r7, #12]
    ulRCC2 |= ulConfig & SYSCTL_RCC2_SYSDIV2_M;
    1a16:	687b      	ldr	r3, [r7, #4]
    1a18:	f003 53fc 	and.w	r3, r3, #528482304	; 0x1f800000
    1a1c:	68fa      	ldr	r2, [r7, #12]
    1a1e:	4313      	orrs	r3, r2
    1a20:	60fb      	str	r3, [r7, #12]
    if(ulConfig & SYSCTL_RCC2_DIV400)
    1a22:	687b      	ldr	r3, [r7, #4]
    1a24:	f003 4380 	and.w	r3, r3, #1073741824	; 0x40000000
    1a28:	2b00      	cmp	r3, #0
    1a2a:	d010      	beq.n	1a4e <SysCtlClockSet+0x222>
    {
        ulRCC |= SYSCTL_RCC_USESYSDIV;
    1a2c:	693b      	ldr	r3, [r7, #16]
    1a2e:	f443 0380 	orr.w	r3, r3, #4194304	; 0x400000
    1a32:	613b      	str	r3, [r7, #16]
        ulRCC2 &= ~(SYSCTL_RCC_USESYSDIV);
    1a34:	68fb      	ldr	r3, [r7, #12]
    1a36:	f423 0380 	bic.w	r3, r3, #4194304	; 0x400000
    1a3a:	60fb      	str	r3, [r7, #12]
        ulRCC2 |= ulConfig & (SYSCTL_RCC2_DIV400 | SYSCTL_RCC2_SYSDIV2LSB);
    1a3c:	687a      	ldr	r2, [r7, #4]
    1a3e:	2300      	movs	r3, #0
    1a40:	f2c4 0340 	movt	r3, #16448	; 0x4040
    1a44:	4013      	ands	r3, r2
    1a46:	68fa      	ldr	r2, [r7, #12]
    1a48:	4313      	orrs	r3, r2
    1a4a:	60fb      	str	r3, [r7, #12]
    1a4c:	e003      	b.n	1a56 <SysCtlClockSet+0x22a>
    }
    else
    {
        ulRCC2 &= ~(SYSCTL_RCC2_DIV400);
    1a4e:	68fb      	ldr	r3, [r7, #12]
    1a50:	f023 4380 	bic.w	r3, r3, #1073741824	; 0x40000000
    1a54:	60fb      	str	r3, [r7, #12]
    }

    //
    // See if the PLL output is being used to clock the system.
    //
    if(!(ulConfig & SYSCTL_RCC_BYPASS))
    1a56:	687b      	ldr	r3, [r7, #4]
    1a58:	f403 6300 	and.w	r3, r3, #2048	; 0x800
    1a5c:	2b00      	cmp	r3, #0
    1a5e:	d11c      	bne.n	1a9a <SysCtlClockSet+0x26e>
    {
        //
        // Wait until the PLL has locked.
        //
        for(ulDelay = 32768; ulDelay > 0; ulDelay--)
    1a60:	f44f 4300 	mov.w	r3, #32768	; 0x8000
    1a64:	617b      	str	r3, [r7, #20]
    1a66:	e00b      	b.n	1a80 <SysCtlClockSet+0x254>
        {
            if(HWREG(SYSCTL_RIS) & SYSCTL_INT_PLL_LOCK)
    1a68:	f24e 0350 	movw	r3, #57424	; 0xe050
    1a6c:	f2c4 030f 	movt	r3, #16399	; 0x400f
    1a70:	681b      	ldr	r3, [r3, #0]
    1a72:	f003 0340 	and.w	r3, r3, #64	; 0x40
    1a76:	2b00      	cmp	r3, #0
    1a78:	d106      	bne.n	1a88 <SysCtlClockSet+0x25c>
    if(!(ulConfig & SYSCTL_RCC_BYPASS))
    {
        //
        // Wait until the PLL has locked.
        //
        for(ulDelay = 32768; ulDelay > 0; ulDelay--)
    1a7a:	697b      	ldr	r3, [r7, #20]
    1a7c:	3b01      	subs	r3, #1
    1a7e:	617b      	str	r3, [r7, #20]
    1a80:	697b      	ldr	r3, [r7, #20]
    1a82:	2b00      	cmp	r3, #0
    1a84:	d1f0      	bne.n	1a68 <SysCtlClockSet+0x23c>
    1a86:	e000      	b.n	1a8a <SysCtlClockSet+0x25e>
        {
            if(HWREG(SYSCTL_RIS) & SYSCTL_INT_PLL_LOCK)
            {
                break;
    1a88:	bf00      	nop
        }

        //
        // Enable use of the PLL.
        //
        ulRCC &= ~(SYSCTL_RCC_BYPASS);
    1a8a:	693b      	ldr	r3, [r7, #16]
    1a8c:	f423 6300 	bic.w	r3, r3, #2048	; 0x800
    1a90:	613b      	str	r3, [r7, #16]
        ulRCC2 &= ~(SYSCTL_RCC2_BYPASS2);
    1a92:	68fb      	ldr	r3, [r7, #12]
    1a94:	f423 6300 	bic.w	r3, r3, #2048	; 0x800
    1a98:	60fb      	str	r3, [r7, #12]
    }

    //
    // Write the final RCC value.
    //
    HWREG(SYSCTL_RCC) = ulRCC;
    1a9a:	f24e 0360 	movw	r3, #57440	; 0xe060
    1a9e:	f2c4 030f 	movt	r3, #16399	; 0x400f
    1aa2:	693a      	ldr	r2, [r7, #16]
    1aa4:	601a      	str	r2, [r3, #0]
    HWREG(SYSCTL_RCC2) = ulRCC2;
    1aa6:	f24e 0370 	movw	r3, #57456	; 0xe070
    1aaa:	f2c4 030f 	movt	r3, #16399	; 0x400f
    1aae:	68fa      	ldr	r2, [r7, #12]
    1ab0:	601a      	str	r2, [r3, #0]

    //
    // Delay for a little bit so that the system divider takes effect.
    //
    SysCtlDelay(16);
    1ab2:	2010      	movs	r0, #16
    1ab4:	f7ff feb6 	bl	1824 <SysCtlDelay>
    1ab8:	e000      	b.n	1abc <SysCtlClockSet+0x290>
    {
        //
        // Return without changing the clocking because the requested
        // configuration can not be achieved.
        //
        return;
    1aba:	bf00      	nop

    //
    // Delay for a little bit so that the system divider takes effect.
    //
    SysCtlDelay(16);
}
    1abc:	f107 0718 	add.w	r7, r7, #24
    1ac0:	46bd      	mov	sp, r7
    1ac2:	bd80      	pop	{r7, pc}

00001ac4 <SysCtlClockGet>:
//! \return The processor clock rate.
//
//*****************************************************************************
unsigned long
SysCtlClockGet(void)
{
    1ac4:	b480      	push	{r7}
    1ac6:	b087      	sub	sp, #28
    1ac8:	af00      	add	r7, sp, #0
    //
    // Read RCC and RCC2.  For Sandstorm-class devices (which do not have
    // RCC2), the RCC2 read returns 0, indicating that RCC2 is
    // disabled (because the SYSCTL_RCC2_USERCC2 bit is clear).
    //
    ulRCC = HWREG(SYSCTL_RCC);
    1aca:	f24e 0360 	movw	r3, #57440	; 0xe060
    1ace:	f2c4 030f 	movt	r3, #16399	; 0x400f
    1ad2:	681b      	ldr	r3, [r3, #0]
    1ad4:	617b      	str	r3, [r7, #20]
    ulRCC2 = HWREG(SYSCTL_RCC2);
    1ad6:	f24e 0370 	movw	r3, #57456	; 0xe070
    1ada:	f2c4 030f 	movt	r3, #16399	; 0x400f
    1ade:	681b      	ldr	r3, [r3, #0]
    1ae0:	60fb      	str	r3, [r7, #12]

    //
    // Get the base clock rate.
    //
    switch((ulRCC2 & SYSCTL_RCC2_USERCC2) ?
    1ae2:	68fb      	ldr	r3, [r7, #12]
           (ulRCC2 & SYSCTL_RCC2_OSCSRC2_M) :
    1ae4:	2b00      	cmp	r3, #0
    1ae6:	da03      	bge.n	1af0 <SysCtlClockGet+0x2c>
    1ae8:	68fb      	ldr	r3, [r7, #12]
    1aea:	f003 0370 	and.w	r3, r3, #112	; 0x70
    1aee:	e002      	b.n	1af6 <SysCtlClockGet+0x32>
    1af0:	697b      	ldr	r3, [r7, #20]
    1af2:	f003 0330 	and.w	r3, r3, #48	; 0x30
    ulRCC2 = HWREG(SYSCTL_RCC2);

    //
    // Get the base clock rate.
    //
    switch((ulRCC2 & SYSCTL_RCC2_USERCC2) ?
    1af6:	2b20      	cmp	r3, #32
    1af8:	d070      	beq.n	1bdc <SysCtlClockGet+0x118>
    1afa:	2b20      	cmp	r3, #32
    1afc:	d804      	bhi.n	1b08 <SysCtlClockGet+0x44>
    1afe:	2b00      	cmp	r3, #0
    1b00:	d00c      	beq.n	1b1c <SysCtlClockGet+0x58>
    1b02:	2b10      	cmp	r3, #16
    1b04:	d016      	beq.n	1b34 <SysCtlClockGet+0x70>
    1b06:	e0c9      	b.n	1c9c <SysCtlClockGet+0x1d8>
    1b08:	2b60      	cmp	r3, #96	; 0x60
    1b0a:	f000 80bf 	beq.w	1c8c <SysCtlClockGet+0x1c8>
    1b0e:	2b70      	cmp	r3, #112	; 0x70
    1b10:	f000 80c0 	beq.w	1c94 <SysCtlClockGet+0x1d0>
    1b14:	2b30      	cmp	r3, #48	; 0x30
    1b16:	f000 80b5 	beq.w	1c84 <SysCtlClockGet+0x1c0>
    1b1a:	e0bf      	b.n	1c9c <SysCtlClockGet+0x1d8>
        // The main oscillator is the clock source.  Determine its rate from
        // the crystal setting field.
        //
        case SYSCTL_RCC_OSCSRC_MAIN:
        {
            ulClk = g_pulXtals[(ulRCC & SYSCTL_RCC_XTAL_M) >>
    1b1c:	697b      	ldr	r3, [r7, #20]
    1b1e:	f403 63f8 	and.w	r3, r3, #1984	; 0x7c0
    1b22:	099a      	lsrs	r2, r3, #6
    1b24:	f242 2344 	movw	r3, #8772	; 0x2244
    1b28:	f2c0 0300 	movt	r3, #0
    1b2c:	f853 3022 	ldr.w	r3, [r3, r2, lsl #2]
    1b30:	613b      	str	r3, [r7, #16]
                               SYSCTL_RCC_XTAL_S];
            break;
    1b32:	e0b5      	b.n	1ca0 <SysCtlClockGet+0x1dc>
        case SYSCTL_RCC_OSCSRC_INT:
        {
            //
            // See if this is a Sandstorm-class or Fury-class device.
            //
            if(CLASS_IS_SANDSTORM)
    1b34:	f44f 4360 	mov.w	r3, #57344	; 0xe000
    1b38:	f2c4 030f 	movt	r3, #16399	; 0x400f
    1b3c:	681b      	ldr	r3, [r3, #0]
    1b3e:	f003 43e0 	and.w	r3, r3, #1879048192	; 0x70000000
    1b42:	2b00      	cmp	r3, #0
    1b44:	d00b      	beq.n	1b5e <SysCtlClockGet+0x9a>
    1b46:	f44f 4360 	mov.w	r3, #57344	; 0xe000
    1b4a:	f2c4 030f 	movt	r3, #16399	; 0x400f
    1b4e:	681a      	ldr	r2, [r3, #0]
    1b50:	2300      	movs	r3, #0
    1b52:	f2c7 03ff 	movt	r3, #28927	; 0x70ff
    1b56:	4013      	ands	r3, r2
    1b58:	f1b3 5f80 	cmp.w	r3, #268435456	; 0x10000000
    1b5c:	d105      	bne.n	1b6a <SysCtlClockGet+0xa6>
            {
                //
                // The internal oscillator on a Sandstorm-class device is
                // 15 MHz +/- 50%.
                //
                ulClk = 15000000;
    1b5e:	f24e 13c0 	movw	r3, #57792	; 0xe1c0
    1b62:	f2c0 03e4 	movt	r3, #228	; 0xe4
    1b66:	613b      	str	r3, [r7, #16]
    1b68:	e037      	b.n	1bda <SysCtlClockGet+0x116>
            }
            else if((CLASS_IS_FURY && REVISION_IS_A2) ||
    1b6a:	f44f 4360 	mov.w	r3, #57344	; 0xe000
    1b6e:	f2c4 030f 	movt	r3, #16399	; 0x400f
    1b72:	681a      	ldr	r2, [r3, #0]
    1b74:	2300      	movs	r3, #0
    1b76:	f2c7 03ff 	movt	r3, #28927	; 0x70ff
    1b7a:	4013      	ands	r3, r2
    1b7c:	2200      	movs	r2, #0
    1b7e:	f2c1 0201 	movt	r2, #4097	; 0x1001
    1b82:	4293      	cmp	r3, r2
    1b84:	d107      	bne.n	1b96 <SysCtlClockGet+0xd2>
    1b86:	f44f 4360 	mov.w	r3, #57344	; 0xe000
    1b8a:	f2c4 030f 	movt	r3, #16399	; 0x400f
    1b8e:	681b      	ldr	r3, [r3, #0]
    1b90:	b29b      	uxth	r3, r3
    1b92:	2b02      	cmp	r3, #2
    1b94:	d015      	beq.n	1bc2 <SysCtlClockGet+0xfe>
                    (CLASS_IS_DUSTDEVIL && REVISION_IS_A0))
    1b96:	f44f 4360 	mov.w	r3, #57344	; 0xe000
    1b9a:	f2c4 030f 	movt	r3, #16399	; 0x400f
    1b9e:	681a      	ldr	r2, [r3, #0]
    1ba0:	2300      	movs	r3, #0
    1ba2:	f2c7 03ff 	movt	r3, #28927	; 0x70ff
    1ba6:	4013      	ands	r3, r2
                // The internal oscillator on a Sandstorm-class device is
                // 15 MHz +/- 50%.
                //
                ulClk = 15000000;
            }
            else if((CLASS_IS_FURY && REVISION_IS_A2) ||
    1ba8:	2200      	movs	r2, #0
    1baa:	f2c1 0203 	movt	r2, #4099	; 0x1003
    1bae:	4293      	cmp	r3, r2
    1bb0:	d10d      	bne.n	1bce <SysCtlClockGet+0x10a>
                    (CLASS_IS_DUSTDEVIL && REVISION_IS_A0))
    1bb2:	f44f 4360 	mov.w	r3, #57344	; 0xe000
    1bb6:	f2c4 030f 	movt	r3, #16399	; 0x400f
    1bba:	681b      	ldr	r3, [r3, #0]
    1bbc:	b29b      	uxth	r3, r3
    1bbe:	2b00      	cmp	r3, #0
    1bc0:	d105      	bne.n	1bce <SysCtlClockGet+0x10a>
            {
                //
                // The internal oscillator on a rev A2 Fury-class device and a
                // Dustdevil-class device is 12 MHz +/- 30%.
                //
                ulClk = 12000000;
    1bc2:	f44f 53d8 	mov.w	r3, #6912	; 0x1b00
    1bc6:	f2c0 03b7 	movt	r3, #183	; 0xb7
    1bca:	613b      	str	r3, [r7, #16]
    1bcc:	e005      	b.n	1bda <SysCtlClockGet+0x116>
            else
            {
                //
                // The internal oscillator on all other devices is 16 MHz.
                //
                ulClk = 16000000;
    1bce:	f44f 5310 	mov.w	r3, #9216	; 0x2400
    1bd2:	f2c0 03f4 	movt	r3, #244	; 0xf4
    1bd6:	613b      	str	r3, [r7, #16]
            }
            break;
    1bd8:	e062      	b.n	1ca0 <SysCtlClockGet+0x1dc>
    1bda:	e061      	b.n	1ca0 <SysCtlClockGet+0x1dc>
        case SYSCTL_RCC_OSCSRC_INT4:
        {
            //
            // See if this is a Sandstorm-class or Fury-class device.
            //
            if(CLASS_IS_SANDSTORM)
    1bdc:	f44f 4360 	mov.w	r3, #57344	; 0xe000
    1be0:	f2c4 030f 	movt	r3, #16399	; 0x400f
    1be4:	681b      	ldr	r3, [r3, #0]
    1be6:	f003 43e0 	and.w	r3, r3, #1879048192	; 0x70000000
    1bea:	2b00      	cmp	r3, #0
    1bec:	d00b      	beq.n	1c06 <SysCtlClockGet+0x142>
    1bee:	f44f 4360 	mov.w	r3, #57344	; 0xe000
    1bf2:	f2c4 030f 	movt	r3, #16399	; 0x400f
    1bf6:	681a      	ldr	r2, [r3, #0]
    1bf8:	2300      	movs	r3, #0
    1bfa:	f2c7 03ff 	movt	r3, #28927	; 0x70ff
    1bfe:	4013      	ands	r3, r2
    1c00:	f1b3 5f80 	cmp.w	r3, #268435456	; 0x10000000
    1c04:	d105      	bne.n	1c12 <SysCtlClockGet+0x14e>
            {
                //
                // The internal oscillator on a Sandstorm-class device is
                // 15 MHz +/- 50%.
                //
                ulClk = 15000000 / 4;
    1c06:	f643 0370 	movw	r3, #14448	; 0x3870
    1c0a:	f2c0 0339 	movt	r3, #57	; 0x39
    1c0e:	613b      	str	r3, [r7, #16]
    1c10:	e037      	b.n	1c82 <SysCtlClockGet+0x1be>
            }
            else if((CLASS_IS_FURY && REVISION_IS_A2) ||
    1c12:	f44f 4360 	mov.w	r3, #57344	; 0xe000
    1c16:	f2c4 030f 	movt	r3, #16399	; 0x400f
    1c1a:	681a      	ldr	r2, [r3, #0]
    1c1c:	2300      	movs	r3, #0
    1c1e:	f2c7 03ff 	movt	r3, #28927	; 0x70ff
    1c22:	4013      	ands	r3, r2
    1c24:	2200      	movs	r2, #0
    1c26:	f2c1 0201 	movt	r2, #4097	; 0x1001
    1c2a:	4293      	cmp	r3, r2
    1c2c:	d107      	bne.n	1c3e <SysCtlClockGet+0x17a>
    1c2e:	f44f 4360 	mov.w	r3, #57344	; 0xe000
    1c32:	f2c4 030f 	movt	r3, #16399	; 0x400f
    1c36:	681b      	ldr	r3, [r3, #0]
    1c38:	b29b      	uxth	r3, r3
    1c3a:	2b02      	cmp	r3, #2
    1c3c:	d015      	beq.n	1c6a <SysCtlClockGet+0x1a6>
                    (CLASS_IS_DUSTDEVIL && REVISION_IS_A0))
    1c3e:	f44f 4360 	mov.w	r3, #57344	; 0xe000
    1c42:	f2c4 030f 	movt	r3, #16399	; 0x400f
    1c46:	681a      	ldr	r2, [r3, #0]
    1c48:	2300      	movs	r3, #0
    1c4a:	f2c7 03ff 	movt	r3, #28927	; 0x70ff
    1c4e:	4013      	ands	r3, r2
                // The internal oscillator on a Sandstorm-class device is
                // 15 MHz +/- 50%.
                //
                ulClk = 15000000 / 4;
            }
            else if((CLASS_IS_FURY && REVISION_IS_A2) ||
    1c50:	2200      	movs	r2, #0
    1c52:	f2c1 0203 	movt	r2, #4099	; 0x1003
    1c56:	4293      	cmp	r3, r2
    1c58:	d10d      	bne.n	1c76 <SysCtlClockGet+0x1b2>
                    (CLASS_IS_DUSTDEVIL && REVISION_IS_A0))
    1c5a:	f44f 4360 	mov.w	r3, #57344	; 0xe000
    1c5e:	f2c4 030f 	movt	r3, #16399	; 0x400f
    1c62:	681b      	ldr	r3, [r3, #0]
    1c64:	b29b      	uxth	r3, r3
    1c66:	2b00      	cmp	r3, #0
    1c68:	d105      	bne.n	1c76 <SysCtlClockGet+0x1b2>
            {
                //
                // The internal oscillator on a rev A2 Fury-class device and a
                // Dustdevil-class device is 12 MHz +/- 30%.
                //
                ulClk = 12000000 / 4;
    1c6a:	f24c 63c0 	movw	r3, #50880	; 0xc6c0
    1c6e:	f2c0 032d 	movt	r3, #45	; 0x2d
    1c72:	613b      	str	r3, [r7, #16]
    1c74:	e005      	b.n	1c82 <SysCtlClockGet+0x1be>
            else
            {
                //
                // The internal oscillator on a Tempest-class device is 16 MHz.
                //
                ulClk = 16000000 / 4;
    1c76:	f44f 6310 	mov.w	r3, #2304	; 0x900
    1c7a:	f2c0 033d 	movt	r3, #61	; 0x3d
    1c7e:	613b      	str	r3, [r7, #16]
            }
            break;
    1c80:	e00e      	b.n	1ca0 <SysCtlClockGet+0x1dc>
    1c82:	e00d      	b.n	1ca0 <SysCtlClockGet+0x1dc>
        case SYSCTL_RCC_OSCSRC_30:
        {
            //
            // The internal 30-KHz oscillator has an accuracy of +/- 30%.
            //
            ulClk = 30000;
    1c84:	f247 5330 	movw	r3, #30000	; 0x7530
    1c88:	613b      	str	r3, [r7, #16]
            break;
    1c8a:	e009      	b.n	1ca0 <SysCtlClockGet+0x1dc>
        // The 4.194304-MHz clock from the hibernate module is the clock
        // source.
        //
        case SYSCTL_RCC2_OSCSRC2_419:
        {
            ulClk = 4194304;
    1c8c:	f44f 0380 	mov.w	r3, #4194304	; 0x400000
    1c90:	613b      	str	r3, [r7, #16]
            break;
    1c92:	e005      	b.n	1ca0 <SysCtlClockGet+0x1dc>
        //
        // The 32.768-KHz clock from the hibernate module is the source clock.
        //
        case SYSCTL_RCC2_OSCSRC2_32:
        {
            ulClk = 32768;
    1c94:	f44f 4300 	mov.w	r3, #32768	; 0x8000
    1c98:	613b      	str	r3, [r7, #16]
            break;
    1c9a:	e001      	b.n	1ca0 <SysCtlClockGet+0x1dc>
        // An unknown setting, so return a zero clock (that is, an unknown
        // clock rate).
        //
        default:
        {
            return(0);
    1c9c:	2300      	movs	r3, #0
    1c9e:	e0db      	b.n	1e58 <SysCtlClockGet+0x394>
    }

    //
    // See if the PLL is being used.
    //
    if(((ulRCC2 & SYSCTL_RCC2_USERCC2) && !(ulRCC2 & SYSCTL_RCC2_BYPASS2)) ||
    1ca0:	68fb      	ldr	r3, [r7, #12]
    1ca2:	2b00      	cmp	r3, #0
    1ca4:	da04      	bge.n	1cb0 <SysCtlClockGet+0x1ec>
    1ca6:	68fb      	ldr	r3, [r7, #12]
    1ca8:	f403 6300 	and.w	r3, r3, #2048	; 0x800
    1cac:	2b00      	cmp	r3, #0
    1cae:	d009      	beq.n	1cc4 <SysCtlClockGet+0x200>
       (!(ulRCC2 & SYSCTL_RCC2_USERCC2) && !(ulRCC & SYSCTL_RCC_BYPASS)))
    1cb0:	68fb      	ldr	r3, [r7, #12]
    }

    //
    // See if the PLL is being used.
    //
    if(((ulRCC2 & SYSCTL_RCC2_USERCC2) && !(ulRCC2 & SYSCTL_RCC2_BYPASS2)) ||
    1cb2:	2b00      	cmp	r3, #0
    1cb4:	f2c0 8094 	blt.w	1de0 <SysCtlClockGet+0x31c>
       (!(ulRCC2 & SYSCTL_RCC2_USERCC2) && !(ulRCC & SYSCTL_RCC_BYPASS)))
    1cb8:	697b      	ldr	r3, [r7, #20]
    1cba:	f403 6300 	and.w	r3, r3, #2048	; 0x800
    1cbe:	2b00      	cmp	r3, #0
    1cc0:	f040 808e 	bne.w	1de0 <SysCtlClockGet+0x31c>
    {
        //
        // See if this is a Blizzard-class device.
        //
        if(CLASS_IS_BLIZZARD)
    1cc4:	f44f 4360 	mov.w	r3, #57344	; 0xe000
    1cc8:	f2c4 030f 	movt	r3, #16399	; 0x400f
    1ccc:	681a      	ldr	r2, [r3, #0]
    1cce:	2300      	movs	r3, #0
    1cd0:	f2c7 03ff 	movt	r3, #28927	; 0x70ff
    1cd4:	4013      	ands	r3, r2
    1cd6:	2200      	movs	r2, #0
    1cd8:	f2c1 0205 	movt	r2, #4101	; 0x1005
    1cdc:	4293      	cmp	r3, r2
    1cde:	d12f      	bne.n	1d40 <SysCtlClockGet+0x27c>
        {
            //
            // Read the two PLL frequency registers.  The formula for a
            // Blizzard-class device is "(xtal * m) / ((q + 1) * (n + 1))".
            //
            ulPLL = HWREG(SYSCTL_PLLFREQ0);
    1ce0:	f24e 1360 	movw	r3, #57696	; 0xe160
    1ce4:	f2c4 030f 	movt	r3, #16399	; 0x400f
    1ce8:	681b      	ldr	r3, [r3, #0]
    1cea:	60bb      	str	r3, [r7, #8]
            ulPLL1 = HWREG(SYSCTL_PLLFREQ1);
    1cec:	f24e 1364 	movw	r3, #57700	; 0xe164
    1cf0:	f2c4 030f 	movt	r3, #16399	; 0x400f
    1cf4:	681b      	ldr	r3, [r3, #0]
    1cf6:	607b      	str	r3, [r7, #4]

            //
            // Divide the input clock by the dividers.
            //
            ulClk /= ((((ulPLL1 & SYSCTL_PLLFREQ1_Q_M) >>
    1cf8:	687b      	ldr	r3, [r7, #4]
    1cfa:	f403 53f8 	and.w	r3, r3, #7936	; 0x1f00
    1cfe:	0a1b      	lsrs	r3, r3, #8
                        SYSCTL_PLLFREQ1_Q_S) + 1) *
                      (((ulPLL1 & SYSCTL_PLLFREQ1_N_M) >>
                        SYSCTL_PLLFREQ1_N_S) + 1) * 2);
    1d00:	3301      	adds	r3, #1
            //
            // Divide the input clock by the dividers.
            //
            ulClk /= ((((ulPLL1 & SYSCTL_PLLFREQ1_Q_M) >>
                        SYSCTL_PLLFREQ1_Q_S) + 1) *
                      (((ulPLL1 & SYSCTL_PLLFREQ1_N_M) >>
    1d02:	687a      	ldr	r2, [r7, #4]
    1d04:	f002 021f 	and.w	r2, r2, #31
                        SYSCTL_PLLFREQ1_N_S) + 1) * 2);
    1d08:	3201      	adds	r2, #1
    1d0a:	fb02 f303 	mul.w	r3, r2, r3
    1d0e:	005b      	lsls	r3, r3, #1
            ulPLL1 = HWREG(SYSCTL_PLLFREQ1);

            //
            // Divide the input clock by the dividers.
            //
            ulClk /= ((((ulPLL1 & SYSCTL_PLLFREQ1_Q_M) >>
    1d10:	693a      	ldr	r2, [r7, #16]
    1d12:	fbb2 f3f3 	udiv	r3, r2, r3
    1d16:	613b      	str	r3, [r7, #16]

            //
            // Multiply the clock by the multiplier, which is split into an
            // integer part and a fractional part.
            //
            ulClk = ((ulClk * ((ulPLL & SYSCTL_PLLFREQ0_MINT_M) >>
    1d18:	68bb      	ldr	r3, [r7, #8]
    1d1a:	f3c3 0309 	ubfx	r3, r3, #0, #10
    1d1e:	693a      	ldr	r2, [r7, #16]
    1d20:	fb02 f203 	mul.w	r2, r2, r3
                               SYSCTL_PLLFREQ0_MINT_S)) +
                     ((ulClk * ((ulPLL & SYSCTL_PLLFREQ0_MFRAC_M) >>
    1d24:	68b9      	ldr	r1, [r7, #8]
    1d26:	f44f 437c 	mov.w	r3, #64512	; 0xfc00
    1d2a:	f2c0 030f 	movt	r3, #15
    1d2e:	400b      	ands	r3, r1
    1d30:	0a9b      	lsrs	r3, r3, #10
    1d32:	6939      	ldr	r1, [r7, #16]
    1d34:	fb01 f303 	mul.w	r3, r1, r3
                                SYSCTL_PLLFREQ0_MFRAC_S)) >> 10));
    1d38:	0a9b      	lsrs	r3, r3, #10

            //
            // Multiply the clock by the multiplier, which is split into an
            // integer part and a fractional part.
            //
            ulClk = ((ulClk * ((ulPLL & SYSCTL_PLLFREQ0_MINT_M) >>
    1d3a:	18d3      	adds	r3, r2, r3
    1d3c:	613b      	str	r3, [r7, #16]
    1d3e:	e04b      	b.n	1dd8 <SysCtlClockGet+0x314>
        else
        {
            //
            // Get the PLL configuration.
            //
            ulPLL = HWREG(SYSCTL_PLLCFG);
    1d40:	f24e 0364 	movw	r3, #57444	; 0xe064
    1d44:	f2c4 030f 	movt	r3, #16399	; 0x400f
    1d48:	681b      	ldr	r3, [r3, #0]
    1d4a:	60bb      	str	r3, [r7, #8]

            //
            // See if this is a Sandstorm-class or Fury-class device.
            //
            if(CLASS_IS_SANDSTORM)
    1d4c:	f44f 4360 	mov.w	r3, #57344	; 0xe000
    1d50:	f2c4 030f 	movt	r3, #16399	; 0x400f
    1d54:	681b      	ldr	r3, [r3, #0]
    1d56:	f003 43e0 	and.w	r3, r3, #1879048192	; 0x70000000
    1d5a:	2b00      	cmp	r3, #0
    1d5c:	d00b      	beq.n	1d76 <SysCtlClockGet+0x2b2>
    1d5e:	f44f 4360 	mov.w	r3, #57344	; 0xe000
    1d62:	f2c4 030f 	movt	r3, #16399	; 0x400f
    1d66:	681a      	ldr	r2, [r3, #0]
    1d68:	2300      	movs	r3, #0
    1d6a:	f2c7 03ff 	movt	r3, #28927	; 0x70ff
    1d6e:	4013      	ands	r3, r2
    1d70:	f1b3 5f80 	cmp.w	r3, #268435456	; 0x10000000
    1d74:	d110      	bne.n	1d98 <SysCtlClockGet+0x2d4>
                //
                // Compute the PLL output frequency based on its input
                // frequency.  The formula for a Sandstorm-class devices is
                // "(xtal * (f + 2)) / (r + 2)".
                //
                ulClk = ((ulClk * (((ulPLL & SYSCTL_PLLCFG_F_M) >>
    1d76:	68ba      	ldr	r2, [r7, #8]
    1d78:	f643 73e0 	movw	r3, #16352	; 0x3fe0
    1d7c:	4013      	ands	r3, r2
    1d7e:	095b      	lsrs	r3, r3, #5
                                    SYSCTL_PLLCFG_F_S) + 2)) /
    1d80:	3302      	adds	r3, #2
                //
                // Compute the PLL output frequency based on its input
                // frequency.  The formula for a Sandstorm-class devices is
                // "(xtal * (f + 2)) / (r + 2)".
                //
                ulClk = ((ulClk * (((ulPLL & SYSCTL_PLLCFG_F_M) >>
    1d82:	693a      	ldr	r2, [r7, #16]
    1d84:	fb02 f203 	mul.w	r2, r2, r3
                                    SYSCTL_PLLCFG_F_S) + 2)) /
                         (((ulPLL & SYSCTL_PLLCFG_R_M) >>
    1d88:	68bb      	ldr	r3, [r7, #8]
    1d8a:	f003 031f 	and.w	r3, r3, #31
                           SYSCTL_PLLCFG_R_S) + 2));
    1d8e:	3302      	adds	r3, #2
                //
                // Compute the PLL output frequency based on its input
                // frequency.  The formula for a Sandstorm-class devices is
                // "(xtal * (f + 2)) / (r + 2)".
                //
                ulClk = ((ulClk * (((ulPLL & SYSCTL_PLLCFG_F_M) >>
    1d90:	fbb2 f3f3 	udiv	r3, r2, r3
    1d94:	613b      	str	r3, [r7, #16]
    1d96:	e00f      	b.n	1db8 <SysCtlClockGet+0x2f4>
                //
                // Compute the PLL output frequency based on its input
                // frequency.  The formula for a Fury-class device is
                // "(xtal * f) / ((r + 1) * 2)".
                //
                ulClk = ((ulClk * ((ulPLL & SYSCTL_PLLCFG_F_M) >>
    1d98:	68ba      	ldr	r2, [r7, #8]
    1d9a:	f643 73e0 	movw	r3, #16352	; 0x3fe0
    1d9e:	4013      	ands	r3, r2
    1da0:	095b      	lsrs	r3, r3, #5
    1da2:	693a      	ldr	r2, [r7, #16]
    1da4:	fb02 f203 	mul.w	r2, r2, r3
                                   SYSCTL_PLLCFG_F_S)) /
                         ((((ulPLL & SYSCTL_PLLCFG_R_M) >>
    1da8:	68bb      	ldr	r3, [r7, #8]
    1daa:	f003 031f 	and.w	r3, r3, #31
                            SYSCTL_PLLCFG_R_S) + 1) * 2));
    1dae:	3301      	adds	r3, #1
    1db0:	005b      	lsls	r3, r3, #1
                //
                // Compute the PLL output frequency based on its input
                // frequency.  The formula for a Fury-class device is
                // "(xtal * f) / ((r + 1) * 2)".
                //
                ulClk = ((ulClk * ((ulPLL & SYSCTL_PLLCFG_F_M) >>
    1db2:	fbb2 f3f3 	udiv	r3, r2, r3
    1db6:	613b      	str	r3, [r7, #16]
            }

            //
            // See if the optional output divide by 2 is being used.
            //
            if(ulPLL & SYSCTL_PLLCFG_OD_2)
    1db8:	68bb      	ldr	r3, [r7, #8]
    1dba:	f403 4380 	and.w	r3, r3, #16384	; 0x4000
    1dbe:	2b00      	cmp	r3, #0
    1dc0:	d002      	beq.n	1dc8 <SysCtlClockGet+0x304>
            {
                ulClk /= 2;
    1dc2:	693b      	ldr	r3, [r7, #16]
    1dc4:	085b      	lsrs	r3, r3, #1
    1dc6:	613b      	str	r3, [r7, #16]
            }

            //
            // See if the optional output divide by 4 is being used.
            //
            if(ulPLL & SYSCTL_PLLCFG_OD_4)
    1dc8:	68bb      	ldr	r3, [r7, #8]
    1dca:	f403 4300 	and.w	r3, r3, #32768	; 0x8000
    1dce:	2b00      	cmp	r3, #0
    1dd0:	d002      	beq.n	1dd8 <SysCtlClockGet+0x314>
            {
                ulClk /= 4;
    1dd2:	693b      	ldr	r3, [r7, #16]
    1dd4:	089b      	lsrs	r3, r3, #2
    1dd6:	613b      	str	r3, [r7, #16]

        //
        // Force the system divider to be enabled.  It is always used when
        // using the PLL, but in some cases it does not read as being enabled.
        //
        ulRCC |= SYSCTL_RCC_USESYSDIV;
    1dd8:	697b      	ldr	r3, [r7, #20]
    1dda:	f443 0380 	orr.w	r3, r3, #4194304	; 0x400000
    1dde:	617b      	str	r3, [r7, #20]
    }

    //
    // See if the system divider is being used.
    //
    if(ulRCC & SYSCTL_RCC_USESYSDIV)
    1de0:	697b      	ldr	r3, [r7, #20]
    1de2:	f403 0380 	and.w	r3, r3, #4194304	; 0x400000
    1de6:	2b00      	cmp	r3, #0
    1de8:	d035      	beq.n	1e56 <SysCtlClockGet+0x392>
    {
        //
        // Adjust the clock rate by the system clock divider.
        //
        if(ulRCC2 & SYSCTL_RCC2_USERCC2)
    1dea:	68fb      	ldr	r3, [r7, #12]
    1dec:	2b00      	cmp	r3, #0
    1dee:	da29      	bge.n	1e44 <SysCtlClockGet+0x380>
        {
            if((ulRCC2 & SYSCTL_RCC2_DIV400) &&
    1df0:	68fb      	ldr	r3, [r7, #12]
    1df2:	f003 4380 	and.w	r3, r3, #1073741824	; 0x40000000
    1df6:	2b00      	cmp	r3, #0
    1df8:	d01a      	beq.n	1e30 <SysCtlClockGet+0x36c>
               (((ulRCC2 & SYSCTL_RCC2_USERCC2) &&
    1dfa:	68fb      	ldr	r3, [r7, #12]
        //
        // Adjust the clock rate by the system clock divider.
        //
        if(ulRCC2 & SYSCTL_RCC2_USERCC2)
        {
            if((ulRCC2 & SYSCTL_RCC2_DIV400) &&
    1dfc:	2b00      	cmp	r3, #0
    1dfe:	da04      	bge.n	1e0a <SysCtlClockGet+0x346>
               (((ulRCC2 & SYSCTL_RCC2_USERCC2) &&
                 !(ulRCC2 & SYSCTL_RCC2_BYPASS2)) ||
    1e00:	68fb      	ldr	r3, [r7, #12]
    1e02:	f403 6300 	and.w	r3, r3, #2048	; 0x800
        // Adjust the clock rate by the system clock divider.
        //
        if(ulRCC2 & SYSCTL_RCC2_USERCC2)
        {
            if((ulRCC2 & SYSCTL_RCC2_DIV400) &&
               (((ulRCC2 & SYSCTL_RCC2_USERCC2) &&
    1e06:	2b00      	cmp	r3, #0
    1e08:	d007      	beq.n	1e1a <SysCtlClockGet+0x356>
                 !(ulRCC2 & SYSCTL_RCC2_BYPASS2)) ||
                (!(ulRCC2 & SYSCTL_RCC2_USERCC2) &&
    1e0a:	68fb      	ldr	r3, [r7, #12]
        //
        if(ulRCC2 & SYSCTL_RCC2_USERCC2)
        {
            if((ulRCC2 & SYSCTL_RCC2_DIV400) &&
               (((ulRCC2 & SYSCTL_RCC2_USERCC2) &&
                 !(ulRCC2 & SYSCTL_RCC2_BYPASS2)) ||
    1e0c:	2b00      	cmp	r3, #0
    1e0e:	db0f      	blt.n	1e30 <SysCtlClockGet+0x36c>
                (!(ulRCC2 & SYSCTL_RCC2_USERCC2) &&
                 !(ulRCC & SYSCTL_RCC_BYPASS))))
    1e10:	697b      	ldr	r3, [r7, #20]
    1e12:	f403 6300 	and.w	r3, r3, #2048	; 0x800
        if(ulRCC2 & SYSCTL_RCC2_USERCC2)
        {
            if((ulRCC2 & SYSCTL_RCC2_DIV400) &&
               (((ulRCC2 & SYSCTL_RCC2_USERCC2) &&
                 !(ulRCC2 & SYSCTL_RCC2_BYPASS2)) ||
                (!(ulRCC2 & SYSCTL_RCC2_USERCC2) &&
    1e16:	2b00      	cmp	r3, #0
    1e18:	d10a      	bne.n	1e30 <SysCtlClockGet+0x36c>
                 !(ulRCC & SYSCTL_RCC_BYPASS))))

            {
                ulClk = ((ulClk * 2) / (((ulRCC2 & (SYSCTL_RCC2_SYSDIV2_M |
    1e1a:	693b      	ldr	r3, [r7, #16]
    1e1c:	005a      	lsls	r2, r3, #1
    1e1e:	68fb      	ldr	r3, [r7, #12]
    1e20:	f003 53fe 	and.w	r3, r3, #532676608	; 0x1fc00000
                                                    SYSCTL_RCC2_SYSDIV2LSB)) >>
    1e24:	0d9b      	lsrs	r3, r3, #22
                                         (SYSCTL_RCC2_SYSDIV2_S - 1)) + 1));
    1e26:	3301      	adds	r3, #1
                 !(ulRCC2 & SYSCTL_RCC2_BYPASS2)) ||
                (!(ulRCC2 & SYSCTL_RCC2_USERCC2) &&
                 !(ulRCC & SYSCTL_RCC_BYPASS))))

            {
                ulClk = ((ulClk * 2) / (((ulRCC2 & (SYSCTL_RCC2_SYSDIV2_M |
    1e28:	fbb2 f3f3 	udiv	r3, r2, r3
    1e2c:	613b      	str	r3, [r7, #16]
    1e2e:	e012      	b.n	1e56 <SysCtlClockGet+0x392>
                                                    SYSCTL_RCC2_SYSDIV2LSB)) >>
                                         (SYSCTL_RCC2_SYSDIV2_S - 1)) + 1));
            }
            else
            {
                ulClk /= (((ulRCC2 & SYSCTL_RCC2_SYSDIV2_M) >>
    1e30:	68fb      	ldr	r3, [r7, #12]
    1e32:	f003 53fc 	and.w	r3, r3, #528482304	; 0x1f800000
    1e36:	0ddb      	lsrs	r3, r3, #23
                           SYSCTL_RCC2_SYSDIV2_S) + 1);
    1e38:	3301      	adds	r3, #1
                                                    SYSCTL_RCC2_SYSDIV2LSB)) >>
                                         (SYSCTL_RCC2_SYSDIV2_S - 1)) + 1));
            }
            else
            {
                ulClk /= (((ulRCC2 & SYSCTL_RCC2_SYSDIV2_M) >>
    1e3a:	693a      	ldr	r2, [r7, #16]
    1e3c:	fbb2 f3f3 	udiv	r3, r2, r3
    1e40:	613b      	str	r3, [r7, #16]
    1e42:	e008      	b.n	1e56 <SysCtlClockGet+0x392>
                           SYSCTL_RCC2_SYSDIV2_S) + 1);
            }
        }
        else
        {
            ulClk /= (((ulRCC & SYSCTL_RCC_SYSDIV_M) >> SYSCTL_RCC_SYSDIV_S) +
    1e44:	697b      	ldr	r3, [r7, #20]
    1e46:	f003 63f0 	and.w	r3, r3, #125829120	; 0x7800000
    1e4a:	0ddb      	lsrs	r3, r3, #23
    1e4c:	3301      	adds	r3, #1
    1e4e:	693a      	ldr	r2, [r7, #16]
    1e50:	fbb2 f3f3 	udiv	r3, r2, r3
    1e54:	613b      	str	r3, [r7, #16]
    }

    //
    // Return the computed clock rate.
    //
    return(ulClk);
    1e56:	693b      	ldr	r3, [r7, #16]
}
    1e58:	4618      	mov	r0, r3
    1e5a:	f107 071c 	add.w	r7, r7, #28
    1e5e:	46bd      	mov	sp, r7
    1e60:	bc80      	pop	{r7}
    1e62:	4770      	bx	lr

00001e64 <SysTickEnable>:
//! \return None.
//
//*****************************************************************************
void
SysTickEnable(void)
{
    1e64:	b480      	push	{r7}
    1e66:	af00      	add	r7, sp, #0
    //
    // Enable SysTick.
    //
    HWREG(NVIC_ST_CTRL) |= NVIC_ST_CTRL_CLK_SRC | NVIC_ST_CTRL_ENABLE;
    1e68:	f24e 0310 	movw	r3, #57360	; 0xe010
    1e6c:	f2ce 0300 	movt	r3, #57344	; 0xe000
    1e70:	f24e 0210 	movw	r2, #57360	; 0xe010
    1e74:	f2ce 0200 	movt	r2, #57344	; 0xe000
    1e78:	6812      	ldr	r2, [r2, #0]
    1e7a:	f042 0205 	orr.w	r2, r2, #5
    1e7e:	601a      	str	r2, [r3, #0]
}
    1e80:	46bd      	mov	sp, r7
    1e82:	bc80      	pop	{r7}
    1e84:	4770      	bx	lr
    1e86:	bf00      	nop

00001e88 <SysTickIntEnable>:
//! \return None.
//
//*****************************************************************************
void
SysTickIntEnable(void)
{
    1e88:	b480      	push	{r7}
    1e8a:	af00      	add	r7, sp, #0
    //
    // Enable the SysTick interrupt.
    //
    HWREG(NVIC_ST_CTRL) |= NVIC_ST_CTRL_INTEN;
    1e8c:	f24e 0310 	movw	r3, #57360	; 0xe010
    1e90:	f2ce 0300 	movt	r3, #57344	; 0xe000
    1e94:	f24e 0210 	movw	r2, #57360	; 0xe010
    1e98:	f2ce 0200 	movt	r2, #57344	; 0xe000
    1e9c:	6812      	ldr	r2, [r2, #0]
    1e9e:	f042 0202 	orr.w	r2, r2, #2
    1ea2:	601a      	str	r2, [r3, #0]
}
    1ea4:	46bd      	mov	sp, r7
    1ea6:	bc80      	pop	{r7}
    1ea8:	4770      	bx	lr
    1eaa:	bf00      	nop

00001eac <SysTickPeriodSet>:
//! \return None.
//
//*****************************************************************************
void
SysTickPeriodSet(unsigned long ulPeriod)
{
    1eac:	b480      	push	{r7}
    1eae:	b083      	sub	sp, #12
    1eb0:	af00      	add	r7, sp, #0
    1eb2:	6078      	str	r0, [r7, #4]
    ASSERT((ulPeriod > 0) && (ulPeriod <= 16777216));

    //
    // Set the period of the SysTick counter.
    //
    HWREG(NVIC_ST_RELOAD) = ulPeriod - 1;
    1eb4:	f24e 0314 	movw	r3, #57364	; 0xe014
    1eb8:	f2ce 0300 	movt	r3, #57344	; 0xe000
    1ebc:	687a      	ldr	r2, [r7, #4]
    1ebe:	3a01      	subs	r2, #1
    1ec0:	601a      	str	r2, [r3, #0]
}
    1ec2:	f107 070c 	add.w	r7, r7, #12
    1ec6:	46bd      	mov	sp, r7
    1ec8:	bc80      	pop	{r7}
    1eca:	4770      	bx	lr

00001ecc <TimerIntNumberGet>:
//! \return Returns a timer interrupt number, or -1 if \e ulBase is invalid.
//
//*****************************************************************************
static long
TimerIntNumberGet(unsigned long ulBase)
{
    1ecc:	b480      	push	{r7}
    1ece:	b085      	sub	sp, #20
    1ed0:	af00      	add	r7, sp, #0
    1ed2:	6078      	str	r0, [r7, #4]

    //
    // Loop through the table that maps timer base addresses to interrupt
    // numbers.
    //
    for(ulIdx = 0; ulIdx < (sizeof(g_ppulTimerIntMap) /
    1ed4:	2300      	movs	r3, #0
    1ed6:	60fb      	str	r3, [r7, #12]
    1ed8:	e015      	b.n	1f06 <TimerIntNumberGet+0x3a>
                            sizeof(g_ppulTimerIntMap[0])); ulIdx++)
    {
        //
        // See if this base address matches.
        //
        if(g_ppulTimerIntMap[ulIdx][0] == ulBase)
    1eda:	f242 23b0 	movw	r3, #8880	; 0x22b0
    1ede:	f2c0 0300 	movt	r3, #0
    1ee2:	68fa      	ldr	r2, [r7, #12]
    1ee4:	f853 2032 	ldr.w	r2, [r3, r2, lsl #3]
    1ee8:	687b      	ldr	r3, [r7, #4]
    1eea:	429a      	cmp	r2, r3
    1eec:	d108      	bne.n	1f00 <TimerIntNumberGet+0x34>
        {
            //
            // Return the corresponding interrupt number.
            //
            return(g_ppulTimerIntMap[ulIdx][1]);
    1eee:	f242 22b0 	movw	r2, #8880	; 0x22b0
    1ef2:	f2c0 0200 	movt	r2, #0
    1ef6:	68fb      	ldr	r3, [r7, #12]
    1ef8:	00db      	lsls	r3, r3, #3
    1efa:	18d3      	adds	r3, r2, r3
    1efc:	685b      	ldr	r3, [r3, #4]
    1efe:	e007      	b.n	1f10 <TimerIntNumberGet+0x44>
    //
    // Loop through the table that maps timer base addresses to interrupt
    // numbers.
    //
    for(ulIdx = 0; ulIdx < (sizeof(g_ppulTimerIntMap) /
                            sizeof(g_ppulTimerIntMap[0])); ulIdx++)
    1f00:	68fb      	ldr	r3, [r7, #12]
    1f02:	3301      	adds	r3, #1
    1f04:	60fb      	str	r3, [r7, #12]

    //
    // Loop through the table that maps timer base addresses to interrupt
    // numbers.
    //
    for(ulIdx = 0; ulIdx < (sizeof(g_ppulTimerIntMap) /
    1f06:	68fb      	ldr	r3, [r7, #12]
    1f08:	2b0b      	cmp	r3, #11
    1f0a:	d9e6      	bls.n	1eda <TimerIntNumberGet+0xe>
    }

    //
    // The base address could not be found, so return an error.
    //
    return(-1);
    1f0c:	f04f 33ff 	mov.w	r3, #4294967295	; 0xffffffff
}
    1f10:	4618      	mov	r0, r3
    1f12:	f107 0714 	add.w	r7, r7, #20
    1f16:	46bd      	mov	sp, r7
    1f18:	bc80      	pop	{r7}
    1f1a:	4770      	bx	lr

00001f1c <TimerEnable>:
//! \return None.
//
//*****************************************************************************
void
TimerEnable(unsigned long ulBase, unsigned long ulTimer)
{
    1f1c:	b480      	push	{r7}
    1f1e:	b083      	sub	sp, #12
    1f20:	af00      	add	r7, sp, #0
    1f22:	6078      	str	r0, [r7, #4]
    1f24:	6039      	str	r1, [r7, #0]
           (ulTimer == TIMER_BOTH));

    //
    // Enable the timer(s) module.
    //
    HWREG(ulBase + TIMER_O_CTL) |= ulTimer & (TIMER_CTL_TAEN | TIMER_CTL_TBEN);
    1f26:	687b      	ldr	r3, [r7, #4]
    1f28:	330c      	adds	r3, #12
    1f2a:	461a      	mov	r2, r3
    1f2c:	687b      	ldr	r3, [r7, #4]
    1f2e:	330c      	adds	r3, #12
    1f30:	6819      	ldr	r1, [r3, #0]
    1f32:	6838      	ldr	r0, [r7, #0]
    1f34:	f240 1301 	movw	r3, #257	; 0x101
    1f38:	4003      	ands	r3, r0
    1f3a:	430b      	orrs	r3, r1
    1f3c:	6013      	str	r3, [r2, #0]
}
    1f3e:	f107 070c 	add.w	r7, r7, #12
    1f42:	46bd      	mov	sp, r7
    1f44:	bc80      	pop	{r7}
    1f46:	4770      	bx	lr

00001f48 <TimerConfigure>:
//! \return None.
//
//*****************************************************************************
void
TimerConfigure(unsigned long ulBase, unsigned long ulConfig)
{
    1f48:	b480      	push	{r7}
    1f4a:	b083      	sub	sp, #12
    1f4c:	af00      	add	r7, sp, #0
    1f4e:	6078      	str	r0, [r7, #4]
    1f50:	6039      	str	r1, [r7, #0]
             ((ulConfig & 0x0000ff00) == TIMER_CFG_B_PWM))));

    //
    // Disable the timers.
    //
    HWREG(ulBase + TIMER_O_CTL) &= ~(TIMER_CTL_TAEN | TIMER_CTL_TBEN);
    1f52:	687b      	ldr	r3, [r7, #4]
    1f54:	330c      	adds	r3, #12
    1f56:	461a      	mov	r2, r3
    1f58:	687b      	ldr	r3, [r7, #4]
    1f5a:	330c      	adds	r3, #12
    1f5c:	681b      	ldr	r3, [r3, #0]
    1f5e:	f423 7380 	bic.w	r3, r3, #256	; 0x100
    1f62:	f023 0301 	bic.w	r3, r3, #1
    1f66:	6013      	str	r3, [r2, #0]

    //
    // Set the global timer configuration.
    //
    HWREG(ulBase + TIMER_O_CFG) = ulConfig >> 24;
    1f68:	687b      	ldr	r3, [r7, #4]
    1f6a:	683a      	ldr	r2, [r7, #0]
    1f6c:	0e12      	lsrs	r2, r2, #24
    1f6e:	601a      	str	r2, [r3, #0]

    //
    // Set the configuration of the A and B timers.  Note that the B timer
    // configuration is ignored by the hardware in 32-bit modes.
    //
    HWREG(ulBase + TIMER_O_TAMR) = (ulConfig & 255) | TIMER_TAMR_TAPWMIE;
    1f70:	687b      	ldr	r3, [r7, #4]
    1f72:	3304      	adds	r3, #4
    1f74:	683a      	ldr	r2, [r7, #0]
    1f76:	b2d2      	uxtb	r2, r2
    1f78:	f442 7200 	orr.w	r2, r2, #512	; 0x200
    1f7c:	601a      	str	r2, [r3, #0]
    HWREG(ulBase + TIMER_O_TBMR) =
    1f7e:	687b      	ldr	r3, [r7, #4]
    1f80:	3308      	adds	r3, #8
        ((ulConfig >> 8) & 255) | TIMER_TBMR_TBPWMIE;
    1f82:	683a      	ldr	r2, [r7, #0]
    1f84:	0a12      	lsrs	r2, r2, #8
    1f86:	b2d2      	uxtb	r2, r2
    1f88:	f442 7200 	orr.w	r2, r2, #512	; 0x200
    //
    // Set the configuration of the A and B timers.  Note that the B timer
    // configuration is ignored by the hardware in 32-bit modes.
    //
    HWREG(ulBase + TIMER_O_TAMR) = (ulConfig & 255) | TIMER_TAMR_TAPWMIE;
    HWREG(ulBase + TIMER_O_TBMR) =
    1f8c:	601a      	str	r2, [r3, #0]
        ((ulConfig >> 8) & 255) | TIMER_TBMR_TBPWMIE;
}
    1f8e:	f107 070c 	add.w	r7, r7, #12
    1f92:	46bd      	mov	sp, r7
    1f94:	bc80      	pop	{r7}
    1f96:	4770      	bx	lr

00001f98 <TimerControlEvent>:
//
//*****************************************************************************
void
TimerControlEvent(unsigned long ulBase, unsigned long ulTimer,
                  unsigned long ulEvent)
{
    1f98:	b480      	push	{r7}
    1f9a:	b085      	sub	sp, #20
    1f9c:	af00      	add	r7, sp, #0
    1f9e:	60f8      	str	r0, [r7, #12]
    1fa0:	60b9      	str	r1, [r7, #8]
    1fa2:	607a      	str	r2, [r7, #4]
           (ulTimer == TIMER_BOTH));

    //
    // Set the event type.
    //
    ulTimer &= TIMER_CTL_TAEVENT_M | TIMER_CTL_TBEVENT_M;
    1fa4:	68ba      	ldr	r2, [r7, #8]
    1fa6:	f640 430c 	movw	r3, #3084	; 0xc0c
    1faa:	4013      	ands	r3, r2
    1fac:	60bb      	str	r3, [r7, #8]
    HWREG(ulBase + TIMER_O_CTL) = ((HWREG(ulBase + TIMER_O_CTL) & ~ulTimer) |
    1fae:	68fb      	ldr	r3, [r7, #12]
    1fb0:	330c      	adds	r3, #12
    1fb2:	68fa      	ldr	r2, [r7, #12]
    1fb4:	320c      	adds	r2, #12
    1fb6:	6811      	ldr	r1, [r2, #0]
    1fb8:	68ba      	ldr	r2, [r7, #8]
    1fba:	43d2      	mvns	r2, r2
    1fbc:	4011      	ands	r1, r2
                                   (ulEvent & ulTimer));
    1fbe:	6878      	ldr	r0, [r7, #4]
    1fc0:	68ba      	ldr	r2, [r7, #8]
    1fc2:	4002      	ands	r2, r0

    //
    // Set the event type.
    //
    ulTimer &= TIMER_CTL_TAEVENT_M | TIMER_CTL_TBEVENT_M;
    HWREG(ulBase + TIMER_O_CTL) = ((HWREG(ulBase + TIMER_O_CTL) & ~ulTimer) |
    1fc4:	430a      	orrs	r2, r1
    1fc6:	601a      	str	r2, [r3, #0]
                                   (ulEvent & ulTimer));
}
    1fc8:	f107 0714 	add.w	r7, r7, #20
    1fcc:	46bd      	mov	sp, r7
    1fce:	bc80      	pop	{r7}
    1fd0:	4770      	bx	lr
    1fd2:	bf00      	nop

00001fd4 <TimerControlStall>:
//
//*****************************************************************************
void
TimerControlStall(unsigned long ulBase, unsigned long ulTimer,
                  tBoolean bStall)
{
    1fd4:	b480      	push	{r7}
    1fd6:	b085      	sub	sp, #20
    1fd8:	af00      	add	r7, sp, #0
    1fda:	60f8      	str	r0, [r7, #12]
    1fdc:	60b9      	str	r1, [r7, #8]
    1fde:	4613      	mov	r3, r2
    1fe0:	71fb      	strb	r3, [r7, #7]
           (ulTimer == TIMER_BOTH));

    //
    // Set the stall mode.
    //
    ulTimer &= TIMER_CTL_TASTALL | TIMER_CTL_TBSTALL;
    1fe2:	68ba      	ldr	r2, [r7, #8]
    1fe4:	f240 2302 	movw	r3, #514	; 0x202
    1fe8:	4013      	ands	r3, r2
    1fea:	60bb      	str	r3, [r7, #8]
    HWREG(ulBase + TIMER_O_CTL) = (bStall ?
    1fec:	68fb      	ldr	r3, [r7, #12]
    1fee:	330c      	adds	r3, #12
    1ff0:	461a      	mov	r2, r3
                                   (HWREG(ulBase + TIMER_O_CTL) | ulTimer) :
    1ff2:	79fb      	ldrb	r3, [r7, #7]
    1ff4:	2b00      	cmp	r3, #0
    1ff6:	d005      	beq.n	2004 <TimerControlStall+0x30>
    1ff8:	68fb      	ldr	r3, [r7, #12]
    1ffa:	330c      	adds	r3, #12
    1ffc:	6819      	ldr	r1, [r3, #0]
    1ffe:	68bb      	ldr	r3, [r7, #8]
    2000:	430b      	orrs	r3, r1
    2002:	e005      	b.n	2010 <TimerControlStall+0x3c>
                                   (HWREG(ulBase + TIMER_O_CTL) & ~(ulTimer)));
    2004:	68fb      	ldr	r3, [r7, #12]
    2006:	330c      	adds	r3, #12
    2008:	6819      	ldr	r1, [r3, #0]
    200a:	68bb      	ldr	r3, [r7, #8]
    200c:	43db      	mvns	r3, r3
    //
    // Set the stall mode.
    //
    ulTimer &= TIMER_CTL_TASTALL | TIMER_CTL_TBSTALL;
    HWREG(ulBase + TIMER_O_CTL) = (bStall ?
                                   (HWREG(ulBase + TIMER_O_CTL) | ulTimer) :
    200e:	400b      	ands	r3, r1

    //
    // Set the stall mode.
    //
    ulTimer &= TIMER_CTL_TASTALL | TIMER_CTL_TBSTALL;
    HWREG(ulBase + TIMER_O_CTL) = (bStall ?
    2010:	6013      	str	r3, [r2, #0]
                                   (HWREG(ulBase + TIMER_O_CTL) | ulTimer) :
                                   (HWREG(ulBase + TIMER_O_CTL) & ~(ulTimer)));
}
    2012:	f107 0714 	add.w	r7, r7, #20
    2016:	46bd      	mov	sp, r7
    2018:	bc80      	pop	{r7}
    201a:	4770      	bx	lr

0000201c <TimerLoadSet>:
//
//*****************************************************************************
void
TimerLoadSet(unsigned long ulBase, unsigned long ulTimer,
             unsigned long ulValue)
{
    201c:	b480      	push	{r7}
    201e:	b085      	sub	sp, #20
    2020:	af00      	add	r7, sp, #0
    2022:	60f8      	str	r0, [r7, #12]
    2024:	60b9      	str	r1, [r7, #8]
    2026:	607a      	str	r2, [r7, #4]
           (ulTimer == TIMER_BOTH));

    //
    // Set the timer A load value if requested.
    //
    if(ulTimer & TIMER_A)
    2028:	68bb      	ldr	r3, [r7, #8]
    202a:	b2db      	uxtb	r3, r3
    202c:	2b00      	cmp	r3, #0
    202e:	d003      	beq.n	2038 <TimerLoadSet+0x1c>
    {
        HWREG(ulBase + TIMER_O_TAILR) = ulValue;
    2030:	68fb      	ldr	r3, [r7, #12]
    2032:	3328      	adds	r3, #40	; 0x28
    2034:	687a      	ldr	r2, [r7, #4]
    2036:	601a      	str	r2, [r3, #0]
    }

    //
    // Set the timer B load value if requested.
    //
